 SameFolder

 Timestamp is 5dd493b9 (Wed Nov 20 04:15:37 2019)

 Preferred load address is 0000000180000000

 Start         Length     Name                   Class
 0001:00000000 00000008H .CRT$XCA                CODE
 0001:00000008 00000008H .CRT$XCZ                CODE
 0001:00000010 00000008H .CRT$XIA                CODE
 0001:00000018 00000018H .CRT$XIC                CODE
 0001:00000030 00000008H .CRT$XIZ                CODE
 0001:00000038 00000008H .CRT$XPA                CODE
 0001:00000040 00000010H .CRT$XPX                CODE
 0001:00000050 00000008H .CRT$XPXA               CODE
 0001:00000058 00000008H .CRT$XPZ                CODE
 0001:00000060 00000008H .CRT$XTA                CODE
 0001:00000068 00000008H .CRT$XTZ                CODE
 0001:00000070 00000000H .gfids$y                CODE
 0001:00000070 00007410H .rdata                  CODE
 0001:00007480 000001f4H .rdata$r                CODE
 0001:00007674 000002b4H .rdata$zzzdbg           CODE
 0001:00007928 00000008H .rtc$IAA                CODE
 0001:00007930 00000008H .rtc$IZZ                CODE
 0001:00007938 00000008H .rtc$TAA                CODE
 0001:00007940 00000010H .rtc$TZZ                CODE
 0001:00007950 0000cb00H .text$mn                CODE
 0001:00014450 00000020H .text$mn$00             CODE
 0001:00014470 00000250H .text$x                 CODE
 0001:000146c0 00000ca8H .xdata                  CODE
 0001:00015368 000000f8H .xdata$x                CODE
 0001:00015460 000000a8H .edata                  CODE
 0002:00000000 000009f0H .data                   DATA
 0002:000009f0 000000a0H .data$r                 DATA
 0002:00000a90 000014a0H .bss                    DATA
 0003:00000000 00000f90H .pdata                  DATA
 0004:00000000 00000230H .idata$5                DATA
 0004:00000230 00000010H .00cfg                  DATA
 0004:00000240 00000014H .idata$2                DATA
 0004:00000254 00000014H .idata$3                DATA
 0004:00000268 00000230H .idata$4                DATA
 0004:00000498 0000050eH .idata$6                DATA
 0005:00000000 00000060H .rsrc$01                DATA
 0005:00000060 00000388H .rsrc$02                DATA

  Address         Publics by Value              Rva+Base               Lib:Object

 0000:00000000       __hybrid_code_map_count    0000000000000000     <absolute>
 0000:00000000       __hybrid_code_map          0000000000000000     <absolute>
 0000:00000000       __guard_iat_count          0000000000000000     <absolute>
 0000:00000000       __volatile_metadata        0000000000000000     <absolute>
 0000:00000000       __guard_longjmp_count      0000000000000000     <absolute>
 0000:00000000       __guard_longjmp_table      0000000000000000     <absolute>
 0000:00000000       __guard_iat_table          0000000000000000     <absolute>
 0000:00000000       __guard_fids_count         0000000000000000     <absolute>
 0000:00000000       ___safe_se_handler_count   0000000000000000     <absolute>
 0000:00000000       __enclave_config           0000000000000000     <absolute>
 0000:00000000       ___safe_se_handler_table   0000000000000000     <absolute>
 0000:00000000       __guard_fids_table         0000000000000000     <absolute>
 0000:00000000       __hybrid_auxiliary_iat     0000000000000000     <absolute>
 0000:00000000       __dynamic_value_reloc_table 0000000000000000     <absolute>
 0000:00000100       __guard_flags              0000000000000100     <absolute>
 0000:00000000       __ImageBase                0000000180000000     <linker-defined>
 0001:00000000       __xc_a                     0000000180001000     LIBCMT:initializers.obj
 0001:00000008       __xc_z                     0000000180001008     LIBCMT:initializers.obj
 0001:00000010       __xi_a                     0000000180001010     LIBCMT:initializers.obj
 0001:00000018       __acrt_multibyte_initializer 0000000180001018     libucrt:multibyte_initializer.obj
 0001:00000020       __acrt_stdio_initializer   0000000180001020     libucrt:stdio_initializer.obj
 0001:00000028       __acrt_tran_fma3_initializer 0000000180001028     libucrt:fma3_initializer.obj
 0001:00000030       __xi_z                     0000000180001030     LIBCMT:initializers.obj
 0001:00000038       __xp_a                     0000000180001038     LIBCMT:initializers.obj
 0001:00000040       __acrt_locale_terminator   0000000180001040     libucrt:locale_initializer.obj
 0001:00000048       __dcrt_console_output_terminator 0000000180001048     libucrt:console_output_initializer.obj
 0001:00000050       __acrt_stdio_terminator    0000000180001050     libucrt:stdio_initializer.obj
 0001:00000058       __xp_z                     0000000180001058     LIBCMT:initializers.obj
 0001:00000060       __xt_a                     0000000180001060     LIBCMT:initializers.obj
 0001:00000068       __xt_z                     0000000180001068     LIBCMT:initializers.obj
 0001:00000070       MainGuid                   0000000180001070     SameFolder.obj
 0001:00000080       MenuGuid                   0000000180001080     SameFolder.obj
 0001:00000090       ConfigMenuGuid             0000000180001090     SameFolder.obj
 0001:000000a0       DialogGuid                 00000001800010a0     SameFolder.obj
 0001:000000b0       ??_C@_1BK@EJEHIDJM@?$AAA?$AAd?$AAd?$AA2?$AAP?$AAl?$AAu?$AAg?$AAM?$AAe?$AAn?$AAu@ 00000001800010b0     SameFolder.obj
 0001:000000d0       ??_C@_1BM@FDPIJPAH@?$AAA?$AAd?$AAd?$AA2?$AAD?$AAi?$AAs?$AAk?$AAs?$AAM?$AAe?$AAn?$AAu@ 00000001800010d0     SameFolder.obj
 0001:000000f0       ??_C@_1BA@CAPFOHIJ@?$AAS?$AAe?$AAt?$AAM?$AAo?$AAd?$AAe@ 00000001800010f0     SameFolder.obj
 0001:00000100       ??_7?$DialogItemBinding@UFarDialogItem@@@@6B@ 0000000180001100     SameFolder.obj
 0001:00000110       ??_7PluginCheckBoxBinding@@6B@ 0000000180001110     SameFolder.obj
 0001:00000120       ??_7PluginRadioButtonBinding@@6B@ 0000000180001120     SameFolder.obj
 0001:00000130       ??_7PluginIntEditFieldBinding@@6B@ 0000000180001130     SameFolder.obj
 0001:00000140       ??_C@_15EFLNJKHH@?$AA?$CF?$AAu@ 0000000180001140     SameFolder.obj
 0001:00000148       ??_7PluginUIntEditFieldBinding@@6B@ 0000000180001148     SameFolder.obj
 0001:00000158       ??_7?$DialogBuilderBase@UFarDialogItem@@@@6B@ 0000000180001158     SameFolder.obj
 0001:000001a0       ??_7PluginDialogBuilder@@6B@ 00000001800011a0     SameFolder.obj
 0001:000001e8       ??_C@_11LOCGONAA@@         00000001800011e8     SameFolder.obj
 0001:000001f0       ??_C@_1BG@PFMEOFNH@?$AAS?$AAa?$AAm?$AAe?$AAF?$AAo?$AAl?$AAd?$AAe?$AAr@ 00000001800011f0     SameFolder.obj
 0001:00000210       ??_C@_1EG@GJIDGPOM@?$AAS?$AAa?$AAm?$AAe?$AA?5?$AAF?$AAo?$AAl?$AAd?$AAe?$AAr?$AA?5?$AAP?$AAl?$AAu@ 0000000180001210     SameFolder.obj
 0001:00000258       ??_C@_1BE@FDJGEMIB@?$AAF?$AAa?$AAr?$AA?5?$AAG?$AAr?$AAo?$AAu?$AAp@ 0000000180001258     SameFolder.obj
 0001:00000270       ??_C@_1O@BJPKKLLM@?$AAC?$AAo?$AAn?$AAf?$AAi?$AAg@ 0000000180001270     SameFolder.obj
 0001:00000280       __xmm@ffffffffffffffff0000000000000002 0000000180001280     SameFolder.obj
 0001:00000290       __xmm@ffffffffffffffffffffffffffffffff 0000000180001290     SameFolder.obj
 0001:000002a0       _pDefaultRawDllMain        00000001800012a0     LIBCMT:dll_dllmain.obj
 0001:000002a0       _pRawDllMain               00000001800012a0     LIBCMT:dll_dllmain.obj
 0001:000002b0       ??_7exception@std@@6B@     00000001800012b0     LIBCMT:throw_bad_alloc.obj
 0001:000002c0       ??_C@_0BC@EOODALEL@Unknown?5exception@ 00000001800012c0     LIBCMT:throw_bad_alloc.obj
 0001:000002e0       ??_7bad_alloc@std@@6B@     00000001800012e0     LIBCMT:throw_bad_alloc.obj
 0001:000002f0       ??_C@_0P@GHFPNOJB@bad?5allocation@ 00000001800012f0     LIBCMT:throw_bad_alloc.obj
 0001:00000308       ??_7bad_array_new_length@std@@6B@ 0000000180001308     LIBCMT:throw_bad_alloc.obj
 0001:00000318       ??_C@_0BF@KINCDENJ@bad?5array?5new?5length@ 0000000180001318     LIBCMT:throw_bad_alloc.obj
 0001:00000338       ??_7type_info@@6B@         0000000180001338     LIBCMT:std_type_info_static.obj
 0001:00000380       _pDestructExceptionObject  0000000180001380     libvcruntime:ehhelpers.obj
 0001:000006c8       ??_C@_08EHJDFFNH@__based?$CI@ 00000001800016c8     libvcruntime:undname.obj
 0001:000006d8       ??_C@_07KOLFKCDI@__cdecl@  00000001800016d8     libvcruntime:undname.obj
 0001:000006e0       ??_C@_08GHMPAG@__pascal@   00000001800016e0     libvcruntime:undname.obj
 0001:000006f0       ??_C@_09IFJBGAPI@__stdcall@ 00000001800016f0     libvcruntime:undname.obj
 0001:00000700       ??_C@_0L@NPHFGOKO@__thiscall@ 0000000180001700     libvcruntime:undname.obj
 0001:00000710       ??_C@_0L@JMKHOMEK@__fastcall@ 0000000180001710     libvcruntime:undname.obj
 0001:00000720       ??_C@_0N@BCKKPABJ@__vectorcall@ 0000000180001720     libvcruntime:undname.obj
 0001:00000730       ??_C@_09HIJEGCPM@__clrcall@ 0000000180001730     libvcruntime:undname.obj
 0001:0000073c       ??_C@_06GHPCKEAG@__eabi@   000000018000173c     libvcruntime:undname.obj
 0001:00000748       ??_C@_09IOPIDJLG@__swift_1@ 0000000180001748     libvcruntime:undname.obj
 0001:00000758       ??_C@_09KFNFGKHF@__swift_2@ 0000000180001758     libvcruntime:undname.obj
 0001:00000768       ??_C@_07JOMMBBKO@__ptr64@  0000000180001768     libvcruntime:undname.obj
 0001:00000770       ??_C@_0L@PILCLIHE@__restrict@ 0000000180001770     libvcruntime:undname.obj
 0001:00000780       ??_C@_0M@GFIIJFMG@__unaligned@ 0000000180001780     libvcruntime:undname.obj
 0001:00000790       ??_C@_09DHDLOLLB@restrict?$CI@ 0000000180001790     libvcruntime:undname.obj
 0001:0000079a       ??_C@_00CNPNBAHC@@         000000018000179a     libvcruntime:undname.obj
 0001:0000079c       ??_C@_04NIHEBCM@?5new@     000000018000179c     libvcruntime:undname.obj
 0001:000007a8       ??_C@_07FPCDHGMM@?5delete@ 00000001800017a8     libvcruntime:undname.obj
 0001:000007b0       ??_C@_01NEMOKFLO@?$DN@     00000001800017b0     libvcruntime:undname.obj
 0001:000007b4       ??_C@_02GPIOPFAK@?$DO?$DO@ 00000001800017b4     libvcruntime:undname.obj
 0001:000007b8       ??_C@_02FODMEDOG@?$DM?$DM@ 00000001800017b8     libvcruntime:undname.obj
 0001:000007bc       ??_C@_01DCLJPIOD@?$CB@     00000001800017bc     libvcruntime:undname.obj
 0001:000007c0       ??_C@_02EGOFBIJA@?$DN?$DN@ 00000001800017c0     libvcruntime:undname.obj
 0001:000007c4       ??_C@_02FDNJECIE@?$CB?$DN@ 00000001800017c4     libvcruntime:undname.obj
 0001:000007c8       ??_C@_02GPECMEKF@?$FL?$FN@ 00000001800017c8     libvcruntime:undname.obj
 0001:000007d0       ??_C@_08LHJFAFGD@operator@ 00000001800017d0     libvcruntime:undname.obj
 0001:000007dc       ??_C@_02HBOOOICD@?9?$DO@   00000001800017dc     libvcruntime:undname.obj
 0001:000007e0       ??_C@_01NBENCBCI@?$CK@     00000001800017e0     libvcruntime:undname.obj
 0001:000007e4       ??_C@_02ECNGHCIF@?$CL?$CL@ 00000001800017e4     libvcruntime:undname.obj
 0001:000007e8       ??_C@_02BAABKJLB@?9?9@     00000001800017e8     libvcruntime:undname.obj
 0001:000007ec       ??_C@_01JOAMLHOP@?9@       00000001800017ec     libvcruntime:undname.obj
 0001:000007f0       ??_C@_01MIFGBAGJ@?$CL@     00000001800017f0     libvcruntime:undname.obj
 0001:000007f4       ??_C@_01HNPIGOCE@?$CG@     00000001800017f4     libvcruntime:undname.obj
 0001:000007f8       ??_C@_03MNHNFDLC@?9?$DO?$CK@ 00000001800017f8     libvcruntime:undname.obj
 0001:000007fc       ??_C@_01KMDKNFGN@?1@       00000001800017fc     libvcruntime:undname.obj
 0001:00000800       ??_C@_01FGNFDNOH@?$CF@     0000000180001800     libvcruntime:undname.obj
 0001:00000804       ??_C@_01MNNFJEPP@?$DM@     0000000180001804     libvcruntime:undname.obj
 0001:00000808       ??_C@_02EHCHHCKH@?$DM?$DN@ 0000000180001808     libvcruntime:undname.obj
 0001:0000080c       ??_C@_01PPODPGHN@?$DO@     000000018000180c     libvcruntime:undname.obj
 0001:00000810       ??_C@_02EEKDKGMJ@?$DO?$DN@ 0000000180001810     libvcruntime:undname.obj
 0001:00000814       ??_C@_01IHBHIGKO@?0@       0000000180001814     libvcruntime:undname.obj
 0001:00000818       ??_C@_02HCKGKOFO@?$CI?$CJ@ 0000000180001818     libvcruntime:undname.obj
 0001:0000081c       ??_C@_01PJKLJHI@?$HO@      000000018000181c     libvcruntime:undname.obj
 0001:00000820       ??_C@_01JKBOJNNK@?$FO@     0000000180001820     libvcruntime:undname.obj
 0001:00000824       ??_C@_01DNKMNLPK@?$HM@     0000000180001824     libvcruntime:undname.obj
 0001:00000828       ??_C@_02PPKAJPJL@?$CG?$CG@ 0000000180001828     libvcruntime:undname.obj
 0001:0000082c       ??_C@_02NONPIBCD@?$HM?$HM@ 000000018000182c     libvcruntime:undname.obj
 0001:00000830       ??_C@_02FPIMKNGF@?$CK?$DN@ 0000000180001830     libvcruntime:undname.obj
 0001:00000834       ??_C@_02FOEOMHFC@?$CL?$DN@ 0000000180001834     libvcruntime:undname.obj
 0001:00000838       ??_C@_02FKMDLLOA@?9?$DN@   0000000180001838     libvcruntime:undname.obj
 0001:0000083c       ??_C@_02FJEHGPIO@?1?$DN@   000000018000183c     libvcruntime:undname.obj
 0001:00000840       ??_C@_02FENAOKFI@?$CF?$DN@ 0000000180001840     libvcruntime:undname.obj
 0001:00000844       ??_C@_03IKFCCPFF@?$DO?$DO?$DN@ 0000000180001844     libvcruntime:undname.obj
 0001:00000848       ??_C@_03CDNPDDLA@?$DM?$DM?$DN@ 0000000180001848     libvcruntime:undname.obj
 0001:0000084c       ??_C@_02FGJGFEAB@?$CG?$DN@ 000000018000184c     libvcruntime:undname.obj
 0001:00000850       ??_C@_02DHLNPPGH@?$HM?$DN@ 0000000180001850     libvcruntime:undname.obj
 0001:00000854       ??_C@_02MHEGNOJ@?$FO?$DN@  0000000180001854     libvcruntime:undname.obj
 0001:00000858       ??_C@_09IFPLHPGF@?$GAvftable?8@ 0000000180001858     libvcruntime:undname.obj
 0001:00000868       ??_C@_09BLBHBJP@?$GAvbtable?8@ 0000000180001868     libvcruntime:undname.obj
 0001:00000878       ??_C@_07FEEIOKP@?$GAvcall?8@ 0000000180001878     libvcruntime:undname.obj
 0001:00000880       ??_C@_08LLFFHHDJ@?$GAtypeof?8@ 0000000180001880     libvcruntime:undname.obj
 0001:00000890       ??_C@_0BF@KDPPACIK@?$GAlocal?5static?5guard?8@ 0000000180001890     libvcruntime:undname.obj
 0001:000008a8       ??_C@_08OBABFOLI@?$GAstring?8@ 00000001800018a8     libvcruntime:undname.obj
 0001:000008b8       ??_C@_0BD@JDLKDPAB@?$GAvbase?5destructor?8@ 00000001800018b8     libvcruntime:undname.obj
 0001:000008d0       ??_C@_0BN@DEGPLNFK@?$GAvector?5deleting?5destructor?8@ 00000001800018d0     libvcruntime:undname.obj
 0001:000008f0       ??_C@_0BO@OBMKPJIG@?$GAdefault?5constructor?5closure?8@ 00000001800018f0     libvcruntime:undname.obj
 0001:00000910       ??_C@_0BN@IMDCHIKM@?$GAscalar?5deleting?5destructor?8@ 0000000180001910     libvcruntime:undname.obj
 0001:00000930       ??_C@_0BO@PFGOCPJJ@?$GAvector?5constructor?5iterator?8@ 0000000180001930     libvcruntime:undname.obj
 0001:00000950       ??_C@_0BN@LFPFMEDL@?$GAvector?5destructor?5iterator?8@ 0000000180001950     libvcruntime:undname.obj
 0001:00000970       ??_C@_0CE@IKBNEHA@?$GAvector?5vbase?5constructor?5itera@ 0000000180001970     libvcruntime:undname.obj
 0001:00000998       ??_C@_0BL@NILFHHPC@?$GAvirtual?5displacement?5map?8@ 0000000180001998     libvcruntime:undname.obj
 0001:000009b8       ??_C@_0CB@JONCMFFK@?$GAeh?5vector?5constructor?5iterator@ 00000001800019b8     libvcruntime:undname.obj
 0001:000009e0       ??_C@_0CA@GCEOPDGL@?$GAeh?5vector?5destructor?5iterator?8@ 00000001800019e0     libvcruntime:undname.obj
 0001:00000a00       ??_C@_0CH@OOJPLCPH@?$GAeh?5vector?5vbase?5constructor?5it@ 0000000180001a00     libvcruntime:undname.obj
 0001:00000a28       ??_C@_0BL@LLKPOHJI@?$GAcopy?5constructor?5closure?8@ 0000000180001a28     libvcruntime:undname.obj
 0001:00000a48       ??_C@_0BA@KBCDOMBN@?$GAudt?5returning?8@ 0000000180001a48     libvcruntime:undname.obj
 0001:00000a58       ??_C@_03KLGMFNMG@?$GAEH@   0000000180001a58     libvcruntime:undname.obj
 0001:00000a5c       ??_C@_05KHLCHHI@?$GARTTI@  0000000180001a5c     libvcruntime:undname.obj
 0001:00000a68       ??_C@_0BA@KKLDJDLB@?$GAlocal?5vftable?8@ 0000000180001a68     libvcruntime:undname.obj
 0001:00000a78       ??_C@_0CE@IIHCMGGL@?$GAlocal?5vftable?5constructor?5clos@ 0000000180001a78     libvcruntime:undname.obj
 0001:00000a9c       ??_C@_06FHBGPFGH@?5new?$FL?$FN@ 0000000180001a9c     libvcruntime:undname.obj
 0001:00000aa8       ??_C@_09LBNFPBCA@?5delete?$FL?$FN@ 0000000180001aa8     libvcruntime:undname.obj
 0001:00000ab8       ??_C@_0P@HJKNJFNN@?$GAomni?5callsig?8@ 0000000180001ab8     libvcruntime:undname.obj
 0001:00000ac8       ??_C@_0BL@CNOONJFP@?$GAplacement?5delete?5closure?8@ 0000000180001ac8     libvcruntime:undname.obj
 0001:00000ae8       ??_C@_0BN@CKNJLHMB@?$GAplacement?5delete?$FL?$FN?5closure?8@ 0000000180001ae8     libvcruntime:undname.obj
 0001:00000b08       ??_C@_0CG@CFDHKGGD@?$GAmanaged?5vector?5constructor?5ite@ 0000000180001b08     libvcruntime:undname.obj
 0001:00000b30       ??_C@_0CF@IMGKMJNO@?$GAmanaged?5vector?5destructor?5iter@ 0000000180001b30     libvcruntime:undname.obj
 0001:00000b58       ??_C@_0CG@HLDDJMAG@?$GAeh?5vector?5copy?5constructor?5ite@ 0000000180001b58     libvcruntime:undname.obj
 0001:00000b80       ??_C@_0CM@FCBBDIGB@?$GAeh?5vector?5vbase?5copy?5construct@ 0000000180001b80     libvcruntime:undname.obj
 0001:00000bb0       ??_C@_0BL@CLIPGLGB@?$GAdynamic?5initializer?5for?5?8@ 0000000180001bb0     libvcruntime:undname.obj
 0001:00000bd0       ??_C@_0CB@PDBIFEP@?$GAdynamic?5atexit?5destructor?5for?5@ 0000000180001bd0     libvcruntime:undname.obj
 0001:00000bf8       ??_C@_0CD@CGAJBKEJ@?$GAvector?5copy?5constructor?5iterat@ 0000000180001bf8     libvcruntime:undname.obj
 0001:00000c20       ??_C@_0CJ@GJELGAMM@?$GAvector?5vbase?5copy?5constructor?5@ 0000000180001c20     libvcruntime:undname.obj
 0001:00000c50       ??_C@_0CL@FGIJHLCE@?$GAmanaged?5vector?5copy?5constructo@ 0000000180001c50     libvcruntime:undname.obj
 0001:00000c80       ??_C@_0BM@PMGGMLDN@?$GAlocal?5static?5thread?5guard?8@ 0000000180001c80     libvcruntime:undname.obj
 0001:00000ca0       ??_C@_0N@BDNMDMOL@operator?5?$CC?$CC?5@ 0000000180001ca0     libvcruntime:undname.obj
 0001:00000cb0       ??_C@_0BC@GGEBGALA@operator?5co_await@ 0000000180001cb0     libvcruntime:undname.obj
 0001:00000cc8       ??_C@_0BC@DAFEJGAK@?5Type?5Descriptor?8@ 0000000180001cc8     libvcruntime:undname.obj
 0001:00000ce0       ??_C@_0BM@LDKODKLH@?5Base?5Class?5Descriptor?5at?5?$CI@ 0000000180001ce0     libvcruntime:undname.obj
 0001:00000d00       ??_C@_0BD@LGICGFMM@?5Base?5Class?5Array?8@ 0000000180001d00     libvcruntime:undname.obj
 0001:00000d18       ??_C@_0BN@MECKDCOJ@?5Class?5Hierarchy?5Descriptor?8@ 0000000180001d18     libvcruntime:undname.obj
 0001:00000d38       ??_C@_0BK@CFCOFLF@?5Complete?5Object?5Locator?8@ 0000000180001d38     libvcruntime:undname.obj
 0001:00000d70       ??_C@_1DM@KHCHBNEB@?$AAa?$AAp?$AAi?$AA?9?$AAm?$AAs?$AA?9?$AAw?$AAi?$AAn?$AA?9?$AAc?$AAo?$AAr?$AAe@ 0000000180001d70     libvcruntime:winapi_downlevel.obj
 0001:00000db0       ??_C@_1DK@LPPGFMPP@?$AAa?$AAp?$AAi?$AA?9?$AAm?$AAs?$AA?9?$AAw?$AAi?$AAn?$AA?9?$AAc?$AAo?$AAr?$AAe@ 0000000180001db0     libvcruntime:winapi_downlevel.obj
 0001:00000df0       ??_C@_1BC@GDMECMAK@?$AAk?$AAe?$AAr?$AAn?$AAe?$AAl?$AA3?$AA2@ 0000000180001df0     libvcruntime:winapi_downlevel.obj
 0001:00000e08       ??_C@_1BA@PFFKHIOG@?$AAa?$AAp?$AAi?$AA?9?$AAm?$AAs?$AA?9@ 0000000180001e08     libvcruntime:winapi_downlevel.obj
 0001:00000e18       ??_C@_1BA@IAIFMGEF@?$AAe?$AAx?$AAt?$AA?9?$AAm?$AAs?$AA?9@ 0000000180001e18     libvcruntime:winapi_downlevel.obj
 0001:00000e30       ??_C@_08KNHFBNJ@FlsAlloc@  0000000180001e30     libvcruntime:winapi_downlevel.obj
 0001:00000e48       ??_C@_07PEJMOBNF@FlsFree@  0000000180001e48     libvcruntime:winapi_downlevel.obj
 0001:00000e58       ??_C@_0M@GDNOONDI@FlsGetValue@ 0000000180001e58     libvcruntime:winapi_downlevel.obj
 0001:00000e70       ??_C@_0M@JCPCPOEF@FlsSetValue@ 0000000180001e70     libvcruntime:winapi_downlevel.obj
 0001:00000e88       ??_C@_0BM@HCFOFFN@InitializeCriticalSectionEx@ 0000000180001e88     libvcruntime:winapi_downlevel.obj
 0001:00000eb0       __acrt_exception_action_table 0000000180001eb0     libucrt:exception_filter.obj
 0001:00000f70       __acrt_signal_action_table_count 0000000180001f70     libucrt:exception_filter.obj
 0001:00000f78       __acrt_signal_action_first_fpe_index 0000000180001f78     libucrt:exception_filter.obj
 0001:00000f80       __acrt_signal_action_fpe_count 0000000180001f80     libucrt:exception_filter.obj
 0001:00000f88       ??_C@_1BI@BGOHAHKC@?$AAm?$AAs?$AAc?$AAo?$AAr?$AAe?$AAe?$AA?4?$AAd?$AAl?$AAl?$AA?$AA@ 0000000180001f88     libucrt:exit.obj
 0001:00000fa0       ??_C@_0P@MIGLKIOC@CorExitProcess?$AA@ 0000000180001fa0     libucrt:exit.obj
 0001:00001238       ??_C@_1M@HPNHIDJI@?$AAj?$AAa?$AA?9?$AAJ?$AAP?$AA?$AA@ 0000000180002238     libucrt:mbctype.obj
 0001:00001248       ??_C@_1M@BIBDDEMK@?$AAz?$AAh?$AA?9?$AAC?$AAN?$AA?$AA@ 0000000180002248     libucrt:mbctype.obj
 0001:00001258       ??_C@_1M@JLOOOEGK@?$AAk?$AAo?$AA?9?$AAK?$AAR?$AA?$AA@ 0000000180002258     libucrt:mbctype.obj
 0001:00001268       ??_C@_1M@CLNBBOPM@?$AAz?$AAh?$AA?9?$AAT?$AAW?$AA?$AA@ 0000000180002268     libucrt:mbctype.obj
 0001:00001320       ??_C@_1EA@JGEFHKEI@?$AAa?$AAp?$AAi?$AA?9?$AAm?$AAs?$AA?9?$AAw?$AAi?$AAn?$AA?9?$AAc?$AAo?$AAr?$AAe?$AA?9?$AAd?$AAa?$AAt?$AAe?$AAt?$AAi?$AAm?$AAe?$AA?9?$AAl?$AA1?$AA?9?$AA1?$AA?9?$AA1?$AA?$AA@ 0000000180002320     libucrt:winapi_thunks.obj
 0001:00001360       ??_C@_1DM@KHCHBNEB@?$AAa?$AAp?$AAi?$AA?9?$AAm?$AAs?$AA?9?$AAw?$AAi?$AAn?$AA?9?$AAc?$AAo?$AAr?$AAe?$AA?9?$AAf?$AAi?$AAb?$AAe?$AAr?$AAs?$AA?9?$AAl?$AA1?$AA?9?$AA1?$AA?9?$AA1?$AA?$AA@ 0000000180002360     libucrt:winapi_thunks.obj
 0001:000013a0       ??_C@_1DI@IJCEHOCB@?$AAa?$AAp?$AAi?$AA?9?$AAm?$AAs?$AA?9?$AAw?$AAi?$AAn?$AA?9?$AAc?$AAo?$AAr?$AAe?$AA?9?$AAf?$AAi?$AAl?$AAe?$AA?9?$AAl?$AA1?$AA?9?$AA2?$AA?9?$AA2?$AA?$AA@ 00000001800023a0     libucrt:winapi_thunks.obj
 0001:000013e0       ??_C@_1EI@MPIAOHOC@?$AAa?$AAp?$AAi?$AA?9?$AAm?$AAs?$AA?9?$AAw?$AAi?$AAn?$AA?9?$AAc?$AAo?$AAr?$AAe?$AA?9?$AAl?$AAo?$AAc?$AAa?$AAl?$AAi?$AAz?$AAa?$AAt?$AAi?$AAo?$AAn?$AA?9?$AAl?$AA1?$AA?9@ 00000001800023e0     libucrt:winapi_thunks.obj
 0001:00001430       ??_C@_1FK@FPHCKFIE@?$AAa?$AAp?$AAi?$AA?9?$AAm?$AAs?$AA?9?$AAw?$AAi?$AAn?$AA?9?$AAc?$AAo?$AAr?$AAe?$AA?9?$AAl?$AAo?$AAc?$AAa?$AAl?$AAi?$AAz?$AAa?$AAt?$AAi?$AAo?$AAn?$AA?9?$AAo?$AAb?$AAs@ 0000000180002430     libucrt:winapi_thunks.obj
 0001:00001490       ??_C@_1EM@DILCGIIO@?$AAa?$AAp?$AAi?$AA?9?$AAm?$AAs?$AA?9?$AAw?$AAi?$AAn?$AA?9?$AAc?$AAo?$AAr?$AAe?$AA?9?$AAp?$AAr?$AAo?$AAc?$AAe?$AAs?$AAs?$AAt?$AAh?$AAr?$AAe?$AAa?$AAd?$AAs?$AA?9?$AAl@ 0000000180002490     libucrt:winapi_thunks.obj
 0001:000014e0       ??_C@_1DM@LNCGDDPN@?$AAa?$AAp?$AAi?$AA?9?$AAm?$AAs?$AA?9?$AAw?$AAi?$AAn?$AA?9?$AAc?$AAo?$AAr?$AAe?$AA?9?$AAs?$AAt?$AAr?$AAi?$AAn?$AAg?$AA?9?$AAl?$AA1?$AA?9?$AA1?$AA?9?$AA0?$AA?$AA@ 00000001800024e0     libucrt:winapi_thunks.obj
 0001:00001520       ??_C@_1DK@LPPGFMPP@?$AAa?$AAp?$AAi?$AA?9?$AAm?$AAs?$AA?9?$AAw?$AAi?$AAn?$AA?9?$AAc?$AAo?$AAr?$AAe?$AA?9?$AAs?$AAy?$AAn?$AAc?$AAh?$AA?9?$AAl?$AA1?$AA?9?$AA2?$AA?9?$AA0?$AA?$AA@ 0000000180002520     libucrt:winapi_thunks.obj
 0001:00001560       ??_C@_1DO@FPAPJEMD@?$AAa?$AAp?$AAi?$AA?9?$AAm?$AAs?$AA?9?$AAw?$AAi?$AAn?$AA?9?$AAc?$AAo?$AAr?$AAe?$AA?9?$AAs?$AAy?$AAs?$AAi?$AAn?$AAf?$AAo?$AA?9?$AAl?$AA1?$AA?9?$AA2?$AA?9?$AA1?$AA?$AA@ 0000000180002560     libucrt:winapi_thunks.obj
 0001:000015a0       ??_C@_1DK@NDHNAHIO@?$AAa?$AAp?$AAi?$AA?9?$AAm?$AAs?$AA?9?$AAw?$AAi?$AAn?$AA?9?$AAc?$AAo?$AAr?$AAe?$AA?9?$AAw?$AAi?$AAn?$AAr?$AAt?$AA?9?$AAl?$AA1?$AA?9?$AA1?$AA?9?$AA0?$AA?$AA@ 00000001800025a0     libucrt:winapi_thunks.obj
 0001:000015e0       ??_C@_1DM@KGHDGBCM@?$AAa?$AAp?$AAi?$AA?9?$AAm?$AAs?$AA?9?$AAw?$AAi?$AAn?$AA?9?$AAc?$AAo?$AAr?$AAe?$AA?9?$AAx?$AAs?$AAt?$AAa?$AAt?$AAe?$AA?9?$AAl?$AA2?$AA?9?$AA1?$AA?9?$AA0?$AA?$AA@ 00000001800025e0     libucrt:winapi_thunks.obj
 0001:00001620       ??_C@_1EO@IJIOEFOH@?$AAa?$AAp?$AAi?$AA?9?$AAm?$AAs?$AA?9?$AAw?$AAi?$AAn?$AA?9?$AAr?$AAt?$AAc?$AAo?$AAr?$AAe?$AA?9?$AAn?$AAt?$AAu?$AAs?$AAe?$AAr?$AA?9?$AAw?$AAi?$AAn?$AAd?$AAo?$AAw?$AA?9@ 0000000180002620     libucrt:winapi_thunks.obj
 0001:00001670       ??_C@_1FG@HHGEKANL@?$AAa?$AAp?$AAi?$AA?9?$AAm?$AAs?$AA?9?$AAw?$AAi?$AAn?$AA?9?$AAs?$AAe?$AAc?$AAu?$AAr?$AAi?$AAt?$AAy?$AA?9?$AAs?$AAy?$AAs?$AAt?$AAe?$AAm?$AAf?$AAu?$AAn?$AAc?$AAt?$AAi@ 0000000180002670     libucrt:winapi_thunks.obj
 0001:000016d0       ??_C@_1EG@DBIOJECG@?$AAe?$AAx?$AAt?$AA?9?$AAm?$AAs?$AA?9?$AAw?$AAi?$AAn?$AA?9?$AAn?$AAt?$AAu?$AAs?$AAe?$AAr?$AA?9?$AAd?$AAi?$AAa?$AAl?$AAo?$AAg?$AAb?$AAo?$AAx?$AA?9?$AAl?$AA1?$AA?9?$AA1@ 00000001800026d0     libucrt:winapi_thunks.obj
 0001:00001720       ??_C@_1EO@FIHMJCLF@?$AAe?$AAx?$AAt?$AA?9?$AAm?$AAs?$AA?9?$AAw?$AAi?$AAn?$AA?9?$AAn?$AAt?$AAu?$AAs?$AAe?$AAr?$AA?9?$AAw?$AAi?$AAn?$AAd?$AAo?$AAw?$AAs?$AAt?$AAa?$AAt?$AAi?$AAo?$AAn?$AA?9@ 0000000180002720     libucrt:winapi_thunks.obj
 0001:00001770       ??_C@_1BC@DNHGCMLG@?$AAa?$AAd?$AAv?$AAa?$AAp?$AAi?$AA3?$AA2?$AA?$AA@ 0000000180002770     libucrt:winapi_thunks.obj
 0001:00001788       ??_C@_1BC@GDMECMAK@?$AAk?$AAe?$AAr?$AAn?$AAe?$AAl?$AA3?$AA2?$AA?$AA@ 0000000180002788     libucrt:winapi_thunks.obj
 0001:000017a0       ??_C@_1M@OAIMIKLP@?$AAn?$AAt?$AAd?$AAl?$AAl?$AA?$AA@ 00000001800027a0     libucrt:winapi_thunks.obj
 0001:000017b0       ??_C@_1EG@DPGNFKGC@?$AAa?$AAp?$AAi?$AA?9?$AAm?$AAs?$AA?9?$AAw?$AAi?$AAn?$AA?9?$AAa?$AAp?$AAp?$AAm?$AAo?$AAd?$AAe?$AAl?$AA?9?$AAr?$AAu?$AAn?$AAt?$AAi?$AAm?$AAe?$AA?9?$AAl?$AA1?$AA?9?$AA1@ 00000001800027b0     libucrt:winapi_thunks.obj
 0001:000017f8       ??_C@_1O@BCCLBEOE@?$AAu?$AAs?$AAe?$AAr?$AA3?$AA2?$AA?$AA@ 00000001800027f8     libucrt:winapi_thunks.obj
 0001:00001808       ??_C@_1BA@PFFKHIOG@?$AAa?$AAp?$AAi?$AA?9?$AAm?$AAs?$AA?9?$AA?$AA@ 0000000180002808     libucrt:winapi_thunks.obj
 0001:00001818       ??_C@_1BA@IAIFMGEF@?$AAe?$AAx?$AAt?$AA?9?$AAm?$AAs?$AA?9?$AA?$AA@ 0000000180002818     libucrt:winapi_thunks.obj
 0001:00001830       ??_C@_0BA@FHFNEAED@AreFileApisANSI?$AA@ 0000000180002830     libucrt:winapi_thunks.obj
 0001:00001848       ??_C@_08KNHFBNJ@FlsAlloc?$AA@ 0000000180002848     libucrt:winapi_thunks.obj
 0001:00001860       ??_C@_07PEJMOBNF@FlsFree?$AA@ 0000000180002860     libucrt:winapi_thunks.obj
 0001:00001870       ??_C@_0M@GDNOONDI@FlsGetValue?$AA@ 0000000180002870     libucrt:winapi_thunks.obj
 0001:00001888       ??_C@_0M@JCPCPOEF@FlsSetValue?$AA@ 0000000180002888     libucrt:winapi_thunks.obj
 0001:000018a0       ??_C@_0BM@HCFOFFN@InitializeCriticalSectionEx?$AA@ 00000001800028a0     libucrt:winapi_thunks.obj
 0001:000018c8       ??_C@_0O@KKBNKAPF@LCMapStringEx?$AA@ 00000001800028c8     libucrt:winapi_thunks.obj
 0001:000018e0       ??_C@_0BB@HBDEELFH@LocaleNameToLCID?$AA@ 00000001800028e0     libucrt:winapi_thunks.obj
 0001:000018f8       ??_C@_0CF@OJOFEIGO@AppPolicyGetProcessTerminationMe@ 00000001800028f8     libucrt:winapi_thunks.obj
 0001:00001920       __lc_time_c                0000000180002920     libucrt:nlsdata.obj
 0001:00001be0       ??_C@_03KOEHGMDN@Sun?$AA@  0000000180002be0     libucrt:nlsdata.obj
 0001:00001be4       ??_C@_03PDAGKDH@Mon?$AA@   0000000180002be4     libucrt:nlsdata.obj
 0001:00001be8       ??_C@_03NAGEINEP@Tue?$AA@  0000000180002be8     libucrt:nlsdata.obj
 0001:00001bec       ??_C@_03MHOMLAJA@Wed?$AA@  0000000180002bec     libucrt:nlsdata.obj
 0001:00001bf0       ??_C@_03IOFIKPDN@Thu?$AA@  0000000180002bf0     libucrt:nlsdata.obj
 0001:00001bf4       ??_C@_03IDIOELNC@Fri?$AA@  0000000180002bf4     libucrt:nlsdata.obj
 0001:00001bf8       ??_C@_03FEFJNEK@Sat?$AA@   0000000180002bf8     libucrt:nlsdata.obj
 0001:00001bfc       ??_C@_06OOPIFAJ@Sunday?$AA@ 0000000180002bfc     libucrt:nlsdata.obj
 0001:00001c04       ??_C@_06JLEDEDGH@Monday?$AA@ 0000000180002c04     libucrt:nlsdata.obj
 0001:00001c10       ??_C@_07BAAGCFCM@Tuesday?$AA@ 0000000180002c10     libucrt:nlsdata.obj
 0001:00001c18       ??_C@_09DLIGFAKA@Wednesday?$AA@ 0000000180002c18     libucrt:nlsdata.obj
 0001:00001c28       ??_C@_08HACCIKIA@Thursday?$AA@ 0000000180002c28     libucrt:nlsdata.obj
 0001:00001c34       ??_C@_06JECMNKMI@Friday?$AA@ 0000000180002c34     libucrt:nlsdata.obj
 0001:00001c40       ??_C@_08INBOOONO@Saturday?$AA@ 0000000180002c40     libucrt:nlsdata.obj
 0001:00001c4c       ??_C@_03JIHJHPIE@Jan?$AA@  0000000180002c4c     libucrt:nlsdata.obj
 0001:00001c50       ??_C@_03HJBDCHOM@Feb?$AA@  0000000180002c50     libucrt:nlsdata.obj
 0001:00001c54       ??_C@_03ODNJBKGA@Mar?$AA@  0000000180002c54     libucrt:nlsdata.obj
 0001:00001c58       ??_C@_03LEOLGMJP@Apr?$AA@  0000000180002c58     libucrt:nlsdata.obj
 0001:00001c5c       ??_C@_03CNMDKL@May?$AA@    0000000180002c5c     libucrt:nlsdata.obj
 0001:00001c60       ??_C@_03IDFGHECI@Jun?$AA@  0000000180002c60     libucrt:nlsdata.obj
 0001:00001c64       ??_C@_03LBGABGKK@Jul?$AA@  0000000180002c64     libucrt:nlsdata.obj
 0001:00001c68       ??_C@_03IFJFEIGA@Aug?$AA@  0000000180002c68     libucrt:nlsdata.obj
 0001:00001c6c       ??_C@_03GGCAPAJC@Sep?$AA@  0000000180002c6c     libucrt:nlsdata.obj
 0001:00001c70       ??_C@_03BMAOKBAD@Oct?$AA@  0000000180002c70     libucrt:nlsdata.obj
 0001:00001c74       ??_C@_03JPJOFNIA@Nov?$AA@  0000000180002c74     libucrt:nlsdata.obj
 0001:00001c78       ??_C@_03MKABNOCG@Dec?$AA@  0000000180002c78     libucrt:nlsdata.obj
 0001:00001c80       ??_C@_07CGJPFGJA@January?$AA@ 0000000180002c80     libucrt:nlsdata.obj
 0001:00001c88       ??_C@_08GNJGEPFN@February?$AA@ 0000000180002c88     libucrt:nlsdata.obj
 0001:00001c94       ??_C@_05HPCKOFNC@March?$AA@ 0000000180002c94     libucrt:nlsdata.obj
 0001:00001c9c       ??_C@_05DMJDNLEJ@April?$AA@ 0000000180002c9c     libucrt:nlsdata.obj
 0001:00001ca4       ??_C@_04CNLMGBGM@June?$AA@ 0000000180002ca4     libucrt:nlsdata.obj
 0001:00001cac       ??_C@_04MIEPOIFP@July?$AA@ 0000000180002cac     libucrt:nlsdata.obj
 0001:00001cb4       ??_C@_06LBBHFDDG@August?$AA@ 0000000180002cb4     libucrt:nlsdata.obj
 0001:00001cc0       ??_C@_09BHHEALKD@September?$AA@ 0000000180002cc0     libucrt:nlsdata.obj
 0001:00001cd0       ??_C@_07JJNFCEND@October?$AA@ 0000000180002cd0     libucrt:nlsdata.obj
 0001:00001cd8       ??_C@_08HCHEGEOA@November?$AA@ 0000000180002cd8     libucrt:nlsdata.obj
 0001:00001ce8       ??_C@_08EDHMEBNP@December?$AA@ 0000000180002ce8     libucrt:nlsdata.obj
 0001:00001cf4       ??_C@_02DEDBPAFC@AM?$AA@   0000000180002cf4     libucrt:nlsdata.obj
 0001:00001cf8       ??_C@_02CJNFDJBF@PM?$AA@   0000000180002cf8     libucrt:nlsdata.obj
 0001:00001d00       ??_C@_08BPBNCDIB@MM?1dd?1yy?$AA@ 0000000180002d00     libucrt:nlsdata.obj
 0001:00001d10       ??_C@_0BE@CKGJFCPC@dddd?0?5MMMM?5dd?0?5yyyy?$AA@ 0000000180002d10     libucrt:nlsdata.obj
 0001:00001d28       ??_C@_08JCCMCCIL@HH?3mm?3ss?$AA@ 0000000180002d28     libucrt:nlsdata.obj
 0001:00001d38       ??_C@_17MBGCMIPB@?$AAS?$AAu?$AAn?$AA?$AA@ 0000000180002d38     libucrt:nlsdata.obj
 0001:00001d40       ??_C@_17KBOMKBF@?$AAM?$AAo?$AAn?$AA?$AA@ 0000000180002d40     libucrt:nlsdata.obj
 0001:00001d48       ??_C@_17BMKGEGOJ@?$AAT?$AAu?$AAe?$AA?$AA@ 0000000180002d48     libucrt:nlsdata.obj
 0001:00001d50       ??_C@_17CJEDCEPE@?$AAW?$AAe?$AAd?$AA?$AA@ 0000000180002d50     libucrt:nlsdata.obj
 0001:00001d58       ??_C@_17PDPHAADD@?$AAT?$AAh?$AAu?$AA?$AA@ 0000000180002d58     libucrt:nlsdata.obj
 0001:00001d60       ??_C@_17HFOLPPLP@?$AAF?$AAr?$AAi?$AA?$AA@ 0000000180002d60     libucrt:nlsdata.obj
 0001:00001d68       ??_C@_17GGIBDPIH@?$AAS?$AAa?$AAt?$AA?$AA@ 0000000180002d68     libucrt:nlsdata.obj
 0001:00001d70       ??_C@_1O@IHNHDHPB@?$AAS?$AAu?$AAn?$AAd?$AAa?$AAy?$AA?$AA@ 0000000180002d70     libucrt:nlsdata.obj
 0001:00001d80       ??_C@_1O@MMNBFLIA@?$AAM?$AAo?$AAn?$AAd?$AAa?$AAy?$AA?$AA@ 0000000180002d80     libucrt:nlsdata.obj
 0001:00001d90       ??_C@_1BA@ENFBFFEK@?$AAT?$AAu?$AAe?$AAs?$AAd?$AAa?$AAy?$AA?$AA@ 0000000180002d90     libucrt:nlsdata.obj
 0001:00001da0       ??_C@_1BE@EBOGMDOH@?$AAW?$AAe?$AAd?$AAn?$AAe?$AAs?$AAd?$AAa?$AAy?$AA?$AA@ 0000000180002da0     libucrt:nlsdata.obj
 0001:00001db8       ??_C@_1BC@HHMNLIHE@?$AAT?$AAh?$AAu?$AAr?$AAs?$AAd?$AAa?$AAy?$AA?$AA@ 0000000180002db8     libucrt:nlsdata.obj
 0001:00001dd0       ??_C@_1O@PDICJHAG@?$AAF?$AAr?$AAi?$AAd?$AAa?$AAy?$AA?$AA@ 0000000180002dd0     libucrt:nlsdata.obj
 0001:00001de0       ??_C@_1BC@ENMNNPAJ@?$AAS?$AAa?$AAt?$AAu?$AAr?$AAd?$AAa?$AAy?$AA?$AA@ 0000000180002de0     libucrt:nlsdata.obj
 0001:00001df8       ??_C@_17DKNBKCHM@?$AAJ?$AAa?$AAn?$AA?$AA@ 0000000180002df8     libucrt:nlsdata.obj
 0001:00001e00       ??_C@_17LMDJEKJN@?$AAF?$AAe?$AAb?$AA?$AA@ 0000000180002e00     libucrt:nlsdata.obj
 0001:00001e08       ??_C@_17CKNLEDEC@?$AAM?$AAa?$AAr?$AA?$AA@ 0000000180002e08     libucrt:nlsdata.obj
 0001:00001e10       ??_C@_17LFPOIHDD@?$AAA?$AAp?$AAr?$AA?$AA@ 0000000180002e10     libucrt:nlsdata.obj
 0001:00001e18       ??_C@_17PNNKMEED@?$AAM?$AAa?$AAy?$AA?$AA@ 0000000180002e18     libucrt:nlsdata.obj
 0001:00001e20       ??_C@_17KCJGOCPB@?$AAJ?$AAu?$AAn?$AA?$AA@ 0000000180002e20     libucrt:nlsdata.obj
 0001:00001e28       ??_C@_17IJPCKHK@?$AAJ?$AAu?$AAl?$AA?$AA@ 0000000180002e28     libucrt:nlsdata.obj
 0001:00001e30       ??_C@_17ICPELBCN@?$AAA?$AAu?$AAg?$AA?$AA@ 0000000180002e30     libucrt:nlsdata.obj
 0001:00001e38       ??_C@_17HCHCOKMG@?$AAS?$AAe?$AAp?$AA?$AA@ 0000000180002e38     libucrt:nlsdata.obj
 0001:00001e40       ??_C@_17FNLKOI@?$AAO?$AAc?$AAt?$AA?$AA@ 0000000180002e40     libucrt:nlsdata.obj
 0001:00001e48       ??_C@_17BBDMLCIG@?$AAN?$AAo?$AAv?$AA?$AA@ 0000000180002e48     libucrt:nlsdata.obj
 0001:00001e50       ??_C@_17EGKACKIF@?$AAD?$AAe?$AAc?$AA?$AA@ 0000000180002e50     libucrt:nlsdata.obj
 0001:00001e58       ??_C@_1BA@EFMEIEBA@?$AAJ?$AAa?$AAn?$AAu?$AAa?$AAr?$AAy?$AA?$AA@ 0000000180002e58     libucrt:nlsdata.obj
 0001:00001e68       ??_C@_1BC@JGDDFFAM@?$AAF?$AAe?$AAb?$AAr?$AAu?$AAa?$AAr?$AAy?$AA?$AA@ 0000000180002e68     libucrt:nlsdata.obj
 0001:00001e80       ??_C@_1M@IKEENEDF@?$AAM?$AAa?$AAr?$AAc?$AAh?$AA?$AA@ 0000000180002e80     libucrt:nlsdata.obj
 0001:00001e90       ??_C@_1M@GJNLMHFD@?$AAA?$AAp?$AAr?$AAi?$AAl?$AA?$AA@ 0000000180002e90     libucrt:nlsdata.obj
 0001:00001ea0       ??_C@_19EPFLPGAP@?$AAJ?$AAu?$AAn?$AAe?$AA?$AA@ 0000000180002ea0     libucrt:nlsdata.obj
 0001:00001eb0       ??_C@_19BIFMLPCD@?$AAJ?$AAu?$AAl?$AAy?$AA?$AA@ 0000000180002eb0     libucrt:nlsdata.obj
 0001:00001ec0       ??_C@_1O@PAHLKOAC@?$AAA?$AAu?$AAg?$AAu?$AAs?$AAt?$AA?$AA@ 0000000180002ec0     libucrt:nlsdata.obj
 0001:00001ed0       ??_C@_1BE@DKAAMBJL@?$AAS?$AAe?$AAp?$AAt?$AAe?$AAm?$AAb?$AAe?$AAr?$AA?$AA@ 0000000180002ed0     libucrt:nlsdata.obj
 0001:00001ee8       ??_C@_1BA@EPANDLNG@?$AAO?$AAc?$AAt?$AAo?$AAb?$AAe?$AAr?$AA?$AA@ 0000000180002ee8     libucrt:nlsdata.obj
 0001:00001ef8       ??_C@_1BC@BGLIFPF@?$AAN?$AAo?$AAv?$AAe?$AAm?$AAb?$AAe?$AAr?$AA?$AA@ 0000000180002ef8     libucrt:nlsdata.obj
 0001:00001f10       ??_C@_1BC@FEMKIFH@?$AAD?$AAe?$AAc?$AAe?$AAm?$AAb?$AAe?$AAr?$AA?$AA@ 0000000180002f10     libucrt:nlsdata.obj
 0001:00001f24       ??_C@_15ODEHAHHF@?$AAA?$AAM?$AA?$AA@ 0000000180002f24     libucrt:nlsdata.obj
 0001:00001f2c       ??_C@_15CLMNNGEL@?$AAP?$AAM?$AA?$AA@ 0000000180002f2c     libucrt:nlsdata.obj
 0001:00001f38       ??_C@_1BC@IEBCMHCM@?$AAM?$AAM?$AA?1?$AAd?$AAd?$AA?1?$AAy?$AAy?$AA?$AA@ 0000000180002f38     libucrt:nlsdata.obj
 0001:00001f50       ??_C@_1CI@KNAKOEBC@?$AAd?$AAd?$AAd?$AAd?$AA?0?$AA?5?$AAM?$AAM?$AAM?$AAM?$AA?5?$AAd?$AAd?$AA?0?$AA?5?$AAy?$AAy?$AAy?$AAy?$AA?$AA@ 0000000180002f50     libucrt:nlsdata.obj
 0001:00001f78       ??_C@_1BC@GDGBMEMK@?$AAH?$AAH?$AA?3?$AAm?$AAm?$AA?3?$AAs?$AAs?$AA?$AA@ 0000000180002f78     libucrt:nlsdata.obj
 0001:00001f90       ??_C@_1M@BMHNFIME@?$AAe?$AAn?$AA?9?$AAU?$AAS?$AA?$AA@ 0000000180002f90     libucrt:nlsdata.obj
 0001:00001fa0       __newctype                 0000000180002fa0     libucrt:ctype.obj
 0001:000022a0       __newclmap                 00000001800032a0     libucrt:ctype.obj
 0001:00002420       __newcumap                 0000000180003420     libucrt:ctype.obj
 0001:000033e0       ??_C@_15EMKDOKLE@?$AAa?$AAr?$AA?$AA@ 00000001800043e0     libucrt:lcidtoname_downlevel.obj
 0001:000033e8       ??_C@_15KNPADPLH@?$AAb?$AAg?$AA?$AA@ 00000001800043e8     libucrt:lcidtoname_downlevel.obj
 0001:000033f0       ??_C@_15EDMHLDMO@?$AAc?$AAa?$AA?$AA@ 00000001800043f0     libucrt:lcidtoname_downlevel.obj
 0001:000033f8       ??_C@_1O@BPEAJADD@?$AAz?$AAh?$AA?9?$AAC?$AAH?$AAS?$AA?$AA@ 00000001800043f8     libucrt:lcidtoname_downlevel.obj
 0001:00003408       ??_C@_15LJNHCMNK@?$AAc?$AAs?$AA?$AA@ 0000000180004408     libucrt:lcidtoname_downlevel.obj
 0001:00003410       ??_C@_15FOMCIDHG@?$AAd?$AAa?$AA?$AA@ 0000000180004410     libucrt:lcidtoname_downlevel.obj
 0001:00003418       ??_C@_15NBKABECB@?$AAd?$AAe?$AA?$AA@ 0000000180004418     libucrt:lcidtoname_downlevel.obj
 0001:00003420       ??_C@_15GHPEIIAO@?$AAe?$AAl?$AA?$AA@ 0000000180004420     libucrt:lcidtoname_downlevel.obj
 0001:00003428       ??_C@_15MNPNEAIF@?$AAe?$AAn?$AA?$AA@ 0000000180004428     libucrt:lcidtoname_downlevel.obj
 0001:00003430       ??_C@_15GPIOMPMH@?$AAe?$AAs?$AA?$AA@ 0000000180004430     libucrt:lcidtoname_downlevel.obj
 0001:00003438       ??_C@_15NGLOAKJC@?$AAf?$AAi?$AA?$AA@ 0000000180004438     libucrt:lcidtoname_downlevel.obj
 0001:00003440       ??_C@_15FBKGNKAM@?$AAf?$AAr?$AA?$AA@ 0000000180004440     libucrt:lcidtoname_downlevel.obj
 0001:00003448       ??_C@_15KGGCNEFK@?$AAh?$AAe?$AA?$AA@ 0000000180004448     libucrt:lcidtoname_downlevel.obj
 0001:00003450       ??_C@_15PGHLIDMF@?$AAh?$AAu?$AA?$AA@ 0000000180004450     libucrt:lcidtoname_downlevel.obj
 0001:00003458       ??_C@_15BIEMAPLM@?$AAi?$AAs?$AA?$AA@ 0000000180004458     libucrt:lcidtoname_downlevel.obj
 0001:00003460       ??_C@_15IFJLDHAF@?$AAi?$AAt?$AA?$AA@ 0000000180004460     libucrt:lcidtoname_downlevel.obj
 0001:00003468       ??_C@_15GEMIOCAG@?$AAj?$AAa?$AA?$AA@ 0000000180004468     libucrt:lcidtoname_downlevel.obj
 0001:00003470       ??_C@_15EPELEGJA@?$AAk?$AAo?$AA?$AA@ 0000000180004470     libucrt:lcidtoname_downlevel.obj
 0001:00003478       ??_C@_15NDDHIMN@?$AAn?$AAl?$AA?$AA@ 0000000180004478     libucrt:lcidtoname_downlevel.obj
 0001:00003480       ??_C@_15BPIGNHCD@?$AAn?$AAo?$AA?$AA@ 0000000180004480     libucrt:lcidtoname_downlevel.obj
 0001:00003488       ??_C@_15DEOPBLCG@?$AAp?$AAl?$AA?$AA@ 0000000180004488     libucrt:lcidtoname_downlevel.obj
 0001:00003490       ??_C@_15KBECGEFG@?$AAp?$AAt?$AA?$AA@ 0000000180004490     libucrt:lcidtoname_downlevel.obj
 0001:00003498       ??_C@_15GLJCBFMD@?$AAr?$AAo?$AA?$AA@ 0000000180004498     libucrt:lcidtoname_downlevel.obj
 0001:000034a0       ??_C@_15FEDGKCDI@?$AAr?$AAu?$AA?$AA@ 00000001800044a0     libucrt:lcidtoname_downlevel.obj
 0001:000034a8       ??_C@_15GLKMLLHM@?$AAh?$AAr?$AA?$AA@ 00000001800044a8     libucrt:lcidtoname_downlevel.obj
 0001:000034b0       ??_C@_15CPKMFBDB@?$AAs?$AAk?$AA?$AA@ 00000001800044b0     libucrt:lcidtoname_downlevel.obj
 0001:000034b8       ??_C@_15BAAIOGMK@?$AAs?$AAq?$AA?$AA@ 00000001800044b8     libucrt:lcidtoname_downlevel.obj
 0001:000034c0       ??_C@_15INNPNOHD@?$AAs?$AAv?$AA?$AA@ 00000001800044c0     libucrt:lcidtoname_downlevel.obj
 0001:000034c8       ??_C@_15CABMMOGH@?$AAt?$AAh?$AA?$AA@ 00000001800044c8     libucrt:lcidtoname_downlevel.obj
 0001:000034d0       ??_C@_15BPLIHJJM@?$AAt?$AAr?$AA?$AA@ 00000001800044d0     libucrt:lcidtoname_downlevel.obj
 0001:000034d8       ??_C@_15NEOEKKDJ@?$AAu?$AAr?$AA?$AA@ 00000001800044d8     libucrt:lcidtoname_downlevel.obj
 0001:000034e0       ??_C@_15NFICGAJK@?$AAi?$AAd?$AA?$AA@ 00000001800044e0     libucrt:lcidtoname_downlevel.obj
 0001:000034e8       ??_C@_15PJPFLCCM@?$AAu?$AAk?$AA?$AA@ 00000001800044e8     libucrt:lcidtoname_downlevel.obj
 0001:000034f0       ??_C@_15HPJPHDM@?$AAb?$AAe?$AA?$AA@ 00000001800044f0     libucrt:lcidtoname_downlevel.obj
 0001:000034f8       ??_C@_15LCHLGJII@?$AAs?$AAl?$AA?$AA@ 00000001800044f8     libucrt:lcidtoname_downlevel.obj
 0001:00003500       ??_C@_15PCFJPHHO@?$AAe?$AAt?$AA?$AA@ 0000000180004500     libucrt:lcidtoname_downlevel.obj
 0001:00003508       ??_C@_15HPFPGODN@?$AAl?$AAv?$AA?$AA@ 0000000180004508     libucrt:lcidtoname_downlevel.obj
 0001:00003510       ??_C@_15NFFGKGLG@?$AAl?$AAt?$AA?$AA@ 0000000180004510     libucrt:lcidtoname_downlevel.obj
 0001:00003518       ??_C@_15BDAKCCHN@?$AAf?$AAa?$AA?$AA@ 0000000180004518     libucrt:lcidtoname_downlevel.obj
 0001:00003520       ??_C@_15NFGIAIAJ@?$AAv?$AAi?$AA?$AA@ 0000000180004520     libucrt:lcidtoname_downlevel.obj
 0001:00003528       ??_C@_15LMKNDMHN@?$AAh?$AAy?$AA?$AA@ 0000000180004528     libucrt:lcidtoname_downlevel.obj
 0001:00003530       ??_C@_15IJBHMCFL@?$AAa?$AAz?$AA?$AA@ 0000000180004530     libucrt:lcidtoname_downlevel.obj
 0001:00003538       ??_C@_15EKOFJABL@?$AAe?$AAu?$AA?$AA@ 0000000180004538     libucrt:lcidtoname_downlevel.obj
 0001:00003540       ??_C@_15BGHADCNK@?$AAm?$AAk?$AA?$AA@ 0000000180004540     libucrt:lcidtoname_downlevel.obj
 0001:00003548       ??_C@_15JDNICKHM@?$AAa?$AAf?$AA?$AA@ 0000000180004548     libucrt:lcidtoname_downlevel.obj
 0001:00003550       ??_C@_15KPJEDBKD@?$AAk?$AAa?$AA?$AA@ 0000000180004550     libucrt:lcidtoname_downlevel.obj
 0001:00003558       ??_C@_15PDNFFFEO@?$AAf?$AAo?$AA?$AA@ 0000000180004558     libucrt:lcidtoname_downlevel.obj
 0001:00003560       ??_C@_15OMLEGLOC@?$AAh?$AAi?$AA?$AA@ 0000000180004560     libucrt:lcidtoname_downlevel.obj
 0001:00003568       ??_C@_15IDNNENKK@?$AAm?$AAs?$AA?$AA@ 0000000180004568     libucrt:lcidtoname_downlevel.obj
 0001:00003570       ??_C@_15MACJNBMH@?$AAk?$AAk?$AA?$AA@ 0000000180004570     libucrt:lcidtoname_downlevel.obj
 0001:00003578       ??_C@_15DKDJEOND@?$AAk?$AAy?$AA?$AA@ 0000000180004578     libucrt:lcidtoname_downlevel.obj
 0001:00003580       ??_C@_15DFGDLJBG@?$AAs?$AAw?$AA?$AA@ 0000000180004580     libucrt:lcidtoname_downlevel.obj
 0001:00003588       ??_C@_15BBFAICNG@?$AAu?$AAz?$AA?$AA@ 0000000180004588     libucrt:lcidtoname_downlevel.obj
 0001:00003590       ??_C@_15DKNDCGEA@?$AAt?$AAt?$AA?$AA@ 0000000180004590     libucrt:lcidtoname_downlevel.obj
 0001:00003598       ??_C@_15MGIFMDPL@?$AAp?$AAa?$AA?$AA@ 0000000180004598     libucrt:lcidtoname_downlevel.obj
 0001:000035a0       ??_C@_15HCNDBBA@?$AAg?$AAu?$AA?$AA@ 00000001800045a0     libucrt:lcidtoname_downlevel.obj
 0001:000035a8       ??_C@_15FNBEIBON@?$AAt?$AAa?$AA?$AA@ 00000001800045a8     libucrt:lcidtoname_downlevel.obj
 0001:000035b0       ??_C@_15NCHGBGLK@?$AAt?$AAe?$AA?$AA@ 00000001800045b0     libucrt:lcidtoname_downlevel.obj
 0001:000035b8       ??_C@_15PHPHCBPF@?$AAk?$AAn?$AA?$AA@ 00000001800045b8     libucrt:lcidtoname_downlevel.obj
 0001:000035c0       ??_C@_15DLGBCKMP@?$AAm?$AAr?$AA?$AA@ 00000001800045c0     libucrt:lcidtoname_downlevel.obj
 0001:000035c8       ??_C@_15EABBLBFF@?$AAs?$AAa?$AA?$AA@ 00000001800045c8     libucrt:lcidtoname_downlevel.obj
 0001:000035d0       ??_C@_15CBKOMCOI@?$AAm?$AAn?$AA?$AA@ 00000001800045d0     libucrt:lcidtoname_downlevel.obj
 0001:000035d8       ??_C@_15CKDMCJAF@?$AAg?$AAl?$AA?$AA@ 00000001800045d8     libucrt:lcidtoname_downlevel.obj
 0001:000035e0       ??_C@_17CNJFBPG@?$AAk?$AAo?$AAk?$AA?$AA@ 00000001800045e0     libucrt:lcidtoname_downlevel.obj
 0001:000035e8       ??_C@_17FFBJICPL@?$AAs?$AAy?$AAr?$AA?$AA@ 00000001800045e8     libucrt:lcidtoname_downlevel.obj
 0001:000035f0       ??_C@_17KPNDCPAF@?$AAd?$AAi?$AAv?$AA?$AA@ 00000001800045f0     libucrt:lcidtoname_downlevel.obj
 0001:000035f8       ??_C@_11LOCGONAA@?$AA?$AA@ 00000001800045f8     libucrt:lcidtoname_downlevel.obj
 0001:00003600       ??_C@_1M@OKAHONE@?$AAa?$AAr?$AA?9?$AAS?$AAA?$AA?$AA@ 0000000180004600     libucrt:lcidtoname_downlevel.obj
 0001:00003610       ??_C@_1M@FFFIGIGK@?$AAb?$AAg?$AA?9?$AAB?$AAG?$AA?$AA@ 0000000180004610     libucrt:lcidtoname_downlevel.obj
 0001:00003620       ??_C@_1M@BJNKEDC@?$AAc?$AAa?$AA?9?$AAE?$AAS?$AA?$AA@ 0000000180004620     libucrt:lcidtoname_downlevel.obj
 0001:00003630       ??_C@_1M@IJJHFJHA@?$AAc?$AAs?$AA?9?$AAC?$AAZ?$AA?$AA@ 0000000180004630     libucrt:lcidtoname_downlevel.obj
 0001:00003640       ??_C@_1M@CLPEOBGI@?$AAd?$AAa?$AA?9?$AAD?$AAK?$AA?$AA@ 0000000180004640     libucrt:lcidtoname_downlevel.obj
 0001:00003650       ??_C@_1M@MCMADGCB@?$AAd?$AAe?$AA?9?$AAD?$AAE?$AA?$AA@ 0000000180004650     libucrt:lcidtoname_downlevel.obj
 0001:00003660       ??_C@_1M@OOCKEMAM@?$AAe?$AAl?$AA?9?$AAG?$AAR?$AA?$AA@ 0000000180004660     libucrt:lcidtoname_downlevel.obj
 0001:00003670       ??_C@_1M@DDNJFGID@?$AAf?$AAi?$AA?9?$AAF?$AAI?$AA?$AA@ 0000000180004670     libucrt:lcidtoname_downlevel.obj
 0001:00003680       ??_C@_1M@GLIPPMAC@?$AAf?$AAr?$AA?9?$AAF?$AAR?$AA?$AA@ 0000000180004680     libucrt:lcidtoname_downlevel.obj
 0001:00003690       ??_C@_1M@GFMCHPE@?$AAh?$AAe?$AA?9?$AAI?$AAL?$AA?$AA@ 0000000180004690     libucrt:lcidtoname_downlevel.obj
 0001:000036a0       ??_C@_1M@MHLPGNKM@?$AAh?$AAu?$AA?9?$AAH?$AAU?$AA?$AA@ 00000001800046a0     libucrt:lcidtoname_downlevel.obj
 0001:000036b0       ??_C@_1M@LPDDNNPN@?$AAi?$AAs?$AA?9?$AAI?$AAS?$AA?$AA@ 00000001800046b0     libucrt:lcidtoname_downlevel.obj
 0001:000036c0       ??_C@_1M@MADIPODN@?$AAi?$AAt?$AA?9?$AAI?$AAT?$AA?$AA@ 00000001800046c0     libucrt:lcidtoname_downlevel.obj
 0001:000036d0       ??_C@_1M@IHBJJGG@?$AAn?$AAl?$AA?9?$AAN?$AAL?$AA?$AA@ 00000001800046d0     libucrt:lcidtoname_downlevel.obj
 0001:000036e0       ??_C@_1M@EANAGDL@?$AAn?$AAb?$AA?9?$AAN?$AAO?$AA?$AA@ 00000001800046e0     libucrt:lcidtoname_downlevel.obj
 0001:000036f0       ??_C@_1M@NEIEMEGP@?$AAp?$AAl?$AA?9?$AAP?$AAL?$AA?$AA@ 00000001800046f0     libucrt:lcidtoname_downlevel.obj
 0001:00003700       ??_C@_1M@BOCFIGEP@?$AAp?$AAt?$AA?9?$AAB?$AAR?$AA?$AA@ 0000000180004700     libucrt:lcidtoname_downlevel.obj
 0001:00003710       ??_C@_1M@IMPFOPBG@?$AAr?$AAo?$AA?9?$AAR?$AAO?$AA?$AA@ 0000000180004710     libucrt:lcidtoname_downlevel.obj
 0001:00003720       ??_C@_1M@IDNNEJMM@?$AAr?$AAu?$AA?9?$AAR?$AAU?$AA?$AA@ 0000000180004720     libucrt:lcidtoname_downlevel.obj
 0001:00003730       ??_C@_1M@LILEEOGM@?$AAh?$AAr?$AA?9?$AAH?$AAR?$AA?$AA@ 0000000180004730     libucrt:lcidtoname_downlevel.obj
 0001:00003740       ??_C@_1M@FKIFEHPB@?$AAs?$AAk?$AA?9?$AAS?$AAK?$AA?$AA@ 0000000180004740     libucrt:lcidtoname_downlevel.obj
 0001:00003750       ??_C@_1M@LJMAMNPJ@?$AAs?$AAq?$AA?9?$AAA?$AAL?$AA?$AA@ 0000000180004750     libucrt:lcidtoname_downlevel.obj
 0001:00003760       ??_C@_1M@GIAKDKJK@?$AAs?$AAv?$AA?9?$AAS?$AAE?$AA?$AA@ 0000000180004760     libucrt:lcidtoname_downlevel.obj
 0001:00003770       ??_C@_1M@MKJKIKCL@?$AAt?$AAh?$AA?9?$AAT?$AAH?$AA?$AA@ 0000000180004770     libucrt:lcidtoname_downlevel.obj
 0001:00003780       ??_C@_1M@MFLCCMPB@?$AAt?$AAr?$AA?9?$AAT?$AAR?$AA?$AA@ 0000000180004780     libucrt:lcidtoname_downlevel.obj
 0001:00003790       ??_C@_1M@OIJHDKJN@?$AAu?$AAr?$AA?9?$AAP?$AAK?$AA?$AA@ 0000000180004790     libucrt:lcidtoname_downlevel.obj
 0001:000037a0       ??_C@_1M@LHIPCIEK@?$AAi?$AAd?$AA?9?$AAI?$AAD?$AA?$AA@ 00000001800047a0     libucrt:lcidtoname_downlevel.obj
 0001:000037b0       ??_C@_1M@MFMOBGI@?$AAu?$AAk?$AA?9?$AAU?$AAA?$AA?$AA@ 00000001800047b0     libucrt:lcidtoname_downlevel.obj
 0001:000037c0       ??_C@_1M@OBGLJIPL@?$AAb?$AAe?$AA?9?$AAB?$AAY?$AA?$AA@ 00000001800047c0     libucrt:lcidtoname_downlevel.obj
 0001:000037d0       ??_C@_1M@BCFAJEAD@?$AAs?$AAl?$AA?9?$AAS?$AAI?$AA?$AA@ 00000001800047d0     libucrt:lcidtoname_downlevel.obj
 0001:000037e0       ??_C@_1M@FKFFEDDN@?$AAe?$AAt?$AA?9?$AAE?$AAE?$AA?$AA@ 00000001800047e0     libucrt:lcidtoname_downlevel.obj
 0001:000037f0       ??_C@_1M@KGKKAACI@?$AAl?$AAv?$AA?9?$AAL?$AAV?$AA?$AA@ 00000001800047f0     libucrt:lcidtoname_downlevel.obj
 0001:00003800       ??_C@_1M@IFGBIJO@?$AAl?$AAt?$AA?9?$AAL?$AAT?$AA?$AA@ 0000000180004800     libucrt:lcidtoname_downlevel.obj
 0001:00003810       ??_C@_1M@FGEAHEDM@?$AAf?$AAa?$AA?9?$AAI?$AAR?$AA?$AA@ 0000000180004810     libucrt:lcidtoname_downlevel.obj
 0001:00003820       ??_C@_1M@KBMAIBFN@?$AAv?$AAi?$AA?9?$AAV?$AAN?$AA?$AA@ 0000000180004820     libucrt:lcidtoname_downlevel.obj
 0001:00003830       ??_C@_1M@GPCBKDJK@?$AAh?$AAy?$AA?9?$AAA?$AAM?$AA?$AA@ 0000000180004830     libucrt:lcidtoname_downlevel.obj
 0001:00003840       ??_C@_1BG@BECMDDJB@?$AAa?$AAz?$AA?9?$AAA?$AAZ?$AA?9?$AAL?$AAa?$AAt?$AAn?$AA?$AA@ 0000000180004840     libucrt:lcidtoname_downlevel.obj
 0001:00003858       ??_C@_1M@MAOFCAEA@?$AAe?$AAu?$AA?9?$AAE?$AAS?$AA?$AA@ 0000000180004858     libucrt:lcidtoname_downlevel.obj
 0001:00003868       ??_C@_1M@IGHABKPI@?$AAm?$AAk?$AA?9?$AAM?$AAK?$AA?$AA@ 0000000180004868     libucrt:lcidtoname_downlevel.obj
 0001:00003878       ??_C@_1M@IAIGNEJG@?$AAt?$AAn?$AA?9?$AAZ?$AAA?$AA?$AA@ 0000000180004878     libucrt:lcidtoname_downlevel.obj
 0001:00003888       ??_C@_1M@IIJCOJFA@?$AAx?$AAh?$AA?9?$AAZ?$AAA?$AA?$AA@ 0000000180004888     libucrt:lcidtoname_downlevel.obj
 0001:00003898       ??_C@_1M@LGPJHNJH@?$AAz?$AAu?$AA?9?$AAZ?$AAA?$AA?$AA@ 0000000180004898     libucrt:lcidtoname_downlevel.obj
 0001:000038a8       ??_C@_1M@HOKAOIO@?$AAa?$AAf?$AA?9?$AAZ?$AAA?$AA?$AA@ 00000001800048a8     libucrt:lcidtoname_downlevel.obj
 0001:000038b8       ??_C@_1M@DPCLHLIE@?$AAk?$AAa?$AA?9?$AAG?$AAE?$AA?$AA@ 00000001800048b8     libucrt:lcidtoname_downlevel.obj
 0001:000038c8       ??_C@_1M@BLKMHJBI@?$AAf?$AAo?$AA?9?$AAF?$AAO?$AA?$AA@ 00000001800048c8     libucrt:lcidtoname_downlevel.obj
 0001:000038d8       ??_C@_1M@LGGJAPPB@?$AAh?$AAi?$AA?9?$AAI?$AAN?$AA?$AA@ 00000001800048d8     libucrt:lcidtoname_downlevel.obj
 0001:000038e8       ??_C@_1M@FIKPIHFE@?$AAm?$AAt?$AA?9?$AAM?$AAT?$AA?$AA@ 00000001800048e8     libucrt:lcidtoname_downlevel.obj
 0001:000038f8       ??_C@_1M@HEGGPBFA@?$AAs?$AAe?$AA?9?$AAN?$AAO?$AA?$AA@ 00000001800048f8     libucrt:lcidtoname_downlevel.obj
 0001:00003908       ??_C@_1M@EIBJEEPA@?$AAm?$AAs?$AA?9?$AAM?$AAY?$AA?$AA@ 0000000180004908     libucrt:lcidtoname_downlevel.obj
 0001:00003918       ??_C@_1M@FHLBGMPP@?$AAk?$AAk?$AA?9?$AAK?$AAZ?$AA?$AA@ 0000000180004918     libucrt:lcidtoname_downlevel.obj
 0001:00003928       ??_C@_1M@NGJJLCGI@?$AAk?$AAy?$AA?9?$AAK?$AAG?$AA?$AA@ 0000000180004928     libucrt:lcidtoname_downlevel.obj
 0001:00003938       ??_C@_1M@GIENNBFC@?$AAs?$AAw?$AA?9?$AAK?$AAE?$AA?$AA@ 0000000180004938     libucrt:lcidtoname_downlevel.obj
 0001:00003948       ??_C@_1BG@NDGMJIMJ@?$AAu?$AAz?$AA?9?$AAU?$AAZ?$AA?9?$AAL?$AAa?$AAt?$AAn?$AA?$AA@ 0000000180004948     libucrt:lcidtoname_downlevel.obj
 0001:00003960       ??_C@_1M@IDCCIHBC@?$AAt?$AAt?$AA?9?$AAR?$AAU?$AA?$AA@ 0000000180004960     libucrt:lcidtoname_downlevel.obj
 0001:00003970       ??_C@_1M@LOICPMOJ@?$AAb?$AAn?$AA?9?$AAI?$AAN?$AA?$AA@ 0000000180004970     libucrt:lcidtoname_downlevel.obj
 0001:00003980       ??_C@_1M@KPKKNEAH@?$AAp?$AAa?$AA?9?$AAI?$AAN?$AA?$AA@ 0000000180004980     libucrt:lcidtoname_downlevel.obj
 0001:00003990       ??_C@_1M@PJGPPBOG@?$AAg?$AAu?$AA?9?$AAI?$AAN?$AA?$AA@ 0000000180004990     libucrt:lcidtoname_downlevel.obj
 0001:000039a0       ??_C@_1M@KMKMOPHI@?$AAt?$AAa?$AA?9?$AAI?$AAN?$AA?$AA@ 00000001800049a0     libucrt:lcidtoname_downlevel.obj
 0001:000039b0       ??_C@_1M@KFEHEPAC@?$AAt?$AAe?$AA?9?$AAI?$AAN?$AA?$AA@ 00000001800049b0     libucrt:lcidtoname_downlevel.obj
 0001:000039c0       ??_C@_1M@CDCLMGHI@?$AAk?$AAn?$AA?9?$AAI?$AAN?$AA?$AA@ 00000001800049c0     libucrt:lcidtoname_downlevel.obj
 0001:000039d0       ??_C@_1M@MIODLDKF@?$AAm?$AAl?$AA?9?$AAI?$AAN?$AA?$AA@ 00000001800049d0     libucrt:lcidtoname_downlevel.obj
 0001:000039e0       ??_C@_1M@PBIEACPO@?$AAm?$AAr?$AA?9?$AAI?$AAN?$AA?$AA@ 00000001800049e0     libucrt:lcidtoname_downlevel.obj
 0001:000039f0       ??_C@_1M@NIDEAGPH@?$AAs?$AAa?$AA?9?$AAI?$AAN?$AA?$AA@ 00000001800049f0     libucrt:lcidtoname_downlevel.obj
 0001:00003a00       ??_C@_1M@FHIHCBIO@?$AAm?$AAn?$AA?9?$AAM?$AAN?$AA?$AA@ 0000000180004a00     libucrt:lcidtoname_downlevel.obj
 0001:00003a10       ??_C@_1M@JAIJPENP@?$AAc?$AAy?$AA?9?$AAG?$AAB?$AA?$AA@ 0000000180004a10     libucrt:lcidtoname_downlevel.obj
 0001:00003a20       ??_C@_1M@PHGFBEPN@?$AAg?$AAl?$AA?9?$AAE?$AAS?$AA?$AA@ 0000000180004a20     libucrt:lcidtoname_downlevel.obj
 0001:00003a30       ??_C@_1O@KPIPDNCP@?$AAk?$AAo?$AAk?$AA?9?$AAI?$AAN?$AA?$AA@ 0000000180004a30     libucrt:lcidtoname_downlevel.obj
 0001:00003a40       ??_C@_1O@KNHJLDJA@?$AAs?$AAy?$AAr?$AA?9?$AAS?$AAY?$AA?$AA@ 0000000180004a40     libucrt:lcidtoname_downlevel.obj
 0001:00003a50       ??_C@_1O@MKEKBLAH@?$AAd?$AAi?$AAv?$AA?9?$AAM?$AAV?$AA?$AA@ 0000000180004a50     libucrt:lcidtoname_downlevel.obj
 0001:00003a60       ??_C@_1O@OHDCKDDF@?$AAq?$AAu?$AAz?$AA?9?$AAB?$AAO?$AA?$AA@ 0000000180004a60     libucrt:lcidtoname_downlevel.obj
 0001:00003a70       ??_C@_1M@LEPJNLFD@?$AAn?$AAs?$AA?9?$AAZ?$AAA?$AA?$AA@ 0000000180004a70     libucrt:lcidtoname_downlevel.obj
 0001:00003a80       ??_C@_1M@OMLEIIJB@?$AAm?$AAi?$AA?9?$AAN?$AAZ?$AA?$AA@ 0000000180004a80     libucrt:lcidtoname_downlevel.obj
 0001:00003a90       ??_C@_1M@PMPEAILG@?$AAa?$AAr?$AA?9?$AAI?$AAQ?$AA?$AA@ 0000000180004a90     libucrt:lcidtoname_downlevel.obj
 0001:00003aa0       ??_C@_1M@CNKPNOEE@?$AAd?$AAe?$AA?9?$AAC?$AAH?$AA?$AA@ 0000000180004aa0     libucrt:lcidtoname_downlevel.obj
 0001:00003ab0       ??_C@_1M@LKMGMLKO@?$AAe?$AAn?$AA?9?$AAG?$AAB?$AA?$AA@ 0000000180004ab0     libucrt:lcidtoname_downlevel.obj
 0001:00003ac0       ??_C@_1M@PGKJFFGL@?$AAe?$AAs?$AA?9?$AAM?$AAX?$AA?$AA@ 0000000180004ac0     libucrt:lcidtoname_downlevel.obj
 0001:00003ad0       ??_C@_1M@DNNANBDC@?$AAf?$AAr?$AA?9?$AAB?$AAE?$AA?$AA@ 0000000180004ad0     libucrt:lcidtoname_downlevel.obj
 0001:00003ae0       ??_C@_1M@HLGMDFHM@?$AAi?$AAt?$AA?9?$AAC?$AAH?$AA?$AA@ 0000000180004ae0     libucrt:lcidtoname_downlevel.obj
 0001:00003af0       ??_C@_1M@CLLBGJH@?$AAn?$AAl?$AA?9?$AAB?$AAE?$AA?$AA@ 0000000180004af0     libucrt:lcidtoname_downlevel.obj
 0001:00003b00       ??_C@_1M@BODBOGLF@?$AAn?$AAn?$AA?9?$AAN?$AAO?$AA?$AA@ 0000000180004b00     libucrt:lcidtoname_downlevel.obj
 0001:00003b10       ??_C@_1M@HFFAHKAD@?$AAp?$AAt?$AA?9?$AAP?$AAT?$AA?$AA@ 0000000180004b10     libucrt:lcidtoname_downlevel.obj
 0001:00003b20       ??_C@_1BG@LNOAKHIE@?$AAs?$AAr?$AA?9?$AAS?$AAP?$AA?9?$AAL?$AAa?$AAt?$AAn?$AA?$AA@ 0000000180004b20     libucrt:lcidtoname_downlevel.obj
 0001:00003b38       ??_C@_1M@HBMHBGAK@?$AAs?$AAv?$AA?9?$AAF?$AAI?$AA?$AA@ 0000000180004b38     libucrt:lcidtoname_downlevel.obj
 0001:00003b48       ??_C@_1BG@DGCJGJBE@?$AAa?$AAz?$AA?9?$AAA?$AAZ?$AA?9?$AAC?$AAy?$AAr?$AAl?$AA?$AA@ 0000000180004b48     libucrt:lcidtoname_downlevel.obj
 0001:00003b60       ??_C@_1M@KEJDAAHB@?$AAs?$AAe?$AA?9?$AAS?$AAE?$AA?$AA@ 0000000180004b60     libucrt:lcidtoname_downlevel.obj
 0001:00003b70       ??_C@_1M@HEIBJJAD@?$AAm?$AAs?$AA?9?$AAB?$AAN?$AA?$AA@ 0000000180004b70     libucrt:lcidtoname_downlevel.obj
 0001:00003b80       ??_C@_1BG@PBGJMCEM@?$AAu?$AAz?$AA?9?$AAU?$AAZ?$AA?9?$AAC?$AAy?$AAr?$AAl?$AA?$AA@ 0000000180004b80     libucrt:lcidtoname_downlevel.obj
 0001:00003b98       ??_C@_1O@LAOBCMDF@?$AAq?$AAu?$AAz?$AA?9?$AAE?$AAC?$AA?$AA@ 0000000180004b98     libucrt:lcidtoname_downlevel.obj
 0001:00003ba8       ??_C@_1M@POEEMAIO@?$AAa?$AAr?$AA?9?$AAE?$AAG?$AA?$AA@ 0000000180004ba8     libucrt:lcidtoname_downlevel.obj
 0001:00003bb8       ??_C@_1M@EFAKDEDL@?$AAz?$AAh?$AA?9?$AAH?$AAK?$AA?$AA@ 0000000180004bb8     libucrt:lcidtoname_downlevel.obj
 0001:00003bc8       ??_C@_1M@HKKIJHGI@?$AAd?$AAe?$AA?9?$AAA?$AAT?$AA?$AA@ 0000000180004bc8     libucrt:lcidtoname_downlevel.obj
 0001:00003bd8       ??_C@_1M@KBFBEHJF@?$AAe?$AAn?$AA?9?$AAA?$AAU?$AA?$AA@ 0000000180004bd8     libucrt:lcidtoname_downlevel.obj
 0001:00003be8       ??_C@_1M@MNPLFAAH@?$AAe?$AAs?$AA?9?$AAE?$AAS?$AA?$AA@ 0000000180004be8     libucrt:lcidtoname_downlevel.obj
 0001:00003bf8       ??_C@_1M@HJOOJFMA@?$AAf?$AAr?$AA?9?$AAC?$AAA?$AA?$AA@ 0000000180004bf8     libucrt:lcidtoname_downlevel.obj
 0001:00003c08       ??_C@_1BG@JPOFPNAB@?$AAs?$AAr?$AA?9?$AAS?$AAP?$AA?9?$AAC?$AAy?$AAr?$AAl?$AA?$AA@ 0000000180004c08     libucrt:lcidtoname_downlevel.obj
 0001:00003c20       ??_C@_1M@LNFOCMOB@?$AAs?$AAe?$AA?9?$AAF?$AAI?$AA?$AA@ 0000000180004c20     libucrt:lcidtoname_downlevel.obj
 0001:00003c30       ??_C@_1O@MGJBOAMB@?$AAq?$AAu?$AAz?$AA?9?$AAP?$AAE?$AA?$AA@ 0000000180004c30     libucrt:lcidtoname_downlevel.obj
 0001:00003c40       ??_C@_1M@GJINLBOK@?$AAa?$AAr?$AA?9?$AAL?$AAY?$AA?$AA@ 0000000180004c40     libucrt:lcidtoname_downlevel.obj
 0001:00003c50       ??_C@_1M@GGMNHJNL@?$AAz?$AAh?$AA?9?$AAS?$AAG?$AA?$AA@ 0000000180004c50     libucrt:lcidtoname_downlevel.obj
 0001:00003c60       ??_C@_1M@HOIKODND@?$AAd?$AAe?$AA?9?$AAL?$AAU?$AA?$AA@ 0000000180004c60     libucrt:lcidtoname_downlevel.obj
 0001:00003c70       ??_C@_1M@DDOCCGFG@?$AAe?$AAn?$AA?9?$AAC?$AAA?$AA?$AA@ 0000000180004c70     libucrt:lcidtoname_downlevel.obj
 0001:00003c80       ??_C@_1M@BNOEMJLF@?$AAe?$AAs?$AA?9?$AAG?$AAT?$AA?$AA@ 0000000180004c80     libucrt:lcidtoname_downlevel.obj
 0001:00003c90       ??_C@_1M@EOGNKEK@?$AAf?$AAr?$AA?9?$AAC?$AAH?$AA?$AA@ 0000000180004c90     libucrt:lcidtoname_downlevel.obj
 0001:00003ca0       ??_C@_1M@FLIDJFHL@?$AAh?$AAr?$AA?9?$AAB?$AAA?$AA?$AA@ 0000000180004ca0     libucrt:lcidtoname_downlevel.obj
 0001:00003cb0       ??_C@_1O@FMCELNAJ@?$AAs?$AAm?$AAj?$AA?9?$AAN?$AAO?$AA?$AA@ 0000000180004cb0     libucrt:lcidtoname_downlevel.obj
 0001:00003cc0       ??_C@_1M@JHGLJMGJ@?$AAa?$AAr?$AA?9?$AAD?$AAZ?$AA?$AA@ 0000000180004cc0     libucrt:lcidtoname_downlevel.obj
 0001:00003cd0       ??_C@_1M@JKKFDCNP@?$AAz?$AAh?$AA?9?$AAM?$AAO?$AA?$AA@ 0000000180004cd0     libucrt:lcidtoname_downlevel.obj
 0001:00003ce0       ??_C@_1M@GEEFALPE@?$AAd?$AAe?$AA?9?$AAL?$AAI?$AA?$AA@ 0000000180004ce0     libucrt:lcidtoname_downlevel.obj
 0001:00003cf0       ??_C@_1M@IGEOFBG@?$AAe?$AAn?$AA?9?$AAN?$AAZ?$AA?$AA@ 0000000180004cf0     libucrt:lcidtoname_downlevel.obj
 0001:00003d00       ??_C@_1M@KDBONEHP@?$AAe?$AAs?$AA?9?$AAC?$AAR?$AA?$AA@ 0000000180004d00     libucrt:lcidtoname_downlevel.obj
 0001:00003d10       ??_C@_1M@FHMDOHNN@?$AAf?$AAr?$AA?9?$AAL?$AAU?$AA?$AA@ 0000000180004d10     libucrt:lcidtoname_downlevel.obj
 0001:00003d20       ??_C@_1BG@NFKKMAFG@?$AAb?$AAs?$AA?9?$AAB?$AAA?$AA?9?$AAL?$AAa?$AAt?$AAn?$AA?$AA@ 0000000180004d20     libucrt:lcidtoname_downlevel.obj
 0001:00003d38       ??_C@_1O@IMNBEMCI@?$AAs?$AAm?$AAj?$AA?9?$AAS?$AAE?$AA?$AA@ 0000000180004d38     libucrt:lcidtoname_downlevel.obj
 0001:00003d48       ??_C@_1M@DHHMBNDP@?$AAa?$AAr?$AA?9?$AAM?$AAA?$AA?$AA@ 0000000180004d48     libucrt:lcidtoname_downlevel.obj
 0001:00003d58       ??_C@_1M@BNBLJCGH@?$AAe?$AAn?$AA?9?$AAI?$AAE?$AA?$AA@ 0000000180004d58     libucrt:lcidtoname_downlevel.obj
 0001:00003d68       ??_C@_1M@GEPAFMDL@?$AAe?$AAs?$AA?9?$AAP?$AAA?$AA?$AA@ 0000000180004d68     libucrt:lcidtoname_downlevel.obj
 0001:00003d78       ??_C@_1M@OJONDMDL@?$AAf?$AAr?$AA?9?$AAM?$AAC?$AA?$AA@ 0000000180004d78     libucrt:lcidtoname_downlevel.obj
 0001:00003d88       ??_C@_1BG@OBCNFJB@?$AAs?$AAr?$AA?9?$AAB?$AAA?$AA?9?$AAL?$AAa?$AAt?$AAn?$AA?$AA@ 0000000180004d88     libucrt:lcidtoname_downlevel.obj
 0001:00003da0       ??_C@_1O@KEMEEGPO@?$AAs?$AAm?$AAa?$AA?9?$AAN?$AAO?$AA?$AA@ 0000000180004da0     libucrt:lcidtoname_downlevel.obj
 0001:00003db0       ??_C@_1M@ELMGFODK@?$AAa?$AAr?$AA?9?$AAT?$AAN?$AA?$AA@ 0000000180004db0     libucrt:lcidtoname_downlevel.obj
 0001:00003dc0       ??_C@_1M@BHDLHFAF@?$AAe?$AAn?$AA?9?$AAZ?$AAA?$AA?$AA@ 0000000180004dc0     libucrt:lcidtoname_downlevel.obj
 0001:00003dd0       ??_C@_1M@BMGIGLIF@?$AAe?$AAs?$AA?9?$AAD?$AAO?$AA?$AA@ 0000000180004dd0     libucrt:lcidtoname_downlevel.obj
 0001:00003de0       ??_C@_1BG@CMBHIPBE@?$AAs?$AAr?$AA?9?$AAB?$AAA?$AA?9?$AAC?$AAy?$AAr?$AAl?$AA?$AA@ 0000000180004de0     libucrt:lcidtoname_downlevel.obj
 0001:00003df8       ??_C@_1O@HEDBLHNP@?$AAs?$AAm?$AAa?$AA?9?$AAS?$AAE?$AA?$AA@ 0000000180004df8     libucrt:lcidtoname_downlevel.obj
 0001:00003e08       ??_C@_1M@DAGCADIM@?$AAa?$AAr?$AA?9?$AAO?$AAM?$AA?$AA@ 0000000180004e08     libucrt:lcidtoname_downlevel.obj
 0001:00003e18       ??_C@_1M@FODLMICG@?$AAe?$AAn?$AA?9?$AAJ?$AAM?$AA?$AA@ 0000000180004e18     libucrt:lcidtoname_downlevel.obj
 0001:00003e28       ??_C@_1M@DNMLCIHB@?$AAe?$AAs?$AA?9?$AAV?$AAE?$AA?$AA@ 0000000180004e28     libucrt:lcidtoname_downlevel.obj
 0001:00003e38       ??_C@_1O@EOKHMKJK@?$AAs?$AAm?$AAs?$AA?9?$AAF?$AAI?$AA?$AA@ 0000000180004e38     libucrt:lcidtoname_downlevel.obj
 0001:00003e48       ??_C@_1M@CAFJMKOF@?$AAa?$AAr?$AA?9?$AAY?$AAE?$AA?$AA@ 0000000180004e48     libucrt:lcidtoname_downlevel.obj
 0001:00003e58       ??_C@_1M@CBFHIJLI@?$AAe?$AAn?$AA?9?$AAC?$AAB?$AA?$AA@ 0000000180004e58     libucrt:lcidtoname_downlevel.obj
 0001:00003e68       ??_C@_1M@BGNFLDN@?$AAe?$AAs?$AA?9?$AAC?$AAO?$AA?$AA@ 0000000180004e68     libucrt:lcidtoname_downlevel.obj
 0001:00003e78       ??_C@_1O@JMPHMAMC@?$AAs?$AAm?$AAn?$AA?9?$AAF?$AAI?$AA?$AA@ 0000000180004e78     libucrt:lcidtoname_downlevel.obj
 0001:00003e88       ??_C@_1M@JLANABKE@?$AAa?$AAr?$AA?9?$AAS?$AAY?$AA?$AA@ 0000000180004e88     libucrt:lcidtoname_downlevel.obj
 0001:00003e98       ??_C@_1M@HPKGCFGN@?$AAe?$AAn?$AA?9?$AAB?$AAZ?$AA?$AA@ 0000000180004e98     libucrt:lcidtoname_downlevel.obj
 0001:00003ea8       ??_C@_1M@OLJCMLGM@?$AAe?$AAs?$AA?9?$AAP?$AAE?$AA?$AA@ 0000000180004ea8     libucrt:lcidtoname_downlevel.obj
 0001:00003eb8       ??_C@_1M@MKKGFKLE@?$AAa?$AAr?$AA?9?$AAJ?$AAO?$AA?$AA@ 0000000180004eb8     libucrt:lcidtoname_downlevel.obj
 0001:00003ec8       ??_C@_1M@EKPGLDNI@?$AAe?$AAn?$AA?9?$AAT?$AAT?$AA?$AA@ 0000000180004ec8     libucrt:lcidtoname_downlevel.obj
 0001:00003ed8       ??_C@_1M@OONGHFHE@?$AAe?$AAs?$AA?9?$AAA?$AAR?$AA?$AA@ 0000000180004ed8     libucrt:lcidtoname_downlevel.obj
 0001:00003ee8       ??_C@_1M@OOJFGBHE@?$AAa?$AAr?$AA?9?$AAL?$AAB?$AA?$AA@ 0000000180004ee8     libucrt:lcidtoname_downlevel.obj
 0001:00003ef8       ??_C@_1M@GCEJHNEG@?$AAe?$AAn?$AA?9?$AAZ?$AAW?$AA?$AA@ 0000000180004ef8     libucrt:lcidtoname_downlevel.obj
 0001:00003f08       ??_C@_1M@JNOCAHJI@?$AAe?$AAs?$AA?9?$AAE?$AAC?$AA?$AA@ 0000000180004f08     libucrt:lcidtoname_downlevel.obj
 0001:00003f18       ??_C@_1M@JEFHPGGB@?$AAa?$AAr?$AA?9?$AAK?$AAW?$AA?$AA@ 0000000180004f18     libucrt:lcidtoname_downlevel.obj
 0001:00003f28       ??_C@_1M@MLKIBJOJ@?$AAe?$AAn?$AA?9?$AAP?$AAH?$AA?$AA@ 0000000180004f28     libucrt:lcidtoname_downlevel.obj
 0001:00003f38       ??_C@_1M@BDNIPEND@?$AAe?$AAs?$AA?9?$AAC?$AAL?$AA?$AA@ 0000000180004f38     libucrt:lcidtoname_downlevel.obj
 0001:00003f48       ??_C@_1M@MPNMEKBD@?$AAa?$AAr?$AA?9?$AAA?$AAE?$AA?$AA@ 0000000180004f48     libucrt:lcidtoname_downlevel.obj
 0001:00003f58       ??_C@_1M@KBJALCPI@?$AAe?$AAs?$AA?9?$AAU?$AAY?$AA?$AA@ 0000000180004f58     libucrt:lcidtoname_downlevel.obj
 0001:00003f68       ??_C@_1M@LLCCOAGA@?$AAa?$AAr?$AA?9?$AAB?$AAH?$AA?$AA@ 0000000180004f68     libucrt:lcidtoname_downlevel.obj
 0001:00003f78       ??_C@_1M@PBFNCDEL@?$AAe?$AAs?$AA?9?$AAP?$AAY?$AA?$AA@ 0000000180004f78     libucrt:lcidtoname_downlevel.obj
 0001:00003f88       ??_C@_1M@EDGINPNP@?$AAa?$AAr?$AA?9?$AAQ?$AAA?$AA?$AA@ 0000000180004f88     libucrt:lcidtoname_downlevel.obj
 0001:00003f98       ??_C@_1M@MKDBIIJI@?$AAe?$AAs?$AA?9?$AAB?$AAO?$AA?$AA@ 0000000180004f98     libucrt:lcidtoname_downlevel.obj
 0001:00003fa8       ??_C@_1M@CPKKEBLD@?$AAe?$AAs?$AA?9?$AAS?$AAV?$AA?$AA@ 0000000180004fa8     libucrt:lcidtoname_downlevel.obj
 0001:00003fb8       ??_C@_1M@NDBGMMJL@?$AAe?$AAs?$AA?9?$AAH?$AAN?$AA?$AA@ 0000000180004fb8     libucrt:lcidtoname_downlevel.obj
 0001:00003fc8       ??_C@_1M@JIJIBHDP@?$AAe?$AAs?$AA?9?$AAN?$AAI?$AA?$AA@ 0000000180004fc8     libucrt:lcidtoname_downlevel.obj
 0001:00003fd8       ??_C@_1M@CGFMKEEK@?$AAe?$AAs?$AA?9?$AAP?$AAR?$AA?$AA@ 0000000180004fd8     libucrt:lcidtoname_downlevel.obj
 0001:00003fe8       ??_C@_1O@ICJHKIIK@?$AAz?$AAh?$AA?9?$AAC?$AAH?$AAT?$AA?$AA@ 0000000180004fe8     libucrt:lcidtoname_downlevel.obj
 0001:00003ff8       ??_C@_15CLNEJCE@?$AAs?$AAr?$AA?$AA@ 0000000180004ff8     libucrt:lcidtoname_downlevel.obj
 0001:00004e40       ??_C@_1M@KAHEKEIG@?$AAa?$AAf?$AA?9?$AAz?$AAa?$AA?$AA@ 0000000180005e40     libucrt:lcidtoname_downlevel.obj
 0001:00004e50       ??_C@_1M@GIECOABL@?$AAa?$AAr?$AA?9?$AAa?$AAe?$AA?$AA@ 0000000180005e50     libucrt:lcidtoname_downlevel.obj
 0001:00004e60       ??_C@_1M@BMLMEKGI@?$AAa?$AAr?$AA?9?$AAb?$AAh?$AA?$AA@ 0000000180005e60     libucrt:lcidtoname_downlevel.obj
 0001:00004e70       ??_C@_1M@DAPFDGGB@?$AAa?$AAr?$AA?9?$AAd?$AAz?$AA?$AA@ 0000000180005e70     libucrt:lcidtoname_downlevel.obj
 0001:00004e80       ??_C@_1M@FJNKGKIG@?$AAa?$AAr?$AA?9?$AAe?$AAg?$AA?$AA@ 0000000180005e80     libucrt:lcidtoname_downlevel.obj
 0001:00004e90       ??_C@_1M@FLGKKCLO@?$AAa?$AAr?$AA?9?$AAi?$AAq?$AA?$AA@ 0000000180005e90     libucrt:lcidtoname_downlevel.obj
 0001:00004ea0       ??_C@_1M@GNDIPALM@?$AAa?$AAr?$AA?9?$AAj?$AAo?$AA?$AA@ 0000000180005ea0     libucrt:lcidtoname_downlevel.obj
 0001:00004eb0       ??_C@_1M@DDMJFMGJ@?$AAa?$AAr?$AA?9?$AAk?$AAw?$AA?$AA@ 0000000180005eb0     libucrt:lcidtoname_downlevel.obj
 0001:00004ec0       ??_C@_1M@EJALMLHM@?$AAa?$AAr?$AA?9?$AAl?$AAb?$AA?$AA@ 0000000180005ec0     libucrt:lcidtoname_downlevel.obj
 0001:00004ed0       ??_C@_1M@MOBDBLOC@?$AAa?$AAr?$AA?9?$AAl?$AAy?$AA?$AA@ 0000000180005ed0     libucrt:lcidtoname_downlevel.obj
 0001:00004ee0       ??_C@_1M@JAOCLHDH@?$AAa?$AAr?$AA?9?$AAm?$AAa?$AA?$AA@ 0000000180005ee0     libucrt:lcidtoname_downlevel.obj
 0001:00004ef0       ??_C@_1M@JHPMKJIE@?$AAa?$AAr?$AA?9?$AAo?$AAm?$AA?$AA@ 0000000180005ef0     libucrt:lcidtoname_downlevel.obj
 0001:00004f00       ??_C@_1M@OEPGHFNH@?$AAa?$AAr?$AA?9?$AAq?$AAa?$AA?$AA@ 0000000180005f00     libucrt:lcidtoname_downlevel.obj
 0001:00004f10       ??_C@_1M@KJDONENM@?$AAa?$AAr?$AA?9?$AAs?$AAa?$AA?$AA@ 0000000180005f10     libucrt:lcidtoname_downlevel.obj
 0001:00004f20       ??_C@_1M@DMJDKLKM@?$AAa?$AAr?$AA?9?$AAs?$AAy?$AA?$AA@ 0000000180005f20     libucrt:lcidtoname_downlevel.obj
 0001:00004f30       ??_C@_1M@OMFIPEDC@?$AAa?$AAr?$AA?9?$AAt?$AAn?$AA?$AA@ 0000000180005f30     libucrt:lcidtoname_downlevel.obj
 0001:00004f40       ??_C@_1M@IHMHGAON@?$AAa?$AAr?$AA?9?$AAy?$AAe?$AA?$AA@ 0000000180005f40     libucrt:lcidtoname_downlevel.obj
 0001:00004f50       ??_C@_1BG@KDCPGJGB@?$AAa?$AAz?$AA?9?$AAa?$AAz?$AA?9?$AAc?$AAy?$AAr?$AAl?$AA?$AA@ 0000000180005f50     libucrt:lcidtoname_downlevel.obj
 0001:00004f68       ??_C@_1BG@IBCKDDOE@?$AAa?$AAz?$AA?9?$AAa?$AAz?$AA?9?$AAl?$AAa?$AAt?$AAn?$AA?$AA@ 0000000180005f68     libucrt:lcidtoname_downlevel.obj
 0001:00004f80       ??_C@_1M@EGPFDCPD@?$AAb?$AAe?$AA?9?$AAb?$AAy?$AA?$AA@ 0000000180005f80     libucrt:lcidtoname_downlevel.obj
 0001:00004f90       ??_C@_1M@PCMGMCGC@?$AAb?$AAg?$AA?9?$AAb?$AAg?$AA?$AA@ 0000000180005f90     libucrt:lcidtoname_downlevel.obj
 0001:00004fa0       ??_C@_1M@BJBMFGOB@?$AAb?$AAn?$AA?9?$AAi?$AAn?$AA?$AA@ 0000000180005fa0     libucrt:lcidtoname_downlevel.obj
 0001:00004fb0       ??_C@_1BG@EAKMMACD@?$AAb?$AAs?$AA?9?$AAb?$AAa?$AA?9?$AAl?$AAa?$AAt?$AAn?$AA?$AA@ 0000000180005fb0     libucrt:lcidtoname_downlevel.obj
 0001:00004fc8       ??_C@_1M@KGADAODK@?$AAc?$AAa?$AA?9?$AAe?$AAs?$AA?$AA@ 0000000180005fc8     libucrt:lcidtoname_downlevel.obj
 0001:00004fd8       ??_C@_1M@COAJPDHI@?$AAc?$AAs?$AA?9?$AAc?$AAz?$AA?$AA@ 0000000180005fd8     libucrt:lcidtoname_downlevel.obj
 0001:00004fe8       ??_C@_1M@DHBHFONH@?$AAc?$AAy?$AA?9?$AAg?$AAb?$AA?$AA@ 0000000180005fe8     libucrt:lcidtoname_downlevel.obj
 0001:00004ff8       ??_C@_1M@IMGKELGA@?$AAd?$AAa?$AA?9?$AAd?$AAk?$AA?$AA@ 0000000180005ff8     libucrt:lcidtoname_downlevel.obj
 0001:00005008       ??_C@_1M@NNDGDNGA@?$AAd?$AAe?$AA?9?$AAa?$AAt?$AA?$AA@ 0000000180006008     libucrt:lcidtoname_downlevel.obj
 0001:00005018       ??_C@_1M@IKDBHEEM@?$AAd?$AAe?$AA?9?$AAc?$AAh?$AA?$AA@ 0000000180006018     libucrt:lcidtoname_downlevel.obj
 0001:00005028       ??_C@_1M@GFFOJMCJ@?$AAd?$AAe?$AA?9?$AAd?$AAe?$AA?$AA@ 0000000180006028     libucrt:lcidtoname_downlevel.obj
 0001:00005038       ??_C@_1M@MDNLKBPM@?$AAd?$AAe?$AA?9?$AAl?$AAi?$AA?$AA@ 0000000180006038     libucrt:lcidtoname_downlevel.obj
 0001:00005048       ??_C@_1M@NJBEEJNL@?$AAd?$AAe?$AA?9?$AAl?$AAu?$AA?$AA@ 0000000180006048     libucrt:lcidtoname_downlevel.obj
 0001:00005058       ??_C@_1O@GNNELBAP@?$AAd?$AAi?$AAv?$AA?9?$AAm?$AAv?$AA?$AA@ 0000000180006058     libucrt:lcidtoname_downlevel.obj
 0001:00005068       ??_C@_1M@EJLEOGAE@?$AAe?$AAl?$AA?9?$AAg?$AAr?$AA?$AA@ 0000000180006068     libucrt:lcidtoname_downlevel.obj
 0001:00005078       ??_C@_1M@GMPONJN@?$AAe?$AAn?$AA?9?$AAa?$AAu?$AA?$AA@ 0000000180006078     libucrt:lcidtoname_downlevel.obj
 0001:00005088       ??_C@_1M@NIDIIPGF@?$AAe?$AAn?$AA?9?$AAb?$AAz?$AA?$AA@ 0000000180006088     libucrt:lcidtoname_downlevel.obj
 0001:00005098       ??_C@_1M@JEHMIMFO@?$AAe?$AAn?$AA?9?$AAc?$AAa?$AA?$AA@ 0000000180006098     libucrt:lcidtoname_downlevel.obj
 0001:000050a8       ??_C@_1M@IGMJCDLA@?$AAe?$AAn?$AA?9?$AAc?$AAb?$AA?$AA@ 00000001800060a8     libucrt:lcidtoname_downlevel.obj
 0001:000050b8       ??_C@_1M@BNFIGBKG@?$AAe?$AAn?$AA?9?$AAg?$AAb?$AA?$AA@ 00000001800060b8     libucrt:lcidtoname_downlevel.obj
 0001:000050c8       ??_C@_1M@LKIFDIGP@?$AAe?$AAn?$AA?9?$AAi?$AAe?$AA?$AA@ 00000001800060c8     libucrt:lcidtoname_downlevel.obj
 0001:000050d8       ??_C@_1M@PJKFGCCO@?$AAe?$AAn?$AA?9?$AAj?$AAm?$AA?$AA@ 00000001800060d8     libucrt:lcidtoname_downlevel.obj
 0001:000050e8       ??_C@_1M@KPPKEPBO@?$AAe?$AAn?$AA?9?$AAn?$AAz?$AA?$AA@ 00000001800060e8     libucrt:lcidtoname_downlevel.obj
 0001:000050f8       ??_C@_1M@GMDGLDOB@?$AAe?$AAn?$AA?9?$AAp?$AAh?$AA?$AA@ 00000001800060f8     libucrt:lcidtoname_downlevel.obj
 0001:00005108       ??_C@_1M@ONGIBJNA@?$AAe?$AAn?$AA?9?$AAt?$AAt?$AA?$AA@ 0000000180006108     libucrt:lcidtoname_downlevel.obj
 0001:00005118       ??_C@_1M@LLODPCMM@?$AAe?$AAn?$AA?9?$AAu?$AAs?$AA?$AA@ 0000000180006118     libucrt:lcidtoname_downlevel.obj
 0001:00005128       ??_C@_1M@LAKFNPAN@?$AAe?$AAn?$AA?9?$AAz?$AAa?$AA?$AA@ 0000000180006128     libucrt:lcidtoname_downlevel.obj
 0001:00005138       ??_C@_1M@MFNHNHEO@?$AAe?$AAn?$AA?9?$AAz?$AAw?$AA?$AA@ 0000000180006138     libucrt:lcidtoname_downlevel.obj
 0001:00005148       ??_C@_1M@EJEINPHM@?$AAe?$AAs?$AA?9?$AAa?$AAr?$AA?$AA@ 0000000180006148     libucrt:lcidtoname_downlevel.obj
 0001:00005158       ??_C@_1M@GNKPCCJA@?$AAe?$AAs?$AA?9?$AAb?$AAo?$AA?$AA@ 0000000180006158     libucrt:lcidtoname_downlevel.obj
 0001:00005168       ??_C@_1M@LEEGFONL@?$AAe?$AAs?$AA?9?$AAc?$AAl?$AA?$AA@ 0000000180006168     libucrt:lcidtoname_downlevel.obj
 0001:00005178       ??_C@_1M@KGPDPBDF@?$AAe?$AAs?$AA?9?$AAc?$AAo?$AA?$AA@ 0000000180006178     libucrt:lcidtoname_downlevel.obj
 0001:00005188       ??_C@_1M@EIAHOHH@?$AAe?$AAs?$AA?9?$AAc?$AAr?$AA?$AA@ 0000000180006188     libucrt:lcidtoname_downlevel.obj
 0001:00005198       ??_C@_1M@LLPGMBIN@?$AAe?$AAs?$AA?9?$AAd?$AAo?$AA?$AA@ 0000000180006198     libucrt:lcidtoname_downlevel.obj
 0001:000051a8       ??_C@_1M@DKHMKNJA@?$AAe?$AAs?$AA?9?$AAe?$AAc?$AA?$AA@ 00000001800061a8     libucrt:lcidtoname_downlevel.obj
 0001:000051b8       ??_C@_1M@GKGFPKAP@?$AAe?$AAs?$AA?9?$AAe?$AAs?$AA?$AA@ 00000001800061b8     libucrt:lcidtoname_downlevel.obj
 0001:000051c8       ??_C@_1M@LKHKGDLN@?$AAe?$AAs?$AA?9?$AAg?$AAt?$AA?$AA@ 00000001800061c8     libucrt:lcidtoname_downlevel.obj
 0001:000051d8       ??_C@_1M@HEIIGGJD@?$AAe?$AAs?$AA?9?$AAh?$AAn?$AA?$AA@ 00000001800061d8     libucrt:lcidtoname_downlevel.obj
 0001:000051e8       ??_C@_1M@FBDHPPGD@?$AAe?$AAs?$AA?9?$AAm?$AAx?$AA?$AA@ 00000001800061e8     libucrt:lcidtoname_downlevel.obj
 0001:000051f8       ??_C@_1M@DPAGLNDH@?$AAe?$AAs?$AA?9?$AAn?$AAi?$AA?$AA@ 00000001800061f8     libucrt:lcidtoname_downlevel.obj
 0001:00005208       ??_C@_1M@MDGOPGDD@?$AAe?$AAs?$AA?9?$AAp?$AAa?$AA?$AA@ 0000000180006208     libucrt:lcidtoname_downlevel.obj
 0001:00005218       ??_C@_1M@EMAMGBGE@?$AAe?$AAs?$AA?9?$AAp?$AAe?$AA?$AA@ 0000000180006218     libucrt:lcidtoname_downlevel.obj
 0001:00005228       ??_C@_1M@IBMCAOEC@?$AAe?$AAs?$AA?9?$AAp?$AAr?$AA?$AA@ 0000000180006228     libucrt:lcidtoname_downlevel.obj
 0001:00005238       ??_C@_1M@FGMDIJED@?$AAe?$AAs?$AA?9?$AAp?$AAy?$AA?$AA@ 0000000180006238     libucrt:lcidtoname_downlevel.obj
 0001:00005248       ??_C@_1M@IIDEOLLL@?$AAe?$AAs?$AA?9?$AAs?$AAv?$AA?$AA@ 0000000180006248     libucrt:lcidtoname_downlevel.obj
 0001:00005258       ??_C@_1M@GAOBIPA@?$AAe?$AAs?$AA?9?$AAu?$AAy?$AA?$AA@ 0000000180006258     libucrt:lcidtoname_downlevel.obj
 0001:00005268       ??_C@_1M@JKFFICHJ@?$AAe?$AAs?$AA?9?$AAv?$AAe?$AA?$AA@ 0000000180006268     libucrt:lcidtoname_downlevel.obj
 0001:00005278       ??_C@_1M@PNMLOJDF@?$AAe?$AAt?$AA?9?$AAe?$AAe?$AA?$AA@ 0000000180006278     libucrt:lcidtoname_downlevel.obj
 0001:00005288       ??_C@_1M@GHHLIKEI@?$AAe?$AAu?$AA?9?$AAe?$AAs?$AA?$AA@ 0000000180006288     libucrt:lcidtoname_downlevel.obj
 0001:00005298       ??_C@_1M@PBNONODE@?$AAf?$AAa?$AA?9?$AAi?$AAr?$AA?$AA@ 0000000180006298     libucrt:lcidtoname_downlevel.obj
 0001:000052a8       ??_C@_1M@JEEHPMIL@?$AAf?$AAi?$AA?9?$AAf?$AAi?$AA?$AA@ 00000001800062a8     libucrt:lcidtoname_downlevel.obj
 0001:000052b8       ??_C@_1M@LMDCNDBA@?$AAf?$AAo?$AA?9?$AAf?$AAo?$AA?$AA@ 00000001800062b8     libucrt:lcidtoname_downlevel.obj
 0001:000052c8       ??_C@_1M@JKEOHLDK@?$AAf?$AAr?$AA?9?$AAb?$AAe?$AA?$AA@ 00000001800062c8     libucrt:lcidtoname_downlevel.obj
 0001:000052d8       ??_C@_1M@NOHADPMI@?$AAf?$AAr?$AA?9?$AAc?$AAa?$AA?$AA@ 00000001800062d8     libucrt:lcidtoname_downlevel.obj
 0001:000052e8       ??_C@_1M@KDHIHAEC@?$AAf?$AAr?$AA?9?$AAc?$AAh?$AA?$AA@ 00000001800062e8     libucrt:lcidtoname_downlevel.obj
 0001:000052f8       ??_C@_1M@MMBBFGAK@?$AAf?$AAr?$AA?9?$AAf?$AAr?$AA?$AA@ 00000001800062f8     libucrt:lcidtoname_downlevel.obj
 0001:00005308       ??_C@_1M@PAFNENNF@?$AAf?$AAr?$AA?9?$AAl?$AAu?$AA?$AA@ 0000000180006308     libucrt:lcidtoname_downlevel.obj
 0001:00005318       ??_C@_1M@EOHDJGDD@?$AAf?$AAr?$AA?9?$AAm?$AAc?$AA?$AA@ 0000000180006318     libucrt:lcidtoname_downlevel.obj
 0001:00005328       ??_C@_1M@FAPLLOPF@?$AAg?$AAl?$AA?9?$AAe?$AAs?$AA?$AA@ 0000000180006328     libucrt:lcidtoname_downlevel.obj
 0001:00005338       ??_C@_1M@FOPBFLOO@?$AAg?$AAu?$AA?9?$AAi?$AAn?$AA?$AA@ 0000000180006338     libucrt:lcidtoname_downlevel.obj
 0001:00005348       ??_C@_1M@KBMCINPM@?$AAh?$AAe?$AA?9?$AAi?$AAl?$AA?$AA@ 0000000180006348     libucrt:lcidtoname_downlevel.obj
 0001:00005358       ??_C@_1M@BBPHKFPJ@?$AAh?$AAi?$AA?9?$AAi?$AAn?$AA?$AA@ 0000000180006358     libucrt:lcidtoname_downlevel.obj
 0001:00005368       ??_C@_1M@PMBNDPHD@?$AAh?$AAr?$AA?9?$AAb?$AAa?$AA?$AA@ 0000000180006368     libucrt:lcidtoname_downlevel.obj
 0001:00005378       ??_C@_1M@BPCKOEGE@?$AAh?$AAr?$AA?9?$AAh?$AAr?$AA?$AA@ 0000000180006378     libucrt:lcidtoname_downlevel.obj
 0001:00005388       ??_C@_1M@GACBMHKE@?$AAh?$AAu?$AA?9?$AAh?$AAu?$AA?$AA@ 0000000180006388     libucrt:lcidtoname_downlevel.obj
 0001:00005398       ??_C@_1M@MILPAJJC@?$AAh?$AAy?$AA?9?$AAa?$AAm?$AA?$AA@ 0000000180006398     libucrt:lcidtoname_downlevel.obj
 0001:000053a8       ??_C@_1M@BABBICEC@?$AAi?$AAd?$AA?9?$AAi?$AAd?$AA?$AA@ 00000001800063a8     libucrt:lcidtoname_downlevel.obj
 0001:000053b8       ??_C@_1M@BIKNHHPF@?$AAi?$AAs?$AA?9?$AAi?$AAs?$AA?$AA@ 00000001800063b8     libucrt:lcidtoname_downlevel.obj
 0001:000053c8       ??_C@_1M@NMPCJPHE@?$AAi?$AAt?$AA?9?$AAc?$AAh?$AA?$AA@ 00000001800063c8     libucrt:lcidtoname_downlevel.obj
 0001:000053d8       ??_C@_1M@GHKGFEDF@?$AAi?$AAt?$AA?9?$AAi?$AAt?$AA?$AA@ 00000001800063d8     libucrt:lcidtoname_downlevel.obj
 0001:000053e8       ??_C@_1M@NIEJCJJA@?$AAj?$AAa?$AA?9?$AAj?$AAp?$AA?$AA@ 00000001800063e8     libucrt:lcidtoname_downlevel.obj
 0001:000053f8       ??_C@_1M@JILFNBIM@?$AAk?$AAa?$AA?9?$AAg?$AAe?$AA?$AA@ 00000001800063f8     libucrt:lcidtoname_downlevel.obj
 0001:00005408       ??_C@_1M@PACPMGPH@?$AAk?$AAk?$AA?9?$AAk?$AAz?$AA?$AA@ 0000000180006408     libucrt:lcidtoname_downlevel.obj
 0001:00005418       ??_C@_1M@IELFGMHA@?$AAk?$AAn?$AA?9?$AAi?$AAn?$AA?$AA@ 0000000180006418     libucrt:lcidtoname_downlevel.obj
 0001:00005428       ??_C@_1O@IBBJHCH@?$AAk?$AAo?$AAk?$AA?9?$AAi?$AAn?$AA?$AA@ 0000000180006428     libucrt:lcidtoname_downlevel.obj
 0001:00005438       ??_C@_1M@DMHAEOGC@?$AAk?$AAo?$AA?9?$AAk?$AAr?$AA?$AA@ 0000000180006438     libucrt:lcidtoname_downlevel.obj
 0001:00005448       ??_C@_1M@HBAHBIGA@?$AAk?$AAy?$AA?9?$AAk?$AAg?$AA?$AA@ 0000000180006448     libucrt:lcidtoname_downlevel.obj
 0001:00005458       ??_C@_1M@KPMILCJG@?$AAl?$AAt?$AA?9?$AAl?$AAt?$AA?$AA@ 0000000180006458     libucrt:lcidtoname_downlevel.obj
 0001:00005468       ??_C@_1M@BDEKKCA@?$AAl?$AAv?$AA?9?$AAl?$AAv?$AA?$AA@ 0000000180006468     libucrt:lcidtoname_downlevel.obj
 0001:00005478       ??_C@_1M@ELCKCCJJ@?$AAm?$AAi?$AA?9?$AAn?$AAz?$AA?$AA@ 0000000180006478     libucrt:lcidtoname_downlevel.obj
 0001:00005488       ??_C@_1M@CBOOLAPA@?$AAm?$AAk?$AA?9?$AAm?$AAk?$AA?$AA@ 0000000180006488     libucrt:lcidtoname_downlevel.obj
 0001:00005498       ??_C@_1M@GPHNBJKN@?$AAm?$AAl?$AA?9?$AAi?$AAn?$AA?$AA@ 0000000180006498     libucrt:lcidtoname_downlevel.obj
 0001:000054a8       ??_C@_1M@PABJILIG@?$AAm?$AAn?$AA?9?$AAm?$AAn?$AA?$AA@ 00000001800064a8     libucrt:lcidtoname_downlevel.obj
 0001:000054b8       ??_C@_1M@FGBKKIPG@?$AAm?$AAr?$AA?9?$AAi?$AAn?$AA?$AA@ 00000001800064b8     libucrt:lcidtoname_downlevel.obj
 0001:000054c8       ??_C@_1M@NDBPDDAL@?$AAm?$AAs?$AA?9?$AAb?$AAn?$AA?$AA@ 00000001800064c8     libucrt:lcidtoname_downlevel.obj
 0001:000054d8       ??_C@_1M@OPIHOOPI@?$AAm?$AAs?$AA?9?$AAm?$AAy?$AA?$AA@ 00000001800064d8     libucrt:lcidtoname_downlevel.obj
 0001:000054e8       ??_C@_1M@PPDBCNFM@?$AAm?$AAt?$AA?9?$AAm?$AAt?$AA?$AA@ 00000001800064e8     libucrt:lcidtoname_downlevel.obj
 0001:000054f8       ??_C@_1M@KDJDKMDD@?$AAn?$AAb?$AA?9?$AAn?$AAo?$AA?$AA@ 00000001800064f8     libucrt:lcidtoname_downlevel.obj
 0001:00005508       ??_C@_1M@KFCFLMJP@?$AAn?$AAl?$AA?9?$AAb?$AAe?$AA?$AA@ 0000000180006508     libucrt:lcidtoname_downlevel.obj
 0001:00005518       ??_C@_1M@KPOPDDGO@?$AAn?$AAl?$AA?9?$AAn?$AAl?$AA?$AA@ 0000000180006518     libucrt:lcidtoname_downlevel.obj
 0001:00005528       ??_C@_1M@LJKPEMLN@?$AAn?$AAn?$AA?9?$AAn?$AAo?$AA?$AA@ 0000000180006528     libucrt:lcidtoname_downlevel.obj
 0001:00005538       ??_C@_1M@BDGHHBFL@?$AAn?$AAs?$AA?9?$AAz?$AAa?$AA?$AA@ 0000000180006538     libucrt:lcidtoname_downlevel.obj
 0001:00005548       ??_C@_1M@IDEHOAP@?$AAp?$AAa?$AA?9?$AAi?$AAn?$AA?$AA@ 0000000180006548     libucrt:lcidtoname_downlevel.obj
 0001:00005558       ??_C@_1M@HDBKGOGH@?$AAp?$AAl?$AA?9?$AAp?$AAl?$AA?$AA@ 0000000180006558     libucrt:lcidtoname_downlevel.obj
 0001:00005568       ??_C@_1M@LJLLCMEH@?$AAp?$AAt?$AA?9?$AAb?$AAr?$AA?$AA@ 0000000180006568     libucrt:lcidtoname_downlevel.obj
 0001:00005578       ??_C@_1M@NCMONAAL@?$AAp?$AAt?$AA?9?$AAp?$AAt?$AA?$AA@ 0000000180006578     libucrt:lcidtoname_downlevel.obj
 0001:00005588       ??_C@_1O@EAKMAJDN@?$AAq?$AAu?$AAz?$AA?9?$AAb?$AAo?$AA?$AA@ 0000000180006588     libucrt:lcidtoname_downlevel.obj
 0001:00005598       ??_C@_1O@BHHPIGDN@?$AAq?$AAu?$AAz?$AA?9?$AAe?$AAc?$AA?$AA@ 0000000180006598     libucrt:lcidtoname_downlevel.obj
 0001:000055a8       ??_C@_1O@GBAPEKMJ@?$AAq?$AAu?$AAz?$AA?9?$AAp?$AAe?$AA?$AA@ 00000001800065a8     libucrt:lcidtoname_downlevel.obj
 0001:000055b8       ??_C@_1M@CLGLEFBO@?$AAr?$AAo?$AA?9?$AAr?$AAo?$AA?$AA@ 00000001800065b8     libucrt:lcidtoname_downlevel.obj
 0001:000055c8       ??_C@_1M@CEEDODME@?$AAr?$AAu?$AA?9?$AAr?$AAu?$AA?$AA@ 00000001800065c8     libucrt:lcidtoname_downlevel.obj
 0001:000055d8       ??_C@_1M@HPKKKMPP@?$AAs?$AAa?$AA?9?$AAi?$AAn?$AA?$AA@ 00000001800065d8     libucrt:lcidtoname_downlevel.obj
 0001:000055e8       ??_C@_1M@BKMAIGOJ@?$AAs?$AAe?$AA?9?$AAf?$AAi?$AA?$AA@ 00000001800065e8     libucrt:lcidtoname_downlevel.obj
 0001:000055f8       ??_C@_1M@NDPIFLFI@?$AAs?$AAe?$AA?9?$AAn?$AAo?$AA?$AA@ 00000001800065f8     libucrt:lcidtoname_downlevel.obj
 0001:00005608       ??_C@_1M@DANKKHJ@?$AAs?$AAe?$AA?9?$AAs?$AAe?$AA?$AA@ 0000000180006608     libucrt:lcidtoname_downlevel.obj
 0001:00005618       ??_C@_1M@PNBLONPJ@?$AAs?$AAk?$AA?9?$AAs?$AAk?$AA?$AA@ 0000000180006618     libucrt:lcidtoname_downlevel.obj
 0001:00005628       ??_C@_1M@LFMODOAL@?$AAs?$AAl?$AA?9?$AAs?$AAi?$AA?$AA@ 0000000180006628     libucrt:lcidtoname_downlevel.obj
 0001:00005638       ??_C@_1O@DFKOMPG@?$AAs?$AAm?$AAa?$AA?9?$AAn?$AAo?$AA?$AA@ 0000000180006638     libucrt:lcidtoname_downlevel.obj
 0001:00005648       ??_C@_1O@NDKPBNNH@?$AAs?$AAm?$AAa?$AA?9?$AAs?$AAe?$AA?$AA@ 0000000180006648     libucrt:lcidtoname_downlevel.obj
 0001:00005658       ??_C@_1O@PLLKBHAB@?$AAs?$AAm?$AAj?$AA?9?$AAn?$AAo?$AA?$AA@ 0000000180006658     libucrt:lcidtoname_downlevel.obj
 0001:00005668       ??_C@_1O@CLEPOGCA@?$AAs?$AAm?$AAj?$AA?9?$AAs?$AAe?$AA?$AA@ 0000000180006668     libucrt:lcidtoname_downlevel.obj
 0001:00005678       ??_C@_1O@DLGJGKMK@?$AAs?$AAm?$AAn?$AA?9?$AAf?$AAi?$AA?$AA@ 0000000180006678     libucrt:lcidtoname_downlevel.obj
 0001:00005688       ??_C@_1O@OJDJGAJC@?$AAs?$AAm?$AAs?$AA?9?$AAf?$AAi?$AA?$AA@ 0000000180006688     libucrt:lcidtoname_downlevel.obj
 0001:00005698       ??_C@_1M@BOFOGHPB@?$AAs?$AAq?$AA?9?$AAa?$AAl?$AA?$AA@ 0000000180006698     libucrt:lcidtoname_downlevel.obj
 0001:000056a8       ??_C@_1BG@LJBBIPGB@?$AAs?$AAr?$AA?9?$AAb?$AAa?$AA?9?$AAc?$AAy?$AAr?$AAl?$AA?$AA@ 00000001800066a8     libucrt:lcidtoname_downlevel.obj
 0001:000056c0       ??_C@_1BG@JLBENFOE@?$AAs?$AAr?$AA?9?$AAb?$AAa?$AA?9?$AAl?$AAa?$AAt?$AAn?$AA?$AA@ 00000001800066c0     libucrt:lcidtoname_downlevel.obj
 0001:000056d8       ??_C@_1BG@KODPNHE@?$AAs?$AAr?$AA?9?$AAs?$AAp?$AA?9?$AAc?$AAy?$AAr?$AAl?$AA?$AA@ 00000001800066d8     libucrt:lcidtoname_downlevel.obj
 0001:000056f0       ??_C@_1BG@CIOGKHPB@?$AAs?$AAr?$AA?9?$AAs?$AAp?$AA?9?$AAl?$AAa?$AAt?$AAn?$AA?$AA@ 00000001800066f0     libucrt:lcidtoname_downlevel.obj
 0001:00005708       ??_C@_1M@NGFJLMAC@?$AAs?$AAv?$AA?9?$AAf?$AAi?$AA?$AA@ 0000000180006708     libucrt:lcidtoname_downlevel.obj
 0001:00005718       ??_C@_1M@MPJEJAJC@?$AAs?$AAv?$AA?9?$AAs?$AAe?$AA?$AA@ 0000000180006718     libucrt:lcidtoname_downlevel.obj
 0001:00005728       ??_C@_1M@MPNDHLFK@?$AAs?$AAw?$AA?9?$AAk?$AAe?$AA?$AA@ 0000000180006728     libucrt:lcidtoname_downlevel.obj
 0001:00005738       ??_C@_1O@KOHBJJI@?$AAs?$AAy?$AAr?$AA?9?$AAs?$AAy?$AA?$AA@ 0000000180006738     libucrt:lcidtoname_downlevel.obj
 0001:00005748       ??_C@_1M@LDCEFHA@?$AAt?$AAa?$AA?9?$AAi?$AAn?$AA?$AA@ 0000000180006748     libucrt:lcidtoname_downlevel.obj
 0001:00005758       ??_C@_1M@CNJOFAK@?$AAt?$AAe?$AA?9?$AAi?$AAn?$AA?$AA@ 0000000180006758     libucrt:lcidtoname_downlevel.obj
 0001:00005768       ??_C@_1M@GNAECACD@?$AAt?$AAh?$AA?9?$AAt?$AAh?$AA?$AA@ 0000000180006768     libucrt:lcidtoname_downlevel.obj
 0001:00005778       ??_C@_1M@CHBIHOJO@?$AAt?$AAn?$AA?9?$AAz?$AAa?$AA?$AA@ 0000000180006778     libucrt:lcidtoname_downlevel.obj
 0001:00005788       ??_C@_1M@GCCMIGPJ@?$AAt?$AAr?$AA?9?$AAt?$AAr?$AA?$AA@ 0000000180006788     libucrt:lcidtoname_downlevel.obj
 0001:00005798       ??_C@_1M@CELMCNBK@?$AAt?$AAt?$AA?9?$AAr?$AAu?$AA?$AA@ 0000000180006798     libucrt:lcidtoname_downlevel.obj
 0001:000057a8       ??_C@_1M@KLMCELGA@?$AAu?$AAk?$AA?9?$AAu?$AAa?$AA?$AA@ 00000001800067a8     libucrt:lcidtoname_downlevel.obj
 0001:000057b8       ??_C@_1M@EPAJJAJF@?$AAu?$AAr?$AA?9?$AAp?$AAk?$AA?$AA@ 00000001800067b8     libucrt:lcidtoname_downlevel.obj
 0001:000057c8       ??_C@_1BG@GEGPMCDJ@?$AAu?$AAz?$AA?9?$AAu?$AAz?$AA?9?$AAc?$AAy?$AAr?$AAl?$AA?$AA@ 00000001800067c8     libucrt:lcidtoname_downlevel.obj
 0001:000057e0       ??_C@_1BG@EGGKJILM@?$AAu?$AAz?$AA?9?$AAu?$AAz?$AA?9?$AAl?$AAa?$AAt?$AAn?$AA?$AA@ 00000001800067e0     libucrt:lcidtoname_downlevel.obj
 0001:000057f8       ??_C@_1M@GFOCLFF@?$AAv?$AAi?$AA?9?$AAv?$AAn?$AA?$AA@ 00000001800067f8     libucrt:lcidtoname_downlevel.obj
 0001:00005808       ??_C@_1M@CPAMEDFI@?$AAx?$AAh?$AA?9?$AAz?$AAa?$AA?$AA@ 0000000180006808     libucrt:lcidtoname_downlevel.obj
 0001:00005818       ??_C@_1O@EBKIFIGN@?$AAz?$AAh?$AA?9?$AAc?$AAh?$AAs?$AA?$AA@ 0000000180006818     libucrt:lcidtoname_downlevel.obj
 0001:00005828       ??_C@_1O@NMHPGANE@?$AAz?$AAh?$AA?9?$AAc?$AAh?$AAt?$AA?$AA@ 0000000180006828     libucrt:lcidtoname_downlevel.obj
 0001:00005838       ??_C@_1M@LPINJOMC@?$AAz?$AAh?$AA?9?$AAc?$AAn?$AA?$AA@ 0000000180006838     libucrt:lcidtoname_downlevel.obj
 0001:00005848       ??_C@_1M@OCJEJODD@?$AAz?$AAh?$AA?9?$AAh?$AAk?$AA?$AA@ 0000000180006848     libucrt:lcidtoname_downlevel.obj
 0001:00005858       ??_C@_1M@DNDLJINH@?$AAz?$AAh?$AA?9?$AAm?$AAo?$AA?$AA@ 0000000180006858     libucrt:lcidtoname_downlevel.obj
 0001:00005868       ??_C@_1M@MBFDNDND@?$AAz?$AAh?$AA?9?$AAs?$AAg?$AA?$AA@ 0000000180006868     libucrt:lcidtoname_downlevel.obj
 0001:00005878       ??_C@_1M@IMEPLEPE@?$AAz?$AAh?$AA?9?$AAt?$AAw?$AA?$AA@ 0000000180006878     libucrt:lcidtoname_downlevel.obj
 0001:00005888       ??_C@_1M@BBGHNHJP@?$AAz?$AAu?$AA?9?$AAz?$AAa?$AA?$AA@ 0000000180006888     libucrt:lcidtoname_downlevel.obj
 0001:00005894       ??_C@_00CNPNBAHC@?$AA@     0000000180006894     libucrt:mbrtowc.obj
 0001:00005af0       ??_C@_1BA@BALFACEM@?$AAC?$AAO?$AAN?$AAO?$AAU?$AAT?$AA$?$AA?$AA@ 0000000180006af0     libucrt:initcon.obj
 0001:00005b00       __log10_256_lead           0000000180006b00     libucrt:log10_256_lead_tail_table.obj
 0001:00006310       __log10_256_tail           0000000180007310     libucrt:log10_256_lead_tail_table.obj
 0001:00006b20       __log_F_inv_qword          0000000180007b20     libucrt:log_f_inv_qword_table.obj
 0001:00007330       ??_C@_05HGHHAHAP@log10?$AA@ 0000000180008330     libucrt:log_special.obj
 0001:00007380       _load_config_used          0000000180008380     LIBCMT:loadcfg.obj
 0001:00007480       ??_R4exception@std@@6B@    0000000180008480     LIBCMT:throw_bad_alloc.obj
 0001:000074a8       ??_R3exception@std@@8      00000001800084a8     LIBCMT:throw_bad_alloc.obj
 0001:000074c0       ??_R2exception@std@@8      00000001800084c0     LIBCMT:throw_bad_alloc.obj
 0001:000074d0       ??_R1A@?0A@EA@exception@std@@8 00000001800084d0     LIBCMT:throw_bad_alloc.obj
 0001:000074f8       ??_R4bad_alloc@std@@6B@    00000001800084f8     LIBCMT:throw_bad_alloc.obj
 0001:00007520       ??_R3bad_alloc@std@@8      0000000180008520     LIBCMT:throw_bad_alloc.obj
 0001:00007538       ??_R2bad_alloc@std@@8      0000000180008538     LIBCMT:throw_bad_alloc.obj
 0001:00007550       ??_R1A@?0A@EA@bad_alloc@std@@8 0000000180008550     LIBCMT:throw_bad_alloc.obj
 0001:00007578       ??_R4bad_array_new_length@std@@6B@ 0000000180008578     LIBCMT:throw_bad_alloc.obj
 0001:000075a0       ??_R3bad_array_new_length@std@@8 00000001800085a0     LIBCMT:throw_bad_alloc.obj
 0001:000075b8       ??_R2bad_array_new_length@std@@8 00000001800085b8     LIBCMT:throw_bad_alloc.obj
 0001:000075d8       ??_R1A@?0A@EA@bad_array_new_length@std@@8 00000001800085d8     LIBCMT:throw_bad_alloc.obj
 0001:00007600       ??_R4type_info@@6B@        0000000180008600     LIBCMT:std_type_info_static.obj
 0001:00007628       ??_R3type_info@@8          0000000180008628     LIBCMT:std_type_info_static.obj
 0001:00007640       ??_R2type_info@@8          0000000180008640     LIBCMT:std_type_info_static.obj
 0001:00007650       ??_R1A@?0A@EA@type_info@@8 0000000180008650     LIBCMT:std_type_info_static.obj
 0001:00007928       __rtc_iaa                  0000000180008928     LIBCMT:initsect.obj
 0001:00007930       __rtc_izz                  0000000180008930     LIBCMT:initsect.obj
 0001:00007938       __rtc_taa                  0000000180008938     LIBCMT:initsect.obj
 0001:00007940       __rtc_tzz                  0000000180008940     LIBCMT:initsect.obj
 0001:00007960       _alloca_probe              0000000180008960 f   chkstk.obj
 0001:00007960       __chkstk                   0000000180008960 f   chkstk.obj
 0001:000079c0       ??1?$DialogBuilderBase@UFarDialogItem@@@@MEAA@XZ 00000001800089c0 f i SameFolder.obj
 0001:00007a40       ??_G?$DialogBuilderBase@UFarDialogItem@@@@MEAAPEAXI@Z 0000000180008a40 f i SameFolder.obj
 0001:00007a40       ??_E?$DialogBuilderBase@UFarDialogItem@@@@MEAAPEAXI@Z 0000000180008a40 f i SameFolder.obj
 0001:00007a80       ??_E?$DialogItemBinding@UFarDialogItem@@@@UEAAPEAXI@Z 0000000180008a80 f i SameFolder.obj
 0001:00007a80       ??_G?$DialogItemBinding@UFarDialogItem@@@@UEAAPEAXI@Z 0000000180008a80 f i SameFolder.obj
 0001:00007ab0       ??_EPluginCheckBoxBinding@@UEAAPEAXI@Z 0000000180008ab0 f i SameFolder.obj
 0001:00007ab0       ??_GPluginCheckBoxBinding@@UEAAPEAXI@Z 0000000180008ab0 f i SameFolder.obj
 0001:00007ae0       ??_GPluginDialogBuilder@@UEAAPEAXI@Z 0000000180008ae0 f i SameFolder.obj
 0001:00007ae0       ??_EPluginDialogBuilder@@UEAAPEAXI@Z 0000000180008ae0 f i SameFolder.obj
 0001:00007b30       ??_GPluginUIntEditFieldBinding@@UEAAPEAXI@Z 0000000180008b30 f i SameFolder.obj
 0001:00007b30       ??_GPluginIntEditFieldBinding@@UEAAPEAXI@Z 0000000180008b30 f i SameFolder.obj
 0001:00007b30       ??_EPluginUIntEditFieldBinding@@UEAAPEAXI@Z 0000000180008b30 f i SameFolder.obj
 0001:00007b30       ??_EPluginIntEditFieldBinding@@UEAAPEAXI@Z 0000000180008b30 f i SameFolder.obj
 0001:00007b60       ??_GPluginRadioButtonBinding@@UEAAPEAXI@Z 0000000180008b60 f i SameFolder.obj
 0001:00007b60       ??_EPluginRadioButtonBinding@@UEAAPEAXI@Z 0000000180008b60 f i SameFolder.obj
 0001:00007b90       ?AddButtons@?$DialogBuilderBase@UFarDialogItem@@@@QEAAXHPEBHHH@Z 0000000180008b90 f i SameFolder.obj
 0001:00007ea0       ?AddDialogItem@?$DialogBuilderBase@UFarDialogItem@@@@IEAAPEAUFarDialogItem@@W4FARDIALOGITEMTYPES@@PEB_W@Z 0000000180008ea0 f i SameFolder.obj
 0001:00008050       ?CreateCheckBoxBinding@?$DialogBuilderBase@UFarDialogItem@@@@MEAAPEAU?$DialogItemBinding@UFarDialogItem@@@@PEAHH@Z 0000000180009050 f i SameFolder.obj
 0001:00008050       ?CreateRadioButtonBinding@?$DialogBuilderBase@UFarDialogItem@@@@MEAAPEAU?$DialogItemBinding@UFarDialogItem@@@@PEAH@Z 0000000180009050 f i SameFolder.obj
 0001:00008050       ?GetLangString@?$DialogBuilderBase@UFarDialogItem@@@@MEAAPEB_WH@Z 0000000180009050 f i SameFolder.obj
 0001:00008050       ?AddIntEditField@?$DialogBuilderBase@UFarDialogItem@@@@UEAAPEAUFarDialogItem@@PEAHH@Z 0000000180009050 f i SameFolder.obj
 0001:00008050       ?AddUIntEditField@?$DialogBuilderBase@UFarDialogItem@@@@UEAAPEAUFarDialogItem@@PEAIH@Z 0000000180009050 f i SameFolder.obj
 0001:00008060       ?AddIntEditField@PluginDialogBuilder@@UEAAPEAUFarDialogItem@@PEAHH@Z 0000000180009060 f i SameFolder.obj
 0001:000081c0       ?AddUIntEditField@PluginDialogBuilder@@UEAAPEAUFarDialogItem@@PEAIH@Z 00000001800091c0 f i SameFolder.obj
 0001:00008320       ?CreateCheckBoxBinding@PluginDialogBuilder@@MEAAPEAU?$DialogItemBinding@UFarDialogItem@@@@PEAHH@Z 0000000180009320 f i SameFolder.obj
 0001:000083a0       ?CreateRadioButtonBinding@PluginDialogBuilder@@MEAAPEAU?$DialogItemBinding@UFarDialogItem@@@@PEAH@Z 00000001800093a0 f i SameFolder.obj
 0001:00008410       ?DoShowDialog@?$DialogBuilderBase@UFarDialogItem@@@@MEAA_JXZ 0000000180009410 f i SameFolder.obj
 0001:00008420       ?DoShowDialog@PluginDialogBuilder@@MEAA_JXZ 0000000180009420 f i SameFolder.obj
 0001:000084d0       ?GetLangString@PluginDialogBuilder@@MEAAPEB_WH@Z 00000001800094d0 f i SameFolder.obj
 0001:000084e0       _guard_check_icall_nop     00000001800094e0 f i LIBCMT:guard_support.obj
 0001:000084e0       ?InitDialogItem@?$DialogBuilderBase@UFarDialogItem@@@@MEAAXPEAUFarDialogItem@@PEB_W@Z 00000001800094e0 f i SameFolder.obj
 0001:000084e0       ?SaveValue@?$DialogItemBinding@UFarDialogItem@@@@UEAAXPEAUFarDialogItem@@H@Z 00000001800094e0 f i SameFolder.obj
 0001:000084f0       ?InitDialogItem@PluginDialogBuilder@@MEAAXPEAUFarDialogItem@@PEB_W@Z 00000001800094f0 f i SameFolder.obj
 0001:00008520       ?SaveValue@PluginCheckBoxBinding@@UEAAXPEAUFarDialogItem@@H@Z 0000000180009520 f i SameFolder.obj
 0001:00008580       ?SaveValue@PluginIntEditFieldBinding@@UEAAXPEAUFarDialogItem@@H@Z 0000000180009580 f i SameFolder.obj
 0001:000085d0       ?SaveValue@PluginRadioButtonBinding@@UEAAXPEAUFarDialogItem@@H@Z 00000001800095d0 f i SameFolder.obj
 0001:00008620       ?SaveValue@PluginUIntEditFieldBinding@@UEAAXPEAUFarDialogItem@@H@Z 0000000180009620 f i SameFolder.obj
 0001:00008670       ?TextWidth@?$DialogBuilderBase@UFarDialogItem@@@@MEAAHAEBUFarDialogItem@@@Z 0000000180009670 f i SameFolder.obj
 0001:00008680       ?TextWidth@PluginDialogBuilder@@MEAAHAEBUFarDialogItem@@@Z 0000000180009680 f i SameFolder.obj
 0001:00008690       ?UpdateBorderSize@?$DialogBuilderBase@UFarDialogItem@@@@IEAAXXZ 0000000180009690 f i SameFolder.obj
 0001:00008870       ConfigureW                 0000000180009870 f   SameFolder.obj
 0001:00008eb0       GetGlobalInfoW             0000000180009eb0 f   SameFolder.obj
 0001:00008f30       GetPluginInfoW             0000000180009f30 f   SameFolder.obj
 0001:00009010       OpenW                      000000018000a010 f   SameFolder.obj
 0001:00009370       SetStartupInfoW            000000018000a370 f   SameFolder.obj
 0001:000095a8       ??2@YAPEAX_K@Z             000000018000a5a8 f   LIBCMT:new_scalar.obj
 0001:000095e4       ??_V@YAXPEAX@Z             000000018000a5e4 f   LIBCMT:delete_array.obj
 0001:000095e4       ??3@YAXPEAX_K@Z            000000018000a5e4 f   LIBCMT:delete_scalar_size.obj
 0001:000095ec       ??_U@YAPEAX_K@Z            000000018000a5ec f   LIBCMT:new_array.obj
 0001:00009924       _DllMainCRTStartup         000000018000a924 f   LIBCMT:dll_dllmain.obj
 0001:00009964       ??0bad_alloc@std@@QEAA@AEBV01@@Z 000000018000a964 f i LIBCMT:throw_bad_alloc.obj
 0001:000099a4       ??0bad_alloc@std@@QEAA@XZ  000000018000a9a4 f i LIBCMT:throw_bad_alloc.obj
 0001:000099c4       ??0bad_array_new_length@std@@QEAA@AEBV01@@Z 000000018000a9c4 f i LIBCMT:throw_bad_alloc.obj
 0001:00009a04       ??0bad_array_new_length@std@@QEAA@XZ 000000018000aa04 f i LIBCMT:throw_bad_alloc.obj
 0001:00009a24       ??0exception@std@@QEAA@AEBV01@@Z 000000018000aa24 f i LIBCMT:throw_bad_alloc.obj
 0001:00009a5c       ??1bad_alloc@std@@UEAA@XZ  000000018000aa5c f i LIBCMT:throw_bad_alloc.obj
 0001:00009a5c       ??1bad_array_new_length@std@@UEAA@XZ 000000018000aa5c f i LIBCMT:throw_bad_alloc.obj
 0001:00009a70       ??_Gbad_array_new_length@std@@UEAAPEAXI@Z 000000018000aa70 f i LIBCMT:throw_bad_alloc.obj
 0001:00009a70       ??_Gbad_alloc@std@@UEAAPEAXI@Z 000000018000aa70 f i LIBCMT:throw_bad_alloc.obj
 0001:00009a70       ??_Eexception@std@@UEAAPEAXI@Z 000000018000aa70 f i LIBCMT:throw_bad_alloc.obj
 0001:00009a70       ??_Ebad_alloc@std@@UEAAPEAXI@Z 000000018000aa70 f i LIBCMT:throw_bad_alloc.obj
 0001:00009a70       ??_Ebad_array_new_length@std@@UEAAPEAXI@Z 000000018000aa70 f i LIBCMT:throw_bad_alloc.obj
 0001:00009a70       ??_Gexception@std@@UEAAPEAXI@Z 000000018000aa70 f i LIBCMT:throw_bad_alloc.obj
 0001:00009ab4       ?__scrt_throw_std_bad_alloc@@YAXXZ 000000018000aab4 f   LIBCMT:throw_bad_alloc.obj
 0001:00009ad4       ?__scrt_throw_std_bad_array_new_length@@YAXXZ 000000018000aad4 f   LIBCMT:throw_bad_alloc.obj
 0001:00009af4       ?what@exception@std@@UEBAPEBDXZ 000000018000aaf4 f i LIBCMT:throw_bad_alloc.obj
 0001:00009b08       ??3@YAXPEAX@Z              000000018000ab08 f   LIBCMT:delete_scalar.obj
 0001:00009b10       __security_init_cookie     000000018000ab10 f   LIBCMT:gs_support.obj
 0001:00009bbc       DllMain                    000000018000abbc f   LIBCMT:dll_dllmain_stub.obj
 0001:00009bbc       _get_startup_argv_mode     000000018000abbc f   LIBCMT:argv_mode.obj
 0001:00009bc4       ?__scrt_initialize_type_info@@YAXXZ 000000018000abc4 f   LIBCMT:tncleanup.obj
 0001:00009bd4       ?__scrt_uninitialize_type_info@@YAXXZ 000000018000abd4 f   LIBCMT:tncleanup.obj
 0001:00009be0       __local_stdio_printf_options 000000018000abe0 f i LIBCMT:default_local_stdio_options.obj
 0001:00009be8       __local_stdio_scanf_options 000000018000abe8 f i LIBCMT:default_local_stdio_options.obj
 0001:00009bf0       __scrt_initialize_default_local_stdio_options 000000018000abf0 f   LIBCMT:default_local_stdio_options.obj
 0001:00009c0c       __scrt_acquire_startup_lock 000000018000ac0c f   LIBCMT:utility.obj
 0001:00009c48       __scrt_dllmain_after_initialize_c 000000018000ac48 f   LIBCMT:utility.obj
 0001:00009c7c       __scrt_dllmain_before_initialize_c 000000018000ac7c f   LIBCMT:utility.obj
 0001:00009c94       __scrt_dllmain_crt_thread_attach 000000018000ac94 f   LIBCMT:utility.obj
 0001:00009cbc       __scrt_dllmain_crt_thread_detach 000000018000acbc f   LIBCMT:utility.obj
 0001:00009cd4       __scrt_dllmain_exception_filter 000000018000acd4 f   LIBCMT:utility.obj
 0001:00009d34       __scrt_dllmain_uninitialize_c 000000018000ad34 f   LIBCMT:utility.obj
 0001:00009d64       __scrt_dllmain_uninitialize_critical 000000018000ad64 f   LIBCMT:utility.obj
 0001:00009d78       __scrt_initialize_crt      000000018000ad78 f   LIBCMT:utility.obj
 0001:00009dc4       __scrt_initialize_onexit_tables 000000018000adc4 f   LIBCMT:utility.obj
 0001:00009e9c       __scrt_is_nonwritable_in_current_image 000000018000ae9c f   LIBCMT:utility.obj
 0001:00009f38       __scrt_release_startup_lock 000000018000af38 f   LIBCMT:utility.obj
 0001:00009f5c       __scrt_uninitialize_crt    000000018000af5c f   LIBCMT:utility.obj
 0001:00009f88       __scrt_get_dyn_tls_init_callback 000000018000af88 f   LIBCMT:dyn_tls_init.obj
 0001:00009f90       __crt_debugger_hook        000000018000af90 f   LIBCMT:utility_desktop.obj
 0001:00009f98       __scrt_fastfail            000000018000af98 f   LIBCMT:utility_desktop.obj
 0001:0000a0e4       _RTC_Initialize            000000018000b0e4 f   LIBCMT:initsect.obj
 0001:0000a120       _RTC_Terminate             000000018000b120 f   LIBCMT:initsect.obj
 0001:0000a15c       ??_Etype_info@@UEAAPEAXI@Z 000000018000b15c f i LIBCMT:std_type_info_static.obj
 0001:0000a15c       ??_Gtype_info@@UEAAPEAXI@Z 000000018000b15c f i LIBCMT:std_type_info_static.obj
 0001:0000a188       __isa_available_init       000000018000b188 f   LIBCMT:cpu_disp.obj
 0001:0000a304       __scrt_is_ucrt_dll_in_use  000000018000b304 f   LIBCMT:ucrt_detection.obj
 0001:0000a320       memset_repmovs             000000018000b320 f   libvcruntime:memset.obj
 0001:0000a340       memset                     000000018000b340 f   libvcruntime:memset.obj
 0001:0000a4d0       __C_specific_handler       000000018000b4d0 f   libvcruntime:riscchandler.obj
 0001:0000a6dc       __std_exception_copy       000000018000b6dc f   libvcruntime:std_exception.obj
 0001:0000a76c       __std_exception_destroy    000000018000b76c f   libvcruntime:std_exception.obj
 0001:0000a794       _CxxThrowException         000000018000b794 f   libvcruntime:throw.obj
 0001:0000a854       __std_type_info_destroy_list 000000018000b854 f   libvcruntime:std_type_info.obj
 0001:0000a880       __vcrt_initialize          000000018000b880 f   libvcruntime:initialization.obj
 0001:0000a8b4       __vcrt_thread_attach       000000018000b8b4 f   libvcruntime:initialization.obj
 0001:0000a8c8       __vcrt_thread_detach       000000018000b8c8 f   libvcruntime:initialization.obj
 0001:0000a8dc       __vcrt_uninitialize        000000018000b8dc f   libvcruntime:initialization.obj
 0001:0000a8fc       __vcrt_uninitialize_critical 000000018000b8fc f   libvcruntime:initialization.obj
 0001:0000a920       _NLG_Notify                000000018000b920 f   libvcruntime:notify.obj
 0001:0000a940       __NLG_Dispatch2            000000018000b940 f   libvcruntime:notify.obj
 0001:0000a950       __NLG_Return2              000000018000b950 f   libvcruntime:notify.obj
 0001:0000a954       __except_validate_context_record 000000018000b954 f   libvcruntime:jbcxrval.obj
 0001:0000a98c       __DestructExceptionObject  000000018000b98c f   libvcruntime:ehhelpers.obj
 0001:0000aa00       ?_CallMemberFunction0@@YAXQEAX0@Z 000000018000ba00 f i libvcruntime:ehhelpers.obj
 0001:0000aa04       __vcrt_freefls             000000018000ba04 f   libvcruntime:per_thread_data.obj
 0001:0000aa24       __vcrt_freeptd             000000018000ba24 f   libvcruntime:per_thread_data.obj
 0001:0000aa74       __vcrt_getptd_noexit       000000018000ba74 f   libvcruntime:per_thread_data.obj
 0001:0000ab40       __vcrt_initialize_ptd      000000018000bb40 f   libvcruntime:per_thread_data.obj
 0001:0000ab94       __vcrt_uninitialize_ptd    000000018000bb94 f   libvcruntime:per_thread_data.obj
 0001:0000abb8       __vcrt_initialize_locks    000000018000bbb8 f   libvcruntime:locks.obj
 0001:0000ac00       __vcrt_uninitialize_locks  000000018000bc00 f   libvcruntime:locks.obj
 0001:0000ae10       __vcrt_FlsAlloc            000000018000be10 f   libvcruntime:winapi_downlevel.obj
 0001:0000ae58       __vcrt_FlsFree             000000018000be58 f   libvcruntime:winapi_downlevel.obj
 0001:0000aea0       __vcrt_FlsGetValue         000000018000bea0 f   libvcruntime:winapi_downlevel.obj
 0001:0000aee8       __vcrt_FlsSetValue         000000018000bee8 f   libvcruntime:winapi_downlevel.obj
 0001:0000af3c       __vcrt_InitializeCriticalSectionEx 000000018000bf3c f   libvcruntime:winapi_downlevel.obj
 0001:0000afa0       __vcrt_initialize_winapi_thunks 000000018000bfa0 f   libvcruntime:winapi_downlevel.obj
 0001:0000afd0       __vcrt_uninitialize_winapi_thunks 000000018000bfd0 f   libvcruntime:winapi_downlevel.obj
 0001:0000b010       __vcrt_initialize_pure_virtual_call_handler 000000018000c010 f   libvcruntime:purevirt_data.obj
 0001:0000b030       memcpy_repmovs             000000018000c030 f   libvcruntime:memcpy.obj
 0001:0000b050       memcpy                     000000018000c050 f   libvcruntime:memcpy.obj
 0001:0000b050       memmove                    000000018000c050 f   libvcruntime:memcpy.obj
 0001:0000b490       _CallSettingFrame          000000018000c490 f   libvcruntime:handlers.obj
 0001:0000b4e0       _CallSettingFrameEncoded   000000018000c4e0 f   libvcruntime:handlers.obj
 0001:0000b528       free                       000000018000c528 f   libucrt:free.obj
 0001:0000b53c       malloc                     000000018000c53c f   libucrt:malloc.obj
 0001:0000b544       __acrt_initialize_new_handler 000000018000c544 f   libucrt:new_handler.obj
 0001:0000b54c       _callnewh                  000000018000c54c f   libucrt:new_handler.obj
 0001:0000b57c       _query_new_handler         000000018000c57c f   libucrt:new_handler.obj
 0001:0000b5b0       _initterm                  000000018000c5b0 f   libucrt:initterm.obj
 0001:0000b614       _initterm_e                000000018000c614 f   libucrt:initterm.obj
 0001:0000b654       _seh_filter_dll            000000018000c654 f   libucrt:exception_filter.obj
 0001:0000b668       _seh_filter_exe            000000018000c668 f   libucrt:exception_filter.obj
 0001:0000ba58       __acrt_initialize_thread_local_exit_callback 000000018000ca58 f   libucrt:exit.obj
 0001:0000ba60       _cexit                     000000018000ca60 f   libucrt:exit.obj
 0001:0000ba70       _exit                      000000018000ca70 f   libucrt:exit.obj
 0001:0000ba7c       _is_c_termination_complete 000000018000ca7c f   libucrt:exit.obj
 0001:0000bc48       __acrt_allocate_buffer_for_argv 000000018000cc48 f   libucrt:argv_parsing.obj
 0001:0000bca8       _configure_narrow_argv     000000018000cca8 f   libucrt:argv_parsing.obj
 0001:0000c020       __dcrt_uninitialize_environments_nolock 000000018000d020 f   libucrt:environment_initialization.obj
 0001:0000c058       _initialize_narrow_environment 000000018000d058 f   libucrt:environment_initialization.obj
 0001:0000c1b4       _execute_onexit_table      000000018000d1b4 f   libucrt:onexit.obj
 0001:0000c1f0       _initialize_onexit_table   000000018000d1f0 f   libucrt:onexit.obj
 0001:0000c250       __acrt_uninitialize_command_line 000000018000d250 f   libucrt:argv_data.obj
 0001:0000c348       __acrt_initialize          000000018000d348 f   libucrt:initialization.obj
 0001:0000c35c       __acrt_thread_attach       000000018000d35c f   libucrt:initialization.obj
 0001:0000c370       __acrt_thread_detach       000000018000d370 f   libucrt:initialization.obj
 0001:0000c380       __acrt_uninitialize        000000018000d380 f   libucrt:initialization.obj
 0001:0000c3b8       __acrt_uninitialize_critical 000000018000d3b8 f   libucrt:initialization.obj
 0001:0000c3c8       terminate                  000000018000d3c8 f   libucrt:terminate.obj
 0001:0000c3e8       strcpy_s                   000000018000d3e8 f   libucrt:strcpy_s.obj
 0001:0000c448       ??0_LocaleUpdate@@QEAA@QEAU__crt_locale_pointers@@@Z 000000018000d448 f i libucrt:output.obj
 0001:0000c500       strncmp                    000000018000d500 f   libucrt:strncmp.obj
 0001:0000c580       abort                      000000018000d580 f   libucrt:abort.obj
 0001:0000c5d8       calloc                     000000018000d5d8 f   libucrt:calloc.obj
 0001:0000c5e0       wcsncmp                    000000018000d5e0 f   libucrt:wcsncmp.obj
 0001:0000c60c       _free_base                 000000018000d60c f   libucrt:free_base.obj
 0001:0000c64c       _malloc_base               000000018000d64c f   libucrt:malloc_base.obj
 0001:0000c6ac       __acrt_initialize_locks    000000018000d6ac f   libucrt:locks.obj
 0001:0000c6f4       __acrt_lock                000000018000d6f4 f   libucrt:locks.obj
 0001:0000c710       __acrt_uninitialize_locks  000000018000d710 f   libucrt:locks.obj
 0001:0000c748       __acrt_unlock              000000018000d748 f   libucrt:locks.obj
 0001:0000cadc       __acrt_freeptd             000000018000dadc f   libucrt:per_thread_data.obj
 0001:0000cb20       __acrt_getptd              000000018000db20 f   libucrt:per_thread_data.obj
 0001:0000cbf4       __acrt_getptd_head         000000018000dbf4 f   libucrt:per_thread_data.obj
 0001:0000cc9c       __acrt_getptd_noexit       000000018000dc9c f   libucrt:per_thread_data.obj
 0001:0000cd68       __acrt_initialize_ptd      000000018000dd68 f   libucrt:per_thread_data.obj
 0001:0000cda4       __acrt_uninitialize_ptd    000000018000dda4 f   libucrt:per_thread_data.obj
 0001:0000cdc8       __acrt_get_process_end_policy 000000018000ddc8 f   libucrt:win_policies.obj
 0001:0000ce04       __acrt_call_reportfault    000000018000de04 f   libucrt:invalid_parameter.obj
 0001:0000cf60       __acrt_initialize_invalid_parameter_handler 000000018000df60 f   libucrt:invalid_parameter.obj
 0001:0000cf68       _invalid_parameter         000000018000df68 f   libucrt:invalid_parameter.obj
 0001:0000d018       _invalid_parameter_noinfo  000000018000e018 f   libucrt:invalid_parameter.obj
 0001:0000d038       _invoke_watson             000000018000e038 f   libucrt:invalid_parameter.obj
 0001:0000d080       __acrt_errno_from_os_error 000000018000e080 f   libucrt:errno.obj
 0001:0000d0c8       __acrt_errno_map_os_error  000000018000e0c8 f   libucrt:errno.obj
 0001:0000d118       __doserrno                 000000018000e118 f   libucrt:errno.obj
 0001:0000d138       _errno                     000000018000e138 f   libucrt:errno.obj
 0001:0000d158       _calloc_base               000000018000e158 f   libucrt:calloc_base.obj
 0001:0000d1e4       ??$__acrt_mbs_to_wcs_cp@U__crt_win32_buffer_internal_dynamic_resizing@@@@YAHQEBDAEAV?$__crt_win32_buffer@_WU__crt_win32_buffer_internal_dynamic_resizing@@@@I@Z 000000018000e1e4 f i libucrt:argv_wildcards.obj
 0001:0000d35c       ??$__acrt_wcs_to_mbs_cp@U__crt_win32_buffer_internal_dynamic_resizing@@@@YAHQEB_WAEAV?$__crt_win32_buffer@DU__crt_win32_buffer_internal_dynamic_resizing@@@@I@Z 000000018000e35c f i libucrt:argv_wildcards.obj
 0001:0000db8c       __acrt_expand_narrow_argv_wildcards 000000018000eb8c f   libucrt:argv_wildcards.obj
 0001:0000db94       ??$__acrt_wcs_to_mbs_cp@U__crt_win32_buffer_no_resizing@@@@YAHQEB_WAEAV?$__crt_win32_buffer@DU__crt_win32_buffer_no_resizing@@@@I@Z 000000018000eb94 f i libucrt:getmodulefilenamea.obj
 0001:0000dca8       __acrt_GetModuleFileNameA  000000018000eca8 f   libucrt:getmodulefilenamea.obj
 0001:0000e4f4       __acrt_initialize_multibyte 000000018000f4f4 f   libucrt:mbctype.obj
 0001:0000e554       __acrt_update_thread_multibyte_data 000000018000f554 f   libucrt:mbctype.obj
 0001:0000e570       _setmbcp_nolock            000000018000f570 f   libucrt:mbctype.obj
 0001:0000e8a4       _ismbblead                 000000018000f8a4 f   libucrt:ismbbyte.obj
 0001:0000e8b8       __acrt_initialize_command_line 000000018000f8b8 f   libucrt:argv_data.obj
 0001:0000e8e0       __acrt_MultiByteToWideChar 000000018000f8e0 f   libucrt:multibytetowidechar.obj
 0001:0000e93c       __acrt_WideCharToMultiByte 000000018000f93c f   libucrt:widechartomultibyte.obj
 0001:0000e9d4       __dcrt_get_narrow_environment_from_os 000000018000f9d4 f   libucrt:get_environment_from_os.obj
 0001:0000ead8       _recalloc_base             000000018000fad8 f   libucrt:recalloc.obj
 0001:0000ed48       __acrt_AppPolicyGetProcessTerminationMethodInternal 000000018000fd48 f   libucrt:winapi_thunks.obj
 0001:0000ed98       __acrt_AreFileApisANSI     000000018000fd98 f   libucrt:winapi_thunks.obj
 0001:0000edd4       __acrt_FlsAlloc            000000018000fdd4 f   libucrt:winapi_thunks.obj
 0001:0000ee1c       __acrt_FlsFree             000000018000fe1c f   libucrt:winapi_thunks.obj
 0001:0000ee64       __acrt_FlsGetValue         000000018000fe64 f   libucrt:winapi_thunks.obj
 0001:0000eeac       __acrt_FlsSetValue         000000018000feac f   libucrt:winapi_thunks.obj
 0001:0000ef00       __acrt_InitializeCriticalSectionEx 000000018000ff00 f   libucrt:winapi_thunks.obj
 0001:0000ef64       __acrt_LCMapStringEx       000000018000ff64 f   libucrt:winapi_thunks.obj
 0001:0000f040       __acrt_LocaleNameToLCID    0000000180010040 f   libucrt:winapi_thunks.obj
 0001:0000f090       __acrt_initialize_winapi_thunks 0000000180010090 f   libucrt:winapi_thunks.obj
 0001:0000f0c4       __acrt_uninitialize_winapi_thunks 00000001800100c4 f   libucrt:winapi_thunks.obj
 0001:0000f108       __acrt_initialize_heap     0000000180010108 f   libucrt:heap_handle.obj
 0001:0000f124       __acrt_uninitialize_heap   0000000180010124 f   libucrt:heap_handle.obj
 0001:0000f32c       __acrt_initialize_lowio    000000018001032c f   libucrt:ioinit.obj
 0001:0000f368       __acrt_uninitialize_lowio  0000000180010368 f   libucrt:ioinit.obj
 0001:0000f3a8       __acrt_execute_initializers 00000001800103a8 f   libucrt:shared_initialization.obj
 0001:0000f428       __acrt_execute_uninitializers 0000000180010428 f   libucrt:shared_initialization.obj
 0001:0000f4ac       __acrt_get_sigabrt_handler 00000001800104ac f   libucrt:signal.obj
 0001:0000f4dc       __acrt_initialize_signal_handlers 00000001800104dc f   libucrt:signal.obj
 0001:0000f4fc       raise                      00000001800104fc f   libucrt:signal.obj
 0001:0000f768       __acrt_has_user_matherr    0000000180010768 f   libucrt:matherr.obj
 0001:0000f788       __acrt_initialize_user_matherr 0000000180010788 f   libucrt:matherr.obj
 0001:0000f790       __acrt_invoke_user_matherr 0000000180010790 f   libucrt:matherr.obj
 0001:0000f99c       __acrt_stdio_flush_nolock  000000018001099c f   libucrt:fflush.obj
 0001:0000fa18       _fflush_nolock             0000000180010a18 f   libucrt:fflush.obj
 0001:0000fa64       _flushall                  0000000180010a64 f   libucrt:fflush.obj
 0001:0000fa6c       __acrt_initialize_stdio    0000000180010a6c f   libucrt:_file.obj
 0001:0000fb8c       __acrt_uninitialize_stdio  0000000180010b8c f   libucrt:_file.obj
 0001:0000fbe8       _lock_file                 0000000180010be8 f   libucrt:_file.obj
 0001:0000fbf4       _unlock_file               0000000180010bf4 f   libucrt:_file.obj
 0001:0000fc00       _mbtowc_l                  0000000180010c00 f   libucrt:mbtowc.obj
 0001:0000fd7c       mbtowc                     0000000180010d7c f   libucrt:mbtowc.obj
 0001:0000fd84       __acrt_update_locale_info  0000000180010d84 f   libucrt:locale_update.obj
 0001:0000fdb8       __acrt_update_multibyte_info 0000000180010db8 f   libucrt:locale_update.obj
 0001:0000fdec       _fileno                    0000000180010dec f   libucrt:fileno.obj
 0001:0000fe84       __acrt_set_locale_changed  0000000180010e84 f   libucrt:wsetlocale.obj
 0001:0000fe90       __acrt_uninitialize_locale 0000000180010e90 f   libucrt:wsetlocale.obj
 0001:0000fec0       __pctype_func              0000000180010ec0 f   libucrt:ctype.obj
 0001:0000fef0       _query_new_mode            0000000180010ef0 f   libucrt:new_mode.obj
 0001:0000fef8       __acrt_add_locale_ref      0000000180010ef8 f   libucrt:locale_refcounting.obj
 0001:0000ff84       __acrt_free_locale         0000000180010f84 f   libucrt:locale_refcounting.obj
 0001:000100fc       __acrt_locale_add_lc_time_reference 00000001800110fc f   libucrt:locale_refcounting.obj
 0001:00010124       __acrt_locale_free_lc_time_if_unreferenced 0000000180011124 f   libucrt:locale_refcounting.obj
 0001:0001015c       __acrt_locale_release_lc_time_reference 000000018001115c f   libucrt:locale_refcounting.obj
 0001:00010184       __acrt_release_locale_ref  0000000180011184 f   libucrt:locale_refcounting.obj
 0001:0001022c       __acrt_update_thread_locale_data 000000018001122c f   libucrt:locale_refcounting.obj
 0001:0001029c       _updatetlocinfoEx_nolock   000000018001129c f   libucrt:locale_refcounting.obj
 0001:00010310       qsort                      0000000180011310 f   libucrt:qsort.obj
 0001:000106d0       strncpy_s                  00000001800116d0 f   libucrt:strncpy_s.obj
 0001:00010850       strpbrk                    0000000180011850 f   libucrt:strpbrk.obj
 0001:00010c30       _mbsdec                    0000000180011c30 f   libucrt:mbsdec.obj
 0001:00010c38       _mbsdec_l                  0000000180011c38 f   libucrt:mbsdec.obj
 0001:00010ccc       __acrt_GetStringTypeA      0000000180011ccc f   libucrt:getstringtypea.obj
 0001:00011174       __acrt_LCMapStringA        0000000180012174 f   libucrt:lcmapstringa.obj
 0001:00011224       _msize_base                0000000180012224 f   libucrt:msize.obj
 0001:00011260       _realloc_base              0000000180012260 f   libucrt:realloc_base.obj
 0001:000113c4       __acrt_DownlevelLocaleNameToLCID 00000001800123c4 f   libucrt:lcidtoname_downlevel.obj
 0001:000113f8       __acrt_lowio_create_handle_array 00000001800123f8 f   libucrt:osfinfo.obj
 0001:000114a0       __acrt_lowio_destroy_handle_array 00000001800124a0 f   libucrt:osfinfo.obj
 0001:000114f0       __acrt_lowio_ensure_fh_exists 00000001800124f0 f   libucrt:osfinfo.obj
 0001:00011598       __acrt_lowio_lock_fh       0000000180012598 f   libucrt:osfinfo.obj
 0001:000115c0       __acrt_lowio_unlock_fh     00000001800125c0 f   libucrt:osfinfo.obj
 0001:000115e8       _free_osfhnd               00000001800125e8 f   libucrt:osfinfo.obj
 0001:000116a4       _get_osfhandle             00000001800126a4 f   libucrt:osfinfo.obj
 0001:000117a8       _commit                    00000001800127a8 f   libucrt:commit.obj
 0001:000120a8       _write                     00000001800130a8 f   libucrt:write.obj
 0001:00012194       _write_nolock              0000000180013194 f   libucrt:write.obj
 0001:00012470       _fcloseall                 0000000180013470 f   libucrt:closeall.obj
 0001:00012524       __acrt_stdio_free_buffer_nolock 0000000180013524 f   libucrt:_freebuf.obj
 0001:00012564       _isatty                    0000000180013564 f   libucrt:isatty.obj
 0001:000125c4       _isleadbyte_l              00000001800135c4 f i libucrt:_wctype.obj
 0001:00012610       ?__mbrtowc_utf8@__crt_mbstring@@YA_KPEA_WPEBD_KPEAU_Mbstatet@@@Z 0000000180013610 f   libucrt:mbrtowc.obj
 0001:0001264c       ?__mbsrtowcs_utf8@__crt_mbstring@@YA_KPEA_WPEAPEBD_KPEAU_Mbstatet@@@Z 000000018001364c f   libucrt:mbrtowc.obj
 0001:000127c4       __acrt_locale_free_monetary 00000001800137c4 f   libucrt:initmon.obj
 0001:000128d0       __acrt_locale_free_numeric 00000001800138d0 f   libucrt:initnum.obj
 0001:00012994       __acrt_locale_free_time    0000000180013994 f   libucrt:inittime.obj
 0001:00012a9c       __strncnt                  0000000180013a9c f   libucrt:strncnt.obj
 0001:00012ab4       _query_app_type            0000000180013ab4 f   libucrt:report_runtime_error.obj
 0001:00012b58       _lseeki64_nolock           0000000180013b58 f   libucrt:lseek.obj
 0001:00012b60       _putwch_nolock             0000000180013b60 f   libucrt:putwch.obj
 0001:00012b9c       _fclose_nolock             0000000180013b9c f   libucrt:fclose.obj
 0001:00012c20       fclose                     0000000180013c20 f   libucrt:fclose.obj
 0001:00012c84       ?__mbrtoc32_utf8@__crt_mbstring@@YA_KPEA_UPEBD_KPEAU_Mbstatet@@@Z 0000000180013c84 f   libucrt:mbrtoc32.obj
 0001:00012e60       log10                      0000000180013e60 f   libucrt:log10.obj
 0001:0001340c       __dcrt_lowio_ensure_console_output_initialized 000000018001440c f   libucrt:initcon.obj
 0001:00013460       __dcrt_terminate_console_output 0000000180014460 f   libucrt:initcon.obj
 0001:0001347c       __dcrt_write_console       000000018001447c f   libucrt:initcon.obj
 0001:000135b0       _close                     00000001800145b0 f   libucrt:close.obj
 0001:00013654       _close_nolock              0000000180014654 f   libucrt:close.obj
 0001:00013714       ?__acrt_stdio_free_stream@@YAXV__crt_stdio_stream@@@Z 0000000180014714 f   libucrt:stream.obj
 0001:00013854       _handle_error              0000000180014854 f   libucrt:libm_error.obj
 0001:00013980       __acrt_initialize_fma3     0000000180014980 f   libucrt:fma3_available.obj
 0001:000139f0       _log10_special             00000001800149f0 f   libucrt:log_special.obj
 0001:00013ac0       _get_fpsr                  0000000180014ac0 f   libucrt:fpsr.obj
 0001:00013ad0       _set_fpsr                  0000000180014ad0 f   libucrt:fpsr.obj
 0001:00013ada       _fclrf                     0000000180014ada f   libucrt:fpsr.obj
 0001:00013aee       _frnd                      0000000180014aee f   libucrt:fpsr.obj
 0001:00013b10       _raise_exc                 0000000180014b10 f   libucrt:fpexcept.obj
 0001:00013b38       _raise_exc_ex              0000000180014b38 f   libucrt:fpexcept.obj
 0001:00013e48       _set_errno_from_matherr    0000000180014e48 f   libucrt:fpexcept.obj
 0001:00013e78       _clrfp                     0000000180014e78 f   libucrt:fpctrl.obj
 0001:00013e98       _ctrlfp                    0000000180014e98 f   libucrt:fpctrl.obj
 0001:00013f14       _set_statfp                0000000180014f14 f   libucrt:fpctrl.obj
 0001:00013f34       _statfp                    0000000180014f34 f   libucrt:fpctrl.obj
 0001:00013f45       IsProcessorFeaturePresent  0000000180014f45 f   kernel32:KERNEL32.dll
 0001:00013f50       _FindPESection             0000000180014f50 f   LIBCMT:pesect.obj
 0001:00013fa0       _IsNonwritableInCurrentImage 0000000180014fa0 f   LIBCMT:pesect.obj
 0001:00013ff0       _ValidateImageBase         0000000180014ff0 f   LIBCMT:pesect.obj
 0001:00014020       __GSHandlerCheck           0000000180015020 f   LIBCMT:gshandler.obj
 0001:00014040       __GSHandlerCheckCommon     0000000180015040 f   LIBCMT:gshandler.obj
 0001:000140b0       __security_check_cookie    00000001800150b0 f   LIBCMT:amdsecgs.obj
 0001:000140d4       __raise_securityfailure    00000001800150d4 f   LIBCMT:gs_report.obj
 0001:00014108       __report_gsfailure         0000000180015108 f   LIBCMT:gs_report.obj
 0001:000141dc       __report_rangecheckfailure 00000001800151dc f   LIBCMT:gs_report.obj
 0001:000141f0       __report_securityfailure   00000001800151f0 f   LIBCMT:gs_report.obj
 0001:00014380       memcmp                     0000000180015380 f   libvcruntime:memcmp.obj
 0001:00014460       _guard_dispatch_icall_nop  0000000180015460 f   LIBCMT:guard_dispatch.obj
 0001:00015368       _TI2?AVbad_alloc@std@@     0000000180016368     LIBCMT:throw_bad_alloc.obj
 0001:00015388       _CTA2?AVbad_alloc@std@@    0000000180016388     LIBCMT:throw_bad_alloc.obj
 0001:000153a0       _CT??_R0?AVbad_alloc@std@@@8??0bad_alloc@std@@QEAA@AEBV01@@Z24 00000001800163a0     LIBCMT:throw_bad_alloc.obj
 0001:000153c8       _CT??_R0?AVexception@std@@@8??0exception@std@@QEAA@AEBV01@@Z24 00000001800163c8     LIBCMT:throw_bad_alloc.obj
 0001:000153f0       _TI3?AVbad_array_new_length@std@@ 00000001800163f0     LIBCMT:throw_bad_alloc.obj
 0001:00015410       _CTA3?AVbad_array_new_length@std@@ 0000000180016410     LIBCMT:throw_bad_alloc.obj
 0001:00015430       _CT??_R0?AVbad_array_new_length@std@@@8??0bad_array_new_length@std@@QEAA@AEBV01@@Z24 0000000180016430     LIBCMT:throw_bad_alloc.obj
 0002:00000000       ?OptName@@3UOptionsName@@A 0000000180017000     SameFolder.obj
 0002:00000018       __scrt_native_dllmain_reason 0000000180017018     LIBCMT:utility.obj
 0002:00000020       __security_cookie_complement 0000000180017020     LIBCMT:gs_cookie.obj
 0002:00000028       __security_cookie          0000000180017028     LIBCMT:gs_cookie.obj
 0002:00000030       __isa_available            0000000180017030     LIBCMT:cpu_disp.obj
 0002:00000034       __isa_enabled              0000000180017034     LIBCMT:cpu_disp.obj
 0002:00000038       __memcpy_nt_iters          0000000180017038     LIBCMT:cpu_disp.obj
 0002:00000050       __abort_behavior           0000000180017050     libucrt:abort.obj
 0002:00000370       __acrt_initial_multibyte_data 0000000180017370     libucrt:mbctype.obj
 0002:000005a0       __acrt_initial_locale_data 00000001800175a0     libucrt:nlsdata.obj
 0002:000006f8       __acrt_initial_locale_pointers 00000001800176f8     libucrt:nlsdata.obj
 0002:00000708       __acrt_wide_c_locale_string 0000000180017708     libucrt:nlsdata.obj
 0002:00000710       _iob                       0000000180017710     libucrt:_file.obj
 0002:00000818       __globallocalestatus       0000000180017818     libucrt:glstatus.obj
 0002:00000820       __acrt_lconv_c             0000000180017820     libucrt:localeconv.obj
 0002:000008b8       __acrt_lconv_static_decimal 00000001800178b8     libucrt:localeconv.obj
 0002:000008bc       __acrt_lconv_static_W_decimal 00000001800178bc     libucrt:localeconv.obj
 0002:000008c0       _lookuptrailbytes          00000001800178c0     libucrt:read.obj
 0002:000009e0       _fltused                   00000001800179e0     LIBCMT:fltused.obj
 0002:000009f0       ??_R0?AVbad_alloc@std@@@8  00000001800179f0     LIBCMT:throw_bad_alloc.obj
 0002:00000a18       ??_R0?AVexception@std@@@8  0000000180017a18     LIBCMT:throw_bad_alloc.obj
 0002:00000a40       ??_R0?AVbad_array_new_length@std@@@8 0000000180017a40     LIBCMT:throw_bad_alloc.obj
 0002:00000a70       ??_R0?AVtype_info@@@8      0000000180017a70     LIBCMT:std_type_info_static.obj
 0002:00000a90       ?Opt@@3UOptions@@A         0000000180017a90     SameFolder.obj
 0002:00000aa0       ?Info@@3UPluginStartupInfo@@A 0000000180017aa0     SameFolder.obj
 0002:00000bb0       ?FSF@@3UFarStandardFunctions@@A 0000000180017bb0     SameFolder.obj
 0002:00000d60       ?__type_info_root_node@@3U__type_info_node@@A 0000000180017d60     LIBCMT:tncleanup.obj
 0002:00000d70       ?_OptionsStorage@?1??__local_stdio_printf_options@@9@4_KA 0000000180017d70     LIBCMT:default_local_stdio_options.obj
 0002:00000d78       ?_OptionsStorage@?1??__local_stdio_scanf_options@@9@4_KA 0000000180017d78     LIBCMT:default_local_stdio_options.obj
 0002:00000d80       __scrt_current_native_startup_state 0000000180017d80     LIBCMT:utility.obj
 0002:00000d88       __scrt_native_startup_lock 0000000180017d88     LIBCMT:utility.obj
 0002:00000dc8       __scrt_debugger_hook_flag  0000000180017dc8     LIBCMT:utility_desktop.obj
 0002:00000dcc       __favor                    0000000180017dcc     LIBCMT:cpu_disp.obj
 0002:00000dd0       ?__WinRTOutOfMemoryExceptionCallback@@3P6APEAXXZEA 0000000180017dd0     libvcruntime:ehhelpers.obj
 0002:00000dd8       ?pArgList@UnDecorator@@0PEAVReplicator@@EA 0000000180017dd8     libvcruntime:undname.obj
 0002:00000de0       ?pZNameList@UnDecorator@@0PEAVReplicator@@EA 0000000180017de0     libvcruntime:undname.obj
 0002:00000de8       ?pTemplateArgList@UnDecorator@@0PEAVReplicator@@EA 0000000180017de8     libvcruntime:undname.obj
 0002:00000df0       ?gName@UnDecorator@@0PEBDEB 0000000180017df0     libvcruntime:undname.obj
 0002:00000df8       ?name@UnDecorator@@0PEBDEB 0000000180017df8     libvcruntime:undname.obj
 0002:00000e00       ?disableFlags@UnDecorator@@0KA 0000000180017e00     libvcruntime:undname.obj
 0002:00000e04       ?fExplicitTemplateParams@UnDecorator@@0_NA 0000000180017e04     libvcruntime:undname.obj
 0002:00000e05       ?fGetTemplateArgumentList@UnDecorator@@0_NA 0000000180017e05     libvcruntime:undname.obj
 0002:00000e08       ?m_pGetParameter@UnDecorator@@0P6APEADJ@ZEA 0000000180017e08     libvcruntime:undname.obj
 0002:00000e10       ?m_CHPENameOffset@UnDecorator@@0KA 0000000180017e10     libvcruntime:undname.obj
 0002:00000e14       ?m_recursionLevel@UnDecorator@@0KA 0000000180017e14     libvcruntime:undname.obj
 0002:00000f40       __pPurecall                0000000180017f40     libvcruntime:purevirt_data.obj
 0002:00000f60       ?c_exit_complete@?1???R<lambda_6e4b09c48022b2350581041d5f6b0c4c>@@QEBA@XZ@4_NA 0000000180017f60     libucrt:exit.obj
 0002:00001078       _environ_table             0000000180018078     libucrt:environment_initialization.obj
 0002:00001080       _wenviron_table            0000000180018080     libucrt:environment_initialization.obj
 0002:00001088       __dcrt_initial_wide_environment 0000000180018088     libucrt:environment_initialization.obj
 0002:00001090       __dcrt_initial_narrow_environment 0000000180018090     libucrt:environment_initialization.obj
 0002:00001098       __acrt_atexit_table        0000000180018098     libucrt:onexit.obj
 0002:000010b0       __acrt_at_quick_exit_table 00000001800180b0     libucrt:onexit.obj
 0002:00001310       _mbctype                   0000000180018310     libucrt:mbctype.obj
 0002:00001318       _mbcasemap                 0000000180018318     libucrt:mbctype.obj
 0002:00001320       __acrt_current_multibyte_data 0000000180018320     libucrt:mbctype.obj
 0002:00001330       _pgmptr                    0000000180018330     libucrt:argv_data.obj
 0002:00001338       __argc                     0000000180018338     libucrt:argv_data.obj
 0002:00001340       __argv                     0000000180018340     libucrt:argv_data.obj
 0002:00001348       __wargv                    0000000180018348     libucrt:argv_data.obj
 0002:00001350       _acmdln                    0000000180018350     libucrt:argv_data.obj
 0002:00001358       _wcmdln                    0000000180018358     libucrt:argv_data.obj
 0002:00001510       __acrt_heap                0000000180018510     libucrt:heap_handle.obj
 0002:00001520       __pioinfo                  0000000180018520     libucrt:ioinit.obj
 0002:00001920       _nhandle                   0000000180018920     libucrt:ioinit.obj
 0002:00001950       __acrt_current_locale_data 0000000180018950     libucrt:nlsdata.obj
 0002:00001958       _nstream                   0000000180018958     libucrt:_file.obj
 0002:00001960       __piob                     0000000180018960     libucrt:_file.obj
 0002:00001968       __acrt_stdout_buffer       0000000180018968     libucrt:_sftbuf.obj
 0002:00001970       __acrt_stderr_buffer       0000000180018970     libucrt:_sftbuf.obj
 0002:00001980       __acrt_locale_changed_data 0000000180018980     libucrt:wsetlocale.obj
 0002:00001988       __acrt_lconv_static_null   0000000180018988     libucrt:localeconv.obj
 0002:0000198c       __acrt_lconv_static_W_null 000000018001898c     libucrt:localeconv.obj
 0002:000019a0       __fma3_is_available        00000001800189a0     libucrt:fma3_available.obj
 0002:000019a4       __use_fma3_lib             00000001800189a4     libucrt:fma3_available.obj
 0002:00001f20       __scrt_ucrt_dll_is_in_use  0000000180018f20     <common>
 0002:00001f28       __dyn_tls_init_callback    0000000180018f28     <common>
 0004:00000000       __imp_lstrcmpW             000000018001a000     kernel32:KERNEL32.dll
 0004:00000008       __imp_lstrlenW             000000018001a008     kernel32:KERNEL32.dll
 0004:00000010       __imp_WriteConsoleW        000000018001a010     kernel32:KERNEL32.dll
 0004:00000018       __imp_QueryPerformanceCounter 000000018001a018     kernel32:KERNEL32.dll
 0004:00000020       __imp_GetCurrentProcessId  000000018001a020     kernel32:KERNEL32.dll
 0004:00000028       __imp_GetCurrentThreadId   000000018001a028     kernel32:KERNEL32.dll
 0004:00000030       __imp_GetSystemTimeAsFileTime 000000018001a030     kernel32:KERNEL32.dll
 0004:00000038       __imp_InitializeSListHead  000000018001a038     kernel32:KERNEL32.dll
 0004:00000040       __imp_RtlCaptureContext    000000018001a040     kernel32:KERNEL32.dll
 0004:00000048       __imp_RtlLookupFunctionEntry 000000018001a048     kernel32:KERNEL32.dll
 0004:00000050       __imp_RtlVirtualUnwind     000000018001a050     kernel32:KERNEL32.dll
 0004:00000058       __imp_IsDebuggerPresent    000000018001a058     kernel32:KERNEL32.dll
 0004:00000060       __imp_UnhandledExceptionFilter 000000018001a060     kernel32:KERNEL32.dll
 0004:00000068       __imp_SetUnhandledExceptionFilter 000000018001a068     kernel32:KERNEL32.dll
 0004:00000070       __imp_GetStartupInfoW      000000018001a070     kernel32:KERNEL32.dll
 0004:00000078       __imp_IsProcessorFeaturePresent 000000018001a078     kernel32:KERNEL32.dll
 0004:00000080       __imp_GetModuleHandleW     000000018001a080     kernel32:KERNEL32.dll
 0004:00000088       __imp_RtlUnwindEx          000000018001a088     kernel32:KERNEL32.dll
 0004:00000090       __imp_RtlPcToFileHeader    000000018001a090     kernel32:KERNEL32.dll
 0004:00000098       __imp_RaiseException       000000018001a098     kernel32:KERNEL32.dll
 0004:000000a0       __imp_InterlockedFlushSList 000000018001a0a0     kernel32:KERNEL32.dll
 0004:000000a8       __imp_GetLastError         000000018001a0a8     kernel32:KERNEL32.dll
 0004:000000b0       __imp_SetLastError         000000018001a0b0     kernel32:KERNEL32.dll
 0004:000000b8       __imp_EnterCriticalSection 000000018001a0b8     kernel32:KERNEL32.dll
 0004:000000c0       __imp_LeaveCriticalSection 000000018001a0c0     kernel32:KERNEL32.dll
 0004:000000c8       __imp_DeleteCriticalSection 000000018001a0c8     kernel32:KERNEL32.dll
 0004:000000d0       __imp_InitializeCriticalSectionAndSpinCount 000000018001a0d0     kernel32:KERNEL32.dll
 0004:000000d8       __imp_TlsAlloc             000000018001a0d8     kernel32:KERNEL32.dll
 0004:000000e0       __imp_TlsGetValue          000000018001a0e0     kernel32:KERNEL32.dll
 0004:000000e8       __imp_TlsSetValue          000000018001a0e8     kernel32:KERNEL32.dll
 0004:000000f0       __imp_TlsFree              000000018001a0f0     kernel32:KERNEL32.dll
 0004:000000f8       __imp_FreeLibrary          000000018001a0f8     kernel32:KERNEL32.dll
 0004:00000100       __imp_GetProcAddress       000000018001a100     kernel32:KERNEL32.dll
 0004:00000108       __imp_LoadLibraryExW       000000018001a108     kernel32:KERNEL32.dll
 0004:00000110       __imp_GetCurrentProcess    000000018001a110     kernel32:KERNEL32.dll
 0004:00000118       __imp_ExitProcess          000000018001a118     kernel32:KERNEL32.dll
 0004:00000120       __imp_TerminateProcess     000000018001a120     kernel32:KERNEL32.dll
 0004:00000128       __imp_GetModuleHandleExW   000000018001a128     kernel32:KERNEL32.dll
 0004:00000130       __imp_GetModuleFileNameW   000000018001a130     kernel32:KERNEL32.dll
 0004:00000138       __imp_HeapFree             000000018001a138     kernel32:KERNEL32.dll
 0004:00000140       __imp_HeapAlloc            000000018001a140     kernel32:KERNEL32.dll
 0004:00000148       __imp_FindClose            000000018001a148     kernel32:KERNEL32.dll
 0004:00000150       __imp_FindFirstFileExW     000000018001a150     kernel32:KERNEL32.dll
 0004:00000158       __imp_FindNextFileW        000000018001a158     kernel32:KERNEL32.dll
 0004:00000160       __imp_IsValidCodePage      000000018001a160     kernel32:KERNEL32.dll
 0004:00000168       __imp_GetACP               000000018001a168     kernel32:KERNEL32.dll
 0004:00000170       __imp_GetOEMCP             000000018001a170     kernel32:KERNEL32.dll
 0004:00000178       __imp_GetCPInfo            000000018001a178     kernel32:KERNEL32.dll
 0004:00000180       __imp_GetCommandLineA      000000018001a180     kernel32:KERNEL32.dll
 0004:00000188       __imp_GetCommandLineW      000000018001a188     kernel32:KERNEL32.dll
 0004:00000190       __imp_MultiByteToWideChar  000000018001a190     kernel32:KERNEL32.dll
 0004:00000198       __imp_WideCharToMultiByte  000000018001a198     kernel32:KERNEL32.dll
 0004:000001a0       __imp_GetEnvironmentStringsW 000000018001a1a0     kernel32:KERNEL32.dll
 0004:000001a8       __imp_FreeEnvironmentStringsW 000000018001a1a8     kernel32:KERNEL32.dll
 0004:000001b0       __imp_LCMapStringW         000000018001a1b0     kernel32:KERNEL32.dll
 0004:000001b8       __imp_GetProcessHeap       000000018001a1b8     kernel32:KERNEL32.dll
 0004:000001c0       __imp_GetStdHandle         000000018001a1c0     kernel32:KERNEL32.dll
 0004:000001c8       __imp_GetFileType          000000018001a1c8     kernel32:KERNEL32.dll
 0004:000001d0       __imp_GetStringTypeW       000000018001a1d0     kernel32:KERNEL32.dll
 0004:000001d8       __imp_HeapSize             000000018001a1d8     kernel32:KERNEL32.dll
 0004:000001e0       __imp_HeapReAlloc          000000018001a1e0     kernel32:KERNEL32.dll
 0004:000001e8       __imp_SetStdHandle         000000018001a1e8     kernel32:KERNEL32.dll
 0004:000001f0       __imp_FlushFileBuffers     000000018001a1f0     kernel32:KERNEL32.dll
 0004:000001f8       __imp_WriteFile            000000018001a1f8     kernel32:KERNEL32.dll
 0004:00000200       __imp_GetConsoleCP         000000018001a200     kernel32:KERNEL32.dll
 0004:00000208       __imp_GetConsoleMode       000000018001a208     kernel32:KERNEL32.dll
 0004:00000210       __imp_SetFilePointerEx     000000018001a210     kernel32:KERNEL32.dll
 0004:00000218       __imp_CreateFileW          000000018001a218     kernel32:KERNEL32.dll
 0004:00000220       __imp_CloseHandle          000000018001a220     kernel32:KERNEL32.dll
 0004:00000228       \177KERNEL32_NULL_THUNK_DATA 000000018001a228     kernel32:KERNEL32.dll
 0004:00000230       __guard_check_icall_fptr   000000018001a230     LIBCMT:guard_support.obj
 0004:00000238       __guard_dispatch_icall_fptr 000000018001a238     LIBCMT:guard_support.obj
 0004:00000240       __IMPORT_DESCRIPTOR_KERNEL32 000000018001a240     kernel32:KERNEL32.dll
 0004:00000254       __NULL_IMPORT_DESCRIPTOR   000000018001a254     kernel32:KERNEL32.dll

 entry point at        0001:00009924

 Static symbols

 0001:00000340       ?ExceptionTemplate@?1??_CxxThrowException@@9@4UEHExceptionRecord@@B 0000000180001340     libvcruntime:throw.obj
 0001:00000390       ?tokenTable@@3QBQEBDB      0000000180001390     libvcruntime:undname.obj
 0001:00000410       ?nameTable@@3QBQEBDB       0000000180001410     libvcruntime:undname.obj
 0001:000006a0       ?rttiTable@@3QBQEBDB       00000001800016a0     libvcruntime:undname.obj
 0001:00000d58       ?module_names@?A0x14c33c87@@3QBQEB_WB 0000000180001d58     libvcruntime:winapi_downlevel.obj
 0001:00000e28       ?candidate_modules@?1??try_get_FlsAlloc@@YAP6AKP6AXPEAX@Z@ZXZ@4QBW4module_id@?A0x14c33c87@@B 0000000180001e28     libvcruntime:winapi_downlevel.obj
 0001:00000e40       ?candidate_modules@?1??try_get_FlsFree@@YAP6AHK@ZXZ@4QBW4module_id@?A0x14c33c87@@B 0000000180001e40     libvcruntime:winapi_downlevel.obj
 0001:00000e50       ?candidate_modules@?1??try_get_FlsGetValue@@YAP6APEAXK@ZXZ@4QBW4module_id@?A0x14c33c87@@B 0000000180001e50     libvcruntime:winapi_downlevel.obj
 0001:00000e68       ?candidate_modules@?1??try_get_FlsSetValue@@YAP6AHKPEAX@ZXZ@4QBW4module_id@?A0x14c33c87@@B 0000000180001e68     libvcruntime:winapi_downlevel.obj
 0001:00000e80       ?candidate_modules@?1??try_get_InitializeCriticalSectionEx@@YAP6AHPEAU_RTL_CRITICAL_SECTION@@KK@ZXZ@4QBW4module_id@?A0x14c33c87@@B 0000000180001e80     libvcruntime:winapi_downlevel.obj
 0001:00000fb0       __acrt_initializers        0000000180001fb0     libucrt:initialization.obj
 0001:000010b0       ?errtable@@3QBUerrentry@?A0x31fdb9ec@@B 00000001800020b0     libucrt:errno.obj
 0001:00001218       ?_mb_locale_names@@3QBQEB_WB 0000000180002218     libucrt:mbctype.obj
 0001:00001280       ?module_names@?A0x391cf84c@@3QBQEB_WB 0000000180002280     libucrt:winapi_thunks.obj
 0001:00001828       ?candidate_modules@?1??try_get_AreFileApisANSI@@YAP6AHXZXZ@4QBW4module_id@?A0x391cf84c@@B 0000000180002828     libucrt:winapi_thunks.obj
 0001:00001840       ?candidate_modules@?1??try_get_FlsAlloc@@YAP6AKP6AXPEAX@Z@ZXZ@4QBW4module_id@?A0x391cf84c@@B 0000000180002840     libucrt:winapi_thunks.obj
 0001:00001858       ?candidate_modules@?1??try_get_FlsFree@@YAP6AHK@ZXZ@4QBW4module_id@?A0x391cf84c@@B 0000000180002858     libucrt:winapi_thunks.obj
 0001:00001868       ?candidate_modules@?1??try_get_FlsGetValue@@YAP6APEAXK@ZXZ@4QBW4module_id@?A0x391cf84c@@B 0000000180002868     libucrt:winapi_thunks.obj
 0001:00001880       ?candidate_modules@?1??try_get_FlsSetValue@@YAP6AHKPEAX@ZXZ@4QBW4module_id@?A0x391cf84c@@B 0000000180002880     libucrt:winapi_thunks.obj
 0001:00001898       ?candidate_modules@?1??try_get_InitializeCriticalSectionEx@@YAP6AHPEAU_RTL_CRITICAL_SECTION@@KK@ZXZ@4QBW4module_id@?A0x391cf84c@@B 0000000180002898     libucrt:winapi_thunks.obj
 0001:000018c0       ?candidate_modules@?1??try_get_LCMapStringEx@@YAP6AHPEB_WK0HPEA_WHPEAU_nlsversioninfo@@PEAX_J@ZXZ@4QBW4module_id@?A0x391cf84c@@B 00000001800028c0     libucrt:winapi_thunks.obj
 0001:000018d8       ?candidate_modules@?1??try_get_LocaleNameToLCID@@YAP6AKPEB_WK@ZXZ@4QBW4module_id@?A0x391cf84c@@B 00000001800028d8     libucrt:winapi_thunks.obj
 0001:000018f4       ?candidate_modules@?1??try_get_AppPolicyGetProcessTerminationMethod@@YAP6AJPEAXPEAW4AppPolicyProcessTerminationMethod@@@ZXZ@4QBW4module_id@?A0x391cf84c@@B 00000001800028f4     libucrt:winapi_thunks.obj
 0001:000025a0       ?LcidToLocaleNameTable@?A0x881e4c05@@3QBULcidToLocaleName@1@B 00000001800035a0     libucrt:lcidtoname_downlevel.obj
 0001:00004000       ?LocaleNameToIndexTable@?A0x881e4c05@@3QBULocaleNameIndex@1@B 0000000180005000     libucrt:lcidtoname_downlevel.obj
 0001:000058a0       __real_ninf                00000001800068a0     libucrt:log10.obj
 0001:000058b0       __real_inf                 00000001800068b0     libucrt:log10.obj
 0001:000058c0       __real_neg_qnan            00000001800068c0     libucrt:log10.obj
 0001:000058d0       __real_qnanbit             00000001800068d0     libucrt:log10.obj
 0001:000058e0       __int_1023                 00000001800068e0     libucrt:log10.obj
 0001:000058f0       __mask_001                 00000001800068f0     libucrt:log10.obj
 0001:00005900       __mask_mant                0000000180006900     libucrt:log10.obj
 0001:00005910       __mask_mant_top8           0000000180006910     libucrt:log10.obj
 0001:00005920       __mask_mant9               0000000180006920     libucrt:log10.obj
 0001:00005930       __real_log10_e             0000000180006930     libucrt:log10.obj
 0001:00005940       __real_log10_e_lead        0000000180006940     libucrt:log10.obj
 0001:00005950       __real_log10_e_tail        0000000180006950     libucrt:log10.obj
 0001:00005960       __real_log10_2_lead        0000000180006960     libucrt:log10.obj
 0001:00005970       __real_log10_2_tail        0000000180006970     libucrt:log10.obj
 0001:00005980       __real_two                 0000000180006980     libucrt:log10.obj
 0001:00005990       __real_one                 0000000180006990     libucrt:log10.obj
 0001:000059a0       __real_half                00000001800069a0     libucrt:log10.obj
 0001:000059b0       __mask_100                 00000001800069b0     libucrt:log10.obj
 0001:000059c0       __real_1_over_512          00000001800069c0     libucrt:log10.obj
 0001:000059d0       __real_1_over_2            00000001800069d0     libucrt:log10.obj
 0001:000059e0       __real_1_over_3            00000001800069e0     libucrt:log10.obj
 0001:000059f0       __real_1_over_4            00000001800069f0     libucrt:log10.obj
 0001:00005a00       __real_1_over_5            0000000180006a00     libucrt:log10.obj
 0001:00005a10       __real_1_over_6            0000000180006a10     libucrt:log10.obj
 0001:00005a20       __real_neg_1023            0000000180006a20     libucrt:log10.obj
 0001:00005a30       __mask_2045                0000000180006a30     libucrt:log10.obj
 0001:00005a40       __real_threshold           0000000180006a40     libucrt:log10.obj
 0001:00005a50       __real_near_one_lt         0000000180006a50     libucrt:log10.obj
 0001:00005a60       __real_near_one_gt         0000000180006a60     libucrt:log10.obj
 0001:00005a70       __real_min_norm            0000000180006a70     libucrt:log10.obj
 0001:00005a80       __real_notsign             0000000180006a80     libucrt:log10.obj
 0001:00005a90       __real_ca1                 0000000180006a90     libucrt:log10.obj
 0001:00005aa0       __real_ca2                 0000000180006aa0     libucrt:log10.obj
 0001:00005ab0       __real_ca3                 0000000180006ab0     libucrt:log10.obj
 0001:00005ac0       __real_ca4                 0000000180006ac0     libucrt:log10.obj
 0001:00005ad0       __mask_lower               0000000180006ad0     libucrt:log10.obj
 0001:00005ae0       __flag_x_zero              0000000180006ae0     libucrt:log10.obj
 0001:00005ae4       __flag_x_neg               0000000180006ae4     libucrt:log10.obj
 0001:00005ae8       __flag_x_nan               0000000180006ae8     libucrt:log10.obj
 0001:00007340       __real@433fffffffffffff    0000000180008340     libucrt:fpsr.obj
 0001:00007348       __real@c33fffffffffffff    0000000180008348     libucrt:fpsr.obj
 0001:00007350       GS_ExceptionPointers       0000000180008350     LIBCMT:gs_report.obj
 0001:00007950       $$000000                   0000000180008950     chkstk.obj
 0001:00007e6c       $LN39                      0000000180008e6c     SameFolder.obj
 0001:00008834       $LN36                      0000000180009834     SameFolder.obj
 0001:00008e4c       $LN138                     0000000180009e4c     SameFolder.obj
 0001:00008e7c       $LN137                     0000000180009e7c     SameFolder.obj
 0001:000095f4       ?dllmain_crt_dispatch@@YAHQEAUHINSTANCE__@@KQEAX@Z 000000018000a5f4 f   LIBCMT:dll_dllmain.obj
 0001:00009644       ?dllmain_crt_process_attach@@YAHQEAUHINSTANCE__@@QEAX@Z 000000018000a644 f   LIBCMT:dll_dllmain.obj
 0001:00009760       ?dllmain_crt_process_detach@@YAH_N@Z 000000018000a760 f   LIBCMT:dll_dllmain.obj
 0001:000097f0       ?dllmain_dispatch@@YAHQEAUHINSTANCE__@@KQEAX@Z 000000018000a7f0 f   LIBCMT:dll_dllmain.obj
 0001:0000a310       $$000000                   000000018000b310     libvcruntime:memset.obj
 0001:0000a40c       MsetTab                    000000018000b40c     libvcruntime:memset.obj
 0001:0000a910       $$000000                   000000018000b910     libvcruntime:notify.obj
 0001:0000ac38       ?try_get_function@@YAPEAXW4function_id@?A0x14c33c87@@QEBDQEBW4module_id@2@2@Z 000000018000bc38 f   libvcruntime:winapi_downlevel.obj
 0001:0000b020       $$000000                   000000018000c020     libvcruntime:memcpy.obj
 0001:0000b0d7       MoveSmall                  000000018000c0d7     libvcruntime:memcpy.obj
 0001:0000b480       $$000000                   000000018000c480     libvcruntime:handlers.obj
 0001:0000b7ec       ??$?RV<lambda_d80eeec6fff315bfe5c115232f3240e3>@@AEAV<lambda_6e4b09c48022b2350581041d5f6b0c4c>@@V<lambda_2358e3775559c9db80273638284d5e45>@@@?$__crt_seh_guarded_call@X@@QEAAX$$QEAV<lambda_d80eeec6fff315bfe5c115232f3240e3>@@AEAV<lambda_6e4b09c48022b2350581041d5f6b0c4c>@@$$QEAV<lambda_2358e3775559c9db80273638284d5e45>@@@Z 000000018000c7ec f   libucrt:exit.obj
 0001:0000b824       ??R<lambda_6e4b09c48022b2350581041d5f6b0c4c>@@QEBA@XZ 000000018000c824 f   libucrt:exit.obj
 0001:0000b8e8       ?atexit_exception_filter@@YAHK@Z 000000018000c8e8 f   libucrt:exit.obj
 0001:0000b8f4       ?common_exit@@YAXHW4_crt_exit_cleanup_mode@@W4_crt_exit_return_mode@@@Z 000000018000c8f4 f   libucrt:exit.obj
 0001:0000b9b0       ?exit_or_terminate_process@@YAXI@Z 000000018000c9b0 f   libucrt:exit.obj
 0001:0000b9fc       ?try_cor_exit_process@@YAXI@Z 000000018000c9fc f   libucrt:exit.obj
 0001:0000ba84       ??$parse_command_line@D@@YAXPEADPEAPEAD0PEA_K2@Z 000000018000ca84 f   libucrt:argv_parsing.obj
 0001:0000be30       ??$common_initialize_environment_nolock@D@@YAHXZ 000000018000ce30 f   libucrt:environment_initialization.obj
 0001:0000be9c       ??$create_environment@D@@YAQEAPEADQEAD@Z 000000018000ce9c f   libucrt:environment_initialization.obj
 0001:0000bfa4       ??$free_environment@_W@@YAXQEAPEA_W@Z 000000018000cfa4 f   libucrt:environment_initialization.obj
 0001:0000bfa4       ??$free_environment@D@@YAXQEAPEAD@Z 000000018000cfa4 f   libucrt:environment_initialization.obj
 0001:0000bfe8       ??$uninitialize_environment_internal@D@@YAXAEAPEAPEAD@Z 000000018000cfe8 f   libucrt:environment_initialization.obj
 0001:0000c004       ??$uninitialize_environment_internal@_W@@YAXAEAPEAPEA_W@Z 000000018000d004 f   libucrt:environment_initialization.obj
 0001:0000c060       ??$?RV<lambda_7777bce6b2f8c936911f934f8298dc43>@@AEAV<lambda_f03950bc5685219e0bcd2087efbe011e>@@V<lambda_3883c3dff614d5e0c5f61bb1ac94921c>@@@?$__crt_seh_guarded_call@H@@QEAAH$$QEAV<lambda_7777bce6b2f8c936911f934f8298dc43>@@AEAV<lambda_f03950bc5685219e0bcd2087efbe011e>@@$$QEAV<lambda_3883c3dff614d5e0c5f61bb1ac94921c>@@@Z 000000018000d060 f   libucrt:onexit.obj
 0001:0000c09c       ??R<lambda_f03950bc5685219e0bcd2087efbe011e>@@QEBAHXZ 000000018000d09c f   libucrt:onexit.obj
 0001:0000c218       initialize_global_variables 000000018000d218 f   libucrt:initialization.obj
 0001:0000c22c       initialize_c               000000018000d22c f   libucrt:initialization.obj
 0001:0000c250       initialize_environment     000000018000d250 f   libucrt:initialization.obj
 0001:0000c250       initialize_global_state_isolation 000000018000d250 f   libucrt:initialization.obj
 0001:0000c250       report_memory_leaks        000000018000d250 f   libucrt:initialization.obj
 0001:0000c250       uninitialize_c             000000018000d250 f   libucrt:initialization.obj
 0001:0000c250       uninitialize_global_state_isolation 000000018000d250 f   libucrt:initialization.obj
 0001:0000c254       uninitialize_environment   000000018000d254 f   libucrt:initialization.obj
 0001:0000c264       initialize_pointers        000000018000d264 f   libucrt:initialization.obj
 0001:0000c2a4       uninitialize_vcruntime     000000018000d2a4 f   libucrt:initialization.obj
 0001:0000c2ac       uninitialize_allocated_memory 000000018000d2ac f   libucrt:initialization.obj
 0001:0000c2ec       uninitialize_allocated_io_buffers 000000018000d2ec f   libucrt:initialization.obj
 0001:0000c4f0       $$000000                   000000018000d4f0     libucrt:strncmp.obj
 0001:0000c764       ??$?RV<lambda_0ae27a3a962d80f24befdcbee591983d>@@AEAV<lambda_8d0ee55de4b1038c4002e0adecdf1839>@@V<lambda_dc504788e8f1664fe9b84e20bfb512f2>@@@?$__crt_seh_guarded_call@X@@QEAAX$$QEAV<lambda_0ae27a3a962d80f24befdcbee591983d>@@AEAV<lambda_8d0ee55de4b1038c4002e0adecdf1839>@@$$QEAV<lambda_dc504788e8f1664fe9b84e20bfb512f2>@@@Z 000000018000d764 f   libucrt:per_thread_data.obj
 0001:0000c7a4       ??$?RV<lambda_2d41944a1d46af3157314b8a01080d33>@@AEAV<lambda_8f455de75cd7d7f24b4096f044d8b9e6>@@V<lambda_aa500f224e6afead328df44964fe2772>@@@?$__crt_seh_guarded_call@X@@QEAAX$$QEAV<lambda_2d41944a1d46af3157314b8a01080d33>@@AEAV<lambda_8f455de75cd7d7f24b4096f044d8b9e6>@@$$QEAV<lambda_aa500f224e6afead328df44964fe2772>@@@Z 000000018000d7a4 f   libucrt:per_thread_data.obj
 0001:0000c7e4       ??$?RV<lambda_aa87e3671a710a21b5dc78c0bdf72e11>@@AEAV<lambda_92619d2358a28f41a33ba319515a20b9>@@V<lambda_6992ecaafeb10aed2b74cb1fae11a551>@@@?$__crt_seh_guarded_call@X@@QEAAX$$QEAV<lambda_aa87e3671a710a21b5dc78c0bdf72e11>@@AEAV<lambda_92619d2358a28f41a33ba319515a20b9>@@$$QEAV<lambda_6992ecaafeb10aed2b74cb1fae11a551>@@@Z 000000018000d7e4 f   libucrt:per_thread_data.obj
 0001:0000c82c       ??$?RV<lambda_f2e299630e499de9f9a165e60fcd3db5>@@AEAV<lambda_2ae9d31cdba2644fcbeaf08da7c24588>@@V<lambda_40d01ff24d0e7b3814fdbdcee8eab3c7>@@@?$__crt_seh_guarded_call@X@@QEAAX$$QEAV<lambda_f2e299630e499de9f9a165e60fcd3db5>@@AEAV<lambda_2ae9d31cdba2644fcbeaf08da7c24588>@@$$QEAV<lambda_40d01ff24d0e7b3814fdbdcee8eab3c7>@@@Z 000000018000d82c f   libucrt:per_thread_data.obj
 0001:0000c88c       ?construct_ptd_array@@YAXQEAU__acrt_ptd@@@Z 000000018000d88c f   libucrt:per_thread_data.obj
 0001:0000c95c       ?destroy_fls@@YAXPEAX@Z    000000018000d95c f   libucrt:per_thread_data.obj
 0001:0000c97c       ?destroy_ptd_array@@YAXQEAU__acrt_ptd@@@Z 000000018000d97c f   libucrt:per_thread_data.obj
 0001:0000ca74       ?replace_current_thread_locale_nolock@@YAXQEAU__acrt_ptd@@QEAU__crt_locale_data@@@Z 000000018000da74 f   libucrt:per_thread_data.obj
 0001:0000d1d0       ?<lambda_invoker_cdecl>@<lambda_c2303d2482d7c3675ea2e24c4cfb6115>@@CAHPEBX0@Z 000000018000e1d0 f   libucrt:argv_wildcards.obj
 0001:0000d4e8       ??$common_expand_argv_wildcards@D@@YAHQEAPEADQEAPEAPEAD@Z 000000018000e4e8 f   libucrt:argv_wildcards.obj
 0001:0000d6f4       ??$copy_and_add_argument_to_buffer@D@@YAHQEBD0_KAEAV?$argument_list@D@?A0x5f5c8891@@@Z 000000018000e6f4 f   libucrt:argv_wildcards.obj
 0001:0000d87c       ??$expand_argument_wildcards@D@@YAHQEAD0AEAV?$argument_list@D@?A0x5f5c8891@@@Z 000000018000e87c f   libucrt:argv_wildcards.obj
 0001:0000ddc8       ??$?RV<lambda_efdfa57d1f175319df784efa44bb7b81>@@AEAV<lambda_5f0a4c1567f8adc6734073e5d1e1b35c>@@V<lambda_2e8a7d3640ea6ccb4c2413664c2db6fd>@@@?$__crt_seh_guarded_call@X@@QEAAX$$QEAV<lambda_efdfa57d1f175319df784efa44bb7b81>@@AEAV<lambda_5f0a4c1567f8adc6734073e5d1e1b35c>@@$$QEAV<lambda_2e8a7d3640ea6ccb4c2413664c2db6fd>@@@Z 000000018000edc8 f   libucrt:mbctype.obj
 0001:0000df84       ?getSystemCP@@YAHH@Z       000000018000ef84 f   libucrt:mbctype.obj
 0001:0000e004       ?setSBCS@@YAXPEAU__crt_multibyte_data@@@Z 000000018000f004 f   libucrt:mbctype.obj
 0001:0000e094       ?setSBUpLow@@YAXPEAU__crt_multibyte_data@@@Z 000000018000f094 f   libucrt:mbctype.obj
 0001:0000e278       ?setmbcp_internal@@YAHH_NQEAU__acrt_ptd@@QEAPEAU__crt_multibyte_data@@@Z 000000018000f278 f   libucrt:mbctype.obj
 0001:0000e43c       ?update_thread_multibyte_data_internal@@YAPEAU__crt_multibyte_data@@QEAU__acrt_ptd@@QEAPEAU1@@Z 000000018000f43c f   libucrt:mbctype.obj
 0001:0000e82c       ?x_ismbbtype_l@@YAHPEAU__crt_locale_pointers@@IHH@Z 000000018000f82c f   libucrt:ismbbyte.obj
 0001:0000eb70       ?try_get_function@@YAPEAXW4function_id@?A0x391cf84c@@QEBDQEBW4module_id@2@2@Z 000000018000fb70 f   libucrt:winapi_thunks.obj
 0001:0000f130       ?initialize_inherited_file_handles_nolock@@YAXXZ 0000000180010130 f   libucrt:ioinit.obj
 0001:0000f220       ?initialize_stdio_handles_nolock@@YAXXZ 0000000180010220 f   libucrt:ioinit.obj
 0001:0000f464       ??$?RV<lambda_450d765d439847d4c735a33c368b5fc0>@@AEAV<lambda_44731a7d0e6d81c3e6aa82d741081786>@@V<lambda_601a2a7da3b7a96e9554ac7215c4b07c>@@@?$__crt_seh_guarded_call@P6AXH@Z@@QEAAP6AXH@Z$$QEAV<lambda_450d765d439847d4c735a33c368b5fc0>@@AEAV<lambda_44731a7d0e6d81c3e6aa82d741081786>@@$$QEAV<lambda_601a2a7da3b7a96e9554ac7215c4b07c>@@@Z 0000000180010464 f   libucrt:signal.obj
 0001:0000f7c0       ??$?RV<lambda_842d9ff0dc9ef11c61343bbaebe7f885>@@AEAV<lambda_c5860995281e5c4ce005b3de8f5874ee>@@V<lambda_d90129c13df834fdcbf8d2b88dafcf2d>@@@?$__crt_seh_guarded_call@X@@QEAAX$$QEAV<lambda_842d9ff0dc9ef11c61343bbaebe7f885>@@AEAV<lambda_c5860995281e5c4ce005b3de8f5874ee>@@$$QEAV<lambda_d90129c13df834fdcbf8d2b88dafcf2d>@@@Z 00000001800107c0 f   libucrt:fflush.obj
 0001:0000f85c       ??$?RV<lambda_886d6c58226a84441f68b9f2b8217b83>@@AEAV<lambda_ab61a845afdef5b7c387490eaf3616ee>@@V<lambda_f7f22ab5edc0698d5f6905b0d3f44752>@@@?$__crt_seh_guarded_call@X@@QEAAX$$QEAV<lambda_886d6c58226a84441f68b9f2b8217b83>@@AEAV<lambda_ab61a845afdef5b7c387490eaf3616ee>@@$$QEAV<lambda_f7f22ab5edc0698d5f6905b0d3f44752>@@@Z 000000018001085c f   libucrt:fflush.obj
 0001:0000f93c       ?common_flush_all@@YAH_N@Z 000000018001093c f   libucrt:fflush.obj
 0001:0000fe14       ??$?RV<lambda_410d79af7f07d98d83a3f525b3859a53>@@AEAV<lambda_3e16ef9562a7dcce91392c22ab16ea36>@@V<lambda_38119f0e861e05405d8a144b9b982f0a>@@@?$__crt_seh_guarded_call@X@@QEAAX$$QEAV<lambda_410d79af7f07d98d83a3f525b3859a53>@@AEAV<lambda_3e16ef9562a7dcce91392c22ab16ea36>@@$$QEAV<lambda_38119f0e861e05405d8a144b9b982f0a>@@@Z 0000000180010e14 f   libucrt:wsetlocale.obj
 0001:000107a4       fallbackMethod             00000001800117a4 f   libucrt:strpbrk.obj
 0001:00010b74       $LN78                      0000000180011b74     libucrt:strpbrk.obj
 0001:00010bb0       $LN77                      0000000180011bb0     libucrt:strpbrk.obj
 0001:00010bf0       $LN76                      0000000180011bf0     libucrt:strpbrk.obj
 0001:00010e5c       ?__acrt_LCMapStringA_stat@@YAHPEAU__crt_locale_pointers@@PEB_WKPEBDHPEADHHH@Z 0000000180011e5c f   libucrt:lcmapstringa.obj
 0001:0001120c       ?initialize_multibyte@@YAHXZ 000000018001220c f   libucrt:multibyte_initializer.obj
 0001:000112dc       ?GetTableIndexFromLocaleName@@YAHPEB_W@Z 00000001800122dc f   libucrt:lcidtoname_downlevel.obj
 0001:0001171c       ??$?RV<lambda_a37b2b86f63e897a80ea819b0eb08c01>@@AEAV<lambda_38ce7e780aa69e748d6df282ebc68efe>@@V<lambda_99fb1378e971ab6e7edea83e3a7a83a2>@@@?$__crt_seh_guarded_call@H@@QEAAH$$QEAV<lambda_a37b2b86f63e897a80ea819b0eb08c01>@@AEAV<lambda_38ce7e780aa69e748d6df282ebc68efe>@@$$QEAV<lambda_99fb1378e971ab6e7edea83e3a7a83a2>@@@Z 000000018001271c f   libucrt:commit.obj
 0001:0001183c       ?write_double_translated_ansi_nolock@@YA?AUwrite_result@?A0x17268360@@HQEBDI@Z 000000018001283c f   libucrt:write.obj
 0001:00011d18       ?write_text_ansi_nolock@@YA?AUwrite_result@?A0x17268360@@HQEBDI@Z 0000000180012d18 f   libucrt:write.obj
 0001:00011e1c       ?write_text_utf16le_nolock@@YA?AUwrite_result@?A0x17268360@@HQEBDI@Z 0000000180012e1c f   libucrt:write.obj
 0001:00011f38       ?write_text_utf8_nolock@@YA?AUwrite_result@?A0x17268360@@HQEBDI@Z 0000000180012f38 f   libucrt:write.obj
 0001:0001293c       ?free_crt_array_internal@@YAXQEAPEBX_K@Z 000000018001393c f   libucrt:inittime.obj
 0001:00012abc       ??$common_lseek_nolock@_J@@YA_JH_JH@Z 0000000180013abc f   libucrt:lseek.obj
 0001:00012e60       $$000000                   0000000180013e60     libucrt:log10.obj
 0001:0001353c       ??$?RV<lambda_751a882b2c74d4b022dec766aa51a29a>@@AEAV<lambda_628dfdc04ba53c8bfc02c9951375f3f5>@@V<lambda_f6c7be5f7998530c34de24c7437d6b54>@@@?$__crt_seh_guarded_call@H@@QEAAH$$QEAV<lambda_751a882b2c74d4b022dec766aa51a29a>@@AEAV<lambda_628dfdc04ba53c8bfc02c9951375f3f5>@@$$QEAV<lambda_f6c7be5f7998530c34de24c7437d6b54>@@@Z 000000018001453c f   libucrt:close.obj
 0001:00013730       _call_matherr              0000000180014730 f   libucrt:libm_error.obj
 0001:00013798       _exception_enabled         0000000180014798 f   libucrt:libm_error.obj
 0001:00013a10       _log_special_common        0000000180014a10 f   libucrt:log_special.obj
 0001:00013ab0       $$000000                   0000000180014ab0     libucrt:fpsr.obj
 0001:000140a0       $$000000                   00000001800150a0     LIBCMT:amdsecgs.obj
 0001:0001428c       capture_current_context    000000018001528c f   LIBCMT:gs_report.obj
 0001:000142fc       capture_previous_context   00000001800152fc f   LIBCMT:gs_report.obj
 0001:00014370       $$000000                   0000000180015370     libvcruntime:memcmp.obj
 0001:00014450       $$000000                   0000000180015450     LIBCMT:guard_dispatch.obj
 0001:00014470       ?fin$0@?0??dllmain_crt_process_attach@@YAHQEAUHINSTANCE__@@QEAX@Z@4HA 0000000180015470 f   LIBCMT:dll_dllmain.obj
 0001:00014487       ?fin$0@?0??dllmain_crt_process_detach@@YAH_N@Z@4HA 0000000180015487 f   LIBCMT:dll_dllmain.obj
 0001:000144a3       ?filt$0@?0??dllmain_dispatch@@YAHQEAUHINSTANCE__@@KQEAX@Z@4HA 00000001800154a3 f   LIBCMT:dll_dllmain.obj
 0001:000144d9       __scrt_is_nonwritable_in_current_image$filt$0 00000001800154d9 f   LIBCMT:utility.obj
 0001:000144f1       __DestructExceptionObject$filt$0 00000001800154f1 f   libvcruntime:ehhelpers.obj
 0001:00014509       _query_new_handler$fin$0   0000000180015509 f   libucrt:new_handler.obj
 0001:0001451f       ?fin$0@?0???$?RV<lambda_efdfa57d1f175319df784efa44bb7b81>@@AEAV<lambda_5f0a4c1567f8adc6734073e5d1e1b35c>@@V<lambda_2e8a7d3640ea6ccb4c2413664c2db6fd>@@@?$__crt_seh_guarded_call@X@@QEAAX$$QEAV<lambda_efdfa57d1f175319df784efa44bb7b81>@@AEAV<lambda_5f0a4c1567f8adc6734073e5d1e1b35c>@@$$QEAV<lambda_2e8a7d3640ea6ccb4c2413664c2db6fd>@@@Z@4HA 000000018001551f f   libucrt:mbctype.obj
 0001:0001451f       ?fin$0@?0???$?RV<lambda_aa87e3671a710a21b5dc78c0bdf72e11>@@AEAV<lambda_92619d2358a28f41a33ba319515a20b9>@@V<lambda_6992ecaafeb10aed2b74cb1fae11a551>@@@?$__crt_seh_guarded_call@X@@QEAAX$$QEAV<lambda_aa87e3671a710a21b5dc78c0bdf72e11>@@AEAV<lambda_92619d2358a28f41a33ba319515a20b9>@@$$QEAV<lambda_6992ecaafeb10aed2b74cb1fae11a551>@@@Z@4HA 000000018001551f f   libucrt:per_thread_data.obj
 0001:0001451f       ?fin$0@?0???$?RV<lambda_2d41944a1d46af3157314b8a01080d33>@@AEAV<lambda_8f455de75cd7d7f24b4096f044d8b9e6>@@V<lambda_aa500f224e6afead328df44964fe2772>@@@?$__crt_seh_guarded_call@X@@QEAAX$$QEAV<lambda_2d41944a1d46af3157314b8a01080d33>@@AEAV<lambda_8f455de75cd7d7f24b4096f044d8b9e6>@@$$QEAV<lambda_aa500f224e6afead328df44964fe2772>@@@Z@4HA 000000018001551f f   libucrt:per_thread_data.obj
 0001:0001451f       ?fin$0@?0???$?RV<lambda_f2e299630e499de9f9a165e60fcd3db5>@@AEAV<lambda_2ae9d31cdba2644fcbeaf08da7c24588>@@V<lambda_40d01ff24d0e7b3814fdbdcee8eab3c7>@@@?$__crt_seh_guarded_call@X@@QEAAX$$QEAV<lambda_f2e299630e499de9f9a165e60fcd3db5>@@AEAV<lambda_2ae9d31cdba2644fcbeaf08da7c24588>@@$$QEAV<lambda_40d01ff24d0e7b3814fdbdcee8eab3c7>@@@Z@4HA 000000018001551f f   libucrt:per_thread_data.obj
 0001:0001451f       ?fin$0@?0???$?RV<lambda_d80eeec6fff315bfe5c115232f3240e3>@@AEAV<lambda_6e4b09c48022b2350581041d5f6b0c4c>@@V<lambda_2358e3775559c9db80273638284d5e45>@@@?$__crt_seh_guarded_call@X@@QEAAX$$QEAV<lambda_d80eeec6fff315bfe5c115232f3240e3>@@AEAV<lambda_6e4b09c48022b2350581041d5f6b0c4c>@@$$QEAV<lambda_2358e3775559c9db80273638284d5e45>@@@Z@4HA 000000018001551f f   libucrt:exit.obj
 0001:0001451f       ?fin$0@?0???$?RV<lambda_7777bce6b2f8c936911f934f8298dc43>@@AEAV<lambda_f03950bc5685219e0bcd2087efbe011e>@@V<lambda_3883c3dff614d5e0c5f61bb1ac94921c>@@@?$__crt_seh_guarded_call@H@@QEAAH$$QEAV<lambda_7777bce6b2f8c936911f934f8298dc43>@@AEAV<lambda_f03950bc5685219e0bcd2087efbe011e>@@$$QEAV<lambda_3883c3dff614d5e0c5f61bb1ac94921c>@@@Z@4HA 000000018001551f f   libucrt:onexit.obj
 0001:0001451f       ?fin$0@?0???$?RV<lambda_0ae27a3a962d80f24befdcbee591983d>@@AEAV<lambda_8d0ee55de4b1038c4002e0adecdf1839>@@V<lambda_dc504788e8f1664fe9b84e20bfb512f2>@@@?$__crt_seh_guarded_call@X@@QEAAX$$QEAV<lambda_0ae27a3a962d80f24befdcbee591983d>@@AEAV<lambda_8d0ee55de4b1038c4002e0adecdf1839>@@$$QEAV<lambda_dc504788e8f1664fe9b84e20bfb512f2>@@@Z@4HA 000000018001551f f   libucrt:per_thread_data.obj
 0001:0001451f       ?fin$0@?0???$?RV<lambda_450d765d439847d4c735a33c368b5fc0>@@AEAV<lambda_44731a7d0e6d81c3e6aa82d741081786>@@V<lambda_601a2a7da3b7a96e9554ac7215c4b07c>@@@?$__crt_seh_guarded_call@P6AXH@Z@@QEAAP6AXH@Z$$QEAV<lambda_450d765d439847d4c735a33c368b5fc0>@@AEAV<lambda_44731a7d0e6d81c3e6aa82d741081786>@@$$QEAV<lambda_601a2a7da3b7a96e9554ac7215c4b07c>@@@Z@4HA 000000018001551f f   libucrt:signal.obj
 0001:00014539       ?filt$0@?0???R<lambda_6e4b09c48022b2350581041d5f6b0c4c>@@QEBA@XZ@4HA 0000000180015539 f   libucrt:exit.obj
 0001:00014554       ?fin$0@?0??update_thread_multibyte_data_internal@@YAPEAU__crt_multibyte_data@@QEAU__acrt_ptd@@QEAPEAU1@@Z@4HA 0000000180015554 f   libucrt:mbctype.obj
 0001:0001456d       __acrt_lowio_ensure_fh_exists$fin$0 000000018001556d f   libucrt:osfinfo.obj
 0001:0001456d       __acrt_initialize_lowio$fin$0 000000018001556d f   libucrt:ioinit.obj
 0001:00014586       raise$fin$0                0000000180015586 f   libucrt:signal.obj
 0001:000145a7       ?fin$0@?0???$?RV<lambda_842d9ff0dc9ef11c61343bbaebe7f885>@@AEAV<lambda_c5860995281e5c4ce005b3de8f5874ee>@@V<lambda_d90129c13df834fdcbf8d2b88dafcf2d>@@@?$__crt_seh_guarded_call@X@@QEAAX$$QEAV<lambda_842d9ff0dc9ef11c61343bbaebe7f885>@@AEAV<lambda_c5860995281e5c4ce005b3de8f5874ee>@@$$QEAV<lambda_d90129c13df834fdcbf8d2b88dafcf2d>@@@Z@4HA 00000001800155a7 f   libucrt:fflush.obj
 0001:000145c2       ?fin$0@?0???$?RV<lambda_886d6c58226a84441f68b9f2b8217b83>@@AEAV<lambda_ab61a845afdef5b7c387490eaf3616ee>@@V<lambda_f7f22ab5edc0698d5f6905b0d3f44752>@@@?$__crt_seh_guarded_call@X@@QEAAX$$QEAV<lambda_886d6c58226a84441f68b9f2b8217b83>@@AEAV<lambda_ab61a845afdef5b7c387490eaf3616ee>@@$$QEAV<lambda_f7f22ab5edc0698d5f6905b0d3f44752>@@@Z@4HA 00000001800155c2 f   libucrt:fflush.obj
 0001:000145df       ?fin$0@?0???$?RV<lambda_410d79af7f07d98d83a3f525b3859a53>@@AEAV<lambda_3e16ef9562a7dcce91392c22ab16ea36>@@V<lambda_38119f0e861e05405d8a144b9b982f0a>@@@?$__crt_seh_guarded_call@X@@QEAAX$$QEAV<lambda_410d79af7f07d98d83a3f525b3859a53>@@AEAV<lambda_3e16ef9562a7dcce91392c22ab16ea36>@@$$QEAV<lambda_38119f0e861e05405d8a144b9b982f0a>@@@Z@4HA 00000001800155df f   libucrt:wsetlocale.obj
 0001:000145f9       __acrt_update_thread_locale_data$fin$0 00000001800155f9 f   libucrt:locale_refcounting.obj
 0001:00014612       ?fin$0@?0???$?RV<lambda_751a882b2c74d4b022dec766aa51a29a>@@AEAV<lambda_628dfdc04ba53c8bfc02c9951375f3f5>@@V<lambda_f6c7be5f7998530c34de24c7437d6b54>@@@?$__crt_seh_guarded_call@H@@QEAAH$$QEAV<lambda_751a882b2c74d4b022dec766aa51a29a>@@AEAV<lambda_628dfdc04ba53c8bfc02c9951375f3f5>@@$$QEAV<lambda_f6c7be5f7998530c34de24c7437d6b54>@@@Z@4HA 0000000180015612 f   libucrt:close.obj
 0001:00014612       ?fin$0@?0???$?RV<lambda_a37b2b86f63e897a80ea819b0eb08c01>@@AEAV<lambda_38ce7e780aa69e748d6df282ebc68efe>@@V<lambda_99fb1378e971ab6e7edea83e3a7a83a2>@@@?$__crt_seh_guarded_call@H@@QEAAH$$QEAV<lambda_a37b2b86f63e897a80ea819b0eb08c01>@@AEAV<lambda_38ce7e780aa69e748d6df282ebc68efe>@@$$QEAV<lambda_99fb1378e971ab6e7edea83e3a7a83a2>@@@Z@4HA 0000000180015612 f   libucrt:commit.obj
 0001:0001462c       _write$fin$0               000000018001562c f   libucrt:write.obj
 0001:00014643       _fcloseall$fin$0           0000000180015643 f   libucrt:closeall.obj
 0001:0001465c       fclose$fin$0               000000018001565c f   libucrt:fclose.obj
 0001:00014674       _ctrlfp$filt$0             0000000180015674 f   libucrt:fpctrl.obj
 0001:000146a0       _IsNonwritableInCurrentImage$filt$0 00000001800156a0 f   LIBCMT:pesect.obj
 0001:000146c0       $xdatasym                  00000001800156c0     chkstk.obj
 0001:000146c8       $unwind$ConfigureW         00000001800156c8     SameFolder.obj
 0001:000146d8       $chain$2$ConfigureW        00000001800156d8     SameFolder.obj
 0001:000146f4       $chain$3$ConfigureW        00000001800156f4     SameFolder.obj
 0001:00014708       $chain$4$ConfigureW        0000000180015708     SameFolder.obj
 0001:00014718       $chain$5$ConfigureW        0000000180015718     SameFolder.obj
 0001:00014728       $unwind$_isatty            0000000180015728     libucrt:isatty.obj
 0001:00014728       $unwind$__acrt_update_thread_multibyte_data 0000000180015728     libucrt:mbctype.obj
 0001:00014728       $unwind$__vcrt_initialize_ptd 0000000180015728     libvcruntime:per_thread_data.obj
 0001:00014728       $unwind$__acrt_thread_detach 0000000180015728     libucrt:initialization.obj
 0001:00014728       $unwind$__acrt_thread_attach 0000000180015728     libucrt:initialization.obj
 0001:00014728       $unwind$abort              0000000180015728     libucrt:abort.obj
 0001:00014728       $unwind$__acrt_uninitialize_critical 0000000180015728     libucrt:initialization.obj
 0001:00014728       $unwind$initialize_c       0000000180015728     libucrt:initialization.obj
 0001:00014728       $unwind$__acrt_uninitialize 0000000180015728     libucrt:initialization.obj
 0001:00014728       $unwind$__acrt_initialize_heap 0000000180015728     libucrt:heap_handle.obj
 0001:00014728       $unwind$__report_rangecheckfailure 0000000180015728     LIBCMT:gs_report.obj
 0001:00014728       $unwind$__doserrno         0000000180015728     libucrt:errno.obj
 0001:00014728       $unwind$__vcrt_uninitialize_ptd 0000000180015728     libvcruntime:per_thread_data.obj
 0001:00014728       $unwind$_errno             0000000180015728     libucrt:errno.obj
 0001:00014728       $unwind$uninitialize_environment 0000000180015728     libucrt:initialization.obj
 0001:00014728       $unwind$_get_osfhandle     0000000180015728     libucrt:osfinfo.obj
 0001:00014728       $unwind$uninitialize_allocated_io_buffers 0000000180015728     libucrt:initialization.obj
 0001:00014728       $unwind$__dcrt_uninitialize_environments_nolock 0000000180015728     libucrt:environment_initialization.obj
 0001:00014728       $unwind$__acrt_initialize_multibyte 0000000180015728     libucrt:mbctype.obj
 0001:00014728       $unwind$__vcrt_thread_detach 0000000180015728     libvcruntime:initialization.obj
 0001:00014728       $unwind$__acrt_DownlevelLocaleNameToLCID 0000000180015728     libucrt:lcidtoname_downlevel.obj
 0001:00014728       $unwind$__GSHandlerCheck   0000000180015728     LIBCMT:gshandler.obj
 0001:00014728       $unwind$_invoke_watson     0000000180015728     libucrt:invalid_parameter.obj
 0001:00014728       $unwind$??$uninitialize_environment_internal@D@@YAXAEAPEAPEAD@Z 0000000180015728     libucrt:environment_initialization.obj
 0001:00014728       $unwind$__vcrt_thread_attach 0000000180015728     libvcruntime:initialization.obj
 0001:00014728       $unwind$?dllmain_crt_dispatch@@YAHQEAUHINSTANCE__@@KQEAX@Z 0000000180015728     LIBCMT:dll_dllmain.obj
 0001:00014728       $unwind$__scrt_initialize_default_local_stdio_options 0000000180015728     LIBCMT:default_local_stdio_options.obj
 0001:00014728       $unwind$_msize_base        0000000180015728     libucrt:msize.obj
 0001:00014728       $unwind$??$uninitialize_environment_internal@_W@@YAXAEAPEAPEA_W@Z 0000000180015728     libucrt:environment_initialization.obj
 0001:00014728       $unwind$?initialize_multibyte@@YAHXZ 0000000180015728     libucrt:multibyte_initializer.obj
 0001:00014728       $unwind$__vcrt_uninitialize_critical 0000000180015728     libvcruntime:initialization.obj
 0001:00014728       $unwind$GetGlobalInfoW     0000000180015728     SameFolder.obj
 0001:00014728       $unwind$__vcrt_uninitialize 0000000180015728     libvcruntime:initialization.obj
 0001:00014728       $unwind$__vcrt_initialize  0000000180015728     libvcruntime:initialization.obj
 0001:00014728       $unwind$__acrt_initialize_command_line 0000000180015728     libucrt:argv_data.obj
 0001:00014728       $unwind$_statfp            0000000180015728     libucrt:fpctrl.obj
 0001:00014728       $unwind$__scrt_acquire_startup_lock 0000000180015728     LIBCMT:utility.obj
 0001:00014728       $unwind$__dcrt_terminate_console_output 0000000180015728     libucrt:initcon.obj
 0001:00014728       $unwind$_fileno            0000000180015728     libucrt:fileno.obj
 0001:00014728       $unwind$__pctype_func      0000000180015728     libucrt:ctype.obj
 0001:00014728       $unwind$__acrt_release_locale_ref 0000000180015728     libucrt:locale_refcounting.obj
 0001:00014728       $unwind$__vcrt_freefls     0000000180015728     libvcruntime:per_thread_data.obj
 0001:00014728       $unwind$_set_errno_from_matherr 0000000180015728     libucrt:fpexcept.obj
 0001:00014728       $unwind$__acrt_uninitialize_ptd 0000000180015728     libucrt:per_thread_data.obj
 0001:00014728       $unwind$__acrt_initialize_ptd 0000000180015728     libucrt:per_thread_data.obj
 0001:00014728       $unwind$__scrt_dllmain_crt_thread_detach 0000000180015728     LIBCMT:utility.obj
 0001:00014728       $unwind$__scrt_dllmain_crt_thread_attach 0000000180015728     LIBCMT:utility.obj
 0001:00014728       $unwind$__scrt_dllmain_uninitialize_critical 0000000180015728     LIBCMT:utility.obj
 0001:00014728       $unwind$__scrt_dllmain_uninitialize_c 0000000180015728     LIBCMT:utility.obj
 0001:00014728       $unwind$__scrt_dllmain_after_initialize_c 0000000180015728     LIBCMT:utility.obj
 0001:00014728       $unwind$__acrt_AreFileApisANSI 0000000180015728     libucrt:winapi_thunks.obj
 0001:00014728       $unwind$__scrt_dllmain_before_initialize_c 0000000180015728     LIBCMT:utility.obj
 0001:00014730       $unwind$__acrt_execute_uninitializers 0000000180015730     libucrt:shared_initialization.obj
 0001:00014730       $unwind$__acrt_uninitialize_lowio 0000000180015730     libucrt:ioinit.obj
 0001:00014730       $unwind$strncpy_s          0000000180015730     libucrt:strncpy_s.obj
 0001:00014730       $unwind$?SaveValue@PluginRadioButtonBinding@@UEAAXPEAUFarDialogItem@@H@Z 0000000180015730     SameFolder.obj
 0001:00014730       $unwind$__acrt_errno_map_os_error 0000000180015730     libucrt:errno.obj
 0001:00014730       $unwind$_updatetlocinfoEx_nolock 0000000180015730     libucrt:locale_refcounting.obj
 0001:00014730       $unwind$??_Gexception@std@@UEAAPEAXI@Z 0000000180015730     LIBCMT:throw_bad_alloc.obj
 0001:00014730       $unwind$??_GPluginDialogBuilder@@UEAAPEAXI@Z 0000000180015730     SameFolder.obj
 0001:00014730       $unwind$??_Gbad_alloc@std@@UEAAPEAXI@Z 0000000180015730     LIBCMT:throw_bad_alloc.obj
 0001:00014730       $unwind$??_Gbad_array_new_length@std@@UEAAPEAXI@Z 0000000180015730     LIBCMT:throw_bad_alloc.obj
 0001:00014730       $unwind$?CreateRadioButtonBinding@PluginDialogBuilder@@MEAAPEAU?$DialogItemBinding@UFarDialogItem@@@@PEAH@Z 0000000180015730     SameFolder.obj
 0001:00014730       $unwind$?InitDialogItem@PluginDialogBuilder@@MEAAXPEAUFarDialogItem@@PEB_W@Z 0000000180015730     SameFolder.obj
 0001:00014730       $unwind$??$common_initialize_environment_nolock@D@@YAHXZ 0000000180015730     libucrt:environment_initialization.obj
 0001:00014730       $unwind$_close_nolock      0000000180015730     libucrt:close.obj
 0001:00014730       $unwind$_RTC_Initialize    0000000180015730     LIBCMT:initsect.obj
 0001:00014730       $unwind$??_G?$DialogBuilderBase@UFarDialogItem@@@@MEAAPEAXI@Z 0000000180015730     SameFolder.obj
 0001:00014730       $unwind$_initterm_e        0000000180015730     libucrt:initterm.obj
 0001:00014730       $unwind$_RTC_Terminate     0000000180015730     LIBCMT:initsect.obj
 0001:00014730       $unwind$_realloc_base      0000000180015730     libucrt:realloc_base.obj
 0001:00014730       $unwind$_fclose_nolock     0000000180015730     libucrt:fclose.obj
 0001:00014730       $unwind$GetPluginInfoW     0000000180015730     SameFolder.obj
 0001:00014730       $unwind$__acrt_FlsSetValue 0000000180015730     libucrt:winapi_thunks.obj
 0001:00014730       $unwind$?replace_current_thread_locale_nolock@@YAXQEAU__acrt_ptd@@QEAU__crt_locale_data@@@Z 0000000180015730     libucrt:per_thread_data.obj
 0001:00014730       $unwind$__acrt_LocaleNameToLCID 0000000180015730     libucrt:winapi_thunks.obj
 0001:00014730       $unwind$__vcrt_FlsSetValue 0000000180015730     libvcruntime:winapi_downlevel.obj
 0001:0001473c       $unwind$OpenW              000000018001573c     SameFolder.obj
 0001:0001474c       $chain$0$OpenW             000000018001574c     SameFolder.obj
 0001:00014760       $chain$2$OpenW             0000000180015760     SameFolder.obj
 0001:00014778       $chain$3$OpenW             0000000180015778     SameFolder.obj
 0001:00014788       $chain$5$OpenW             0000000180015788     SameFolder.obj
 0001:0001479c       $chain$6$OpenW             000000018001579c     SameFolder.obj
 0001:000147ac       $unwind$SetStartupInfoW    00000001800157ac     SameFolder.obj
 0001:000147c0       $unwind$__scrt_release_startup_lock 00000001800157c0     LIBCMT:utility.obj
 0001:000147c0       $unwind$__vcrt_FlsGetValue 00000001800157c0     libvcruntime:winapi_downlevel.obj
 0001:000147c0       $unwind$__vcrt_FlsFree     00000001800157c0     libvcruntime:winapi_downlevel.obj
 0001:000147c0       $unwind$__vcrt_FlsAlloc    00000001800157c0     libvcruntime:winapi_downlevel.obj
 0001:000147c0       $unwind$__std_exception_destroy 00000001800157c0     libvcruntime:std_exception.obj
 0001:000147c0       $unwind$__acrt_uninitialize_stdio 00000001800157c0     libucrt:_file.obj
 0001:000147c0       $unwind$__acrt_update_locale_info 00000001800157c0     libucrt:locale_update.obj
 0001:000147c0       $unwind$__acrt_update_multibyte_info 00000001800157c0     libucrt:locale_update.obj
 0001:000147c0       $unwind$__acrt_AppPolicyGetProcessTerminationMethodInternal 00000001800157c0     libucrt:winapi_thunks.obj
 0001:000147c0       $unwind$??_GPluginRadioButtonBinding@@UEAAPEAXI@Z 00000001800157c0     SameFolder.obj
 0001:000147c0       $unwind$_set_statfp        00000001800157c0     libucrt:fpctrl.obj
 0001:000147c0       $unwind$__std_type_info_destroy_list 00000001800157c0     libvcruntime:std_type_info.obj
 0001:000147c0       $unwind$_clrfp             00000001800157c0     libucrt:fpctrl.obj
 0001:000147c0       $unwind$uninitialize_allocated_memory 00000001800157c0     libucrt:initialization.obj
 0001:000147c0       $unwind$??_G?$DialogItemBinding@UFarDialogItem@@@@UEAAPEAXI@Z 00000001800157c0     SameFolder.obj
 0001:000147c0       $unwind$__acrt_getptd_head 00000001800157c0     libucrt:per_thread_data.obj
 0001:000147c0       $unwind$_callnewh          00000001800157c0     libucrt:new_handler.obj
 0001:000147c0       $unwind$__acrt_get_process_end_policy 00000001800157c0     libucrt:win_policies.obj
 0001:000147c0       $unwind$??_Gtype_info@@UEAAPEAXI@Z 00000001800157c0     LIBCMT:std_type_info_static.obj
 0001:000147c0       $unwind$?SaveValue@PluginCheckBoxBinding@@UEAAXPEAUFarDialogItem@@H@Z 00000001800157c0     SameFolder.obj
 0001:000147c0       $unwind$__scrt_initialize_crt 00000001800157c0     LIBCMT:utility.obj
 0001:000147c0       $unwind$__scrt_uninitialize_crt 00000001800157c0     LIBCMT:utility.obj
 0001:000147c0       $unwind$_fflush_nolock     00000001800157c0     libucrt:fflush.obj
 0001:000147c0       $unwind$__acrt_FlsFree     00000001800157c0     libucrt:winapi_thunks.obj
 0001:000147c0       $unwind$__acrt_uninitialize_locks 00000001800157c0     libucrt:locks.obj
 0001:000147c0       $unwind$??_GPluginUIntEditFieldBinding@@UEAAPEAXI@Z 00000001800157c0     SameFolder.obj
 0001:000147c0       $unwind$??_GPluginCheckBoxBinding@@UEAAPEAXI@Z 00000001800157c0     SameFolder.obj
 0001:000147c0       $unwind$??0bad_array_new_length@std@@QEAA@AEBV01@@Z 00000001800157c0     LIBCMT:throw_bad_alloc.obj
 0001:000147c0       $unwind$?SaveValue@PluginUIntEditFieldBinding@@UEAAXPEAUFarDialogItem@@H@Z 00000001800157c0     SameFolder.obj
 0001:000147c0       $unwind$__acrt_initialize_locks 00000001800157c0     libucrt:locks.obj
 0001:000147c0       $unwind$_malloc_base       00000001800157c0     libucrt:malloc_base.obj
 0001:000147c0       $unwind$__acrt_FlsAlloc    00000001800157c0     libucrt:winapi_thunks.obj
 0001:000147c0       $unwind$__raise_securityfailure 00000001800157c0     LIBCMT:gs_report.obj
 0001:000147c0       $unwind$??0bad_alloc@std@@QEAA@AEBV01@@Z 00000001800157c0     LIBCMT:throw_bad_alloc.obj
 0001:000147c0       $unwind$??_GPluginIntEditFieldBinding@@UEAAPEAXI@Z 00000001800157c0     SameFolder.obj
 0001:000147c0       $unwind$?SaveValue@PluginIntEditFieldBinding@@UEAAXPEAUFarDialogItem@@H@Z 00000001800157c0     SameFolder.obj
 0001:000147c0       $unwind$??0exception@std@@QEAA@AEBV01@@Z 00000001800157c0     LIBCMT:throw_bad_alloc.obj
 0001:000147c0       $unwind$??2@YAPEAX_K@Z     00000001800157c0     LIBCMT:new_scalar.obj
 0001:000147c0       $unwind$strcpy_s           00000001800157c0     libucrt:strcpy_s.obj
 0001:000147c0       $unwind$_calloc_base       00000001800157c0     libucrt:calloc_base.obj
 0001:000147c0       $unwind$__acrt_stdio_free_buffer_nolock 00000001800157c0     libucrt:_freebuf.obj
 0001:000147c0       $unwind$__acrt_allocate_buffer_for_argv 00000001800157c0     libucrt:argv_parsing.obj
 0001:000147c0       $unwind$__vcrt_uninitialize_locks 00000001800157c0     libvcruntime:locks.obj
 0001:000147c0       $unwind$?exit_or_terminate_process@@YAXI@Z 00000001800157c0     libucrt:exit.obj
 0001:000147c0       $unwind$?try_cor_exit_process@@YAXI@Z 00000001800157c0     libucrt:exit.obj
 0001:000147c0       $unwind$initialize_pointers 00000001800157c0     libucrt:initialization.obj
 0001:000147c0       $unwind$__acrt_uninitialize_winapi_thunks 00000001800157c0     libucrt:winapi_thunks.obj
 0001:000147c0       $unwind$__acrt_freeptd     00000001800157c0     libucrt:per_thread_data.obj
 0001:000147c0       $unwind$__vcrt_freeptd     00000001800157c0     libvcruntime:per_thread_data.obj
 0001:000147c0       $unwind$__vcrt_initialize_locks 00000001800157c0     libvcruntime:locks.obj
 0001:000147c0       $unwind$__acrt_FlsGetValue 00000001800157c0     libucrt:winapi_thunks.obj
 0001:000147c8       $unwind$?AddIntEditField@PluginDialogBuilder@@UEAAPEAUFarDialogItem@@PEAHH@Z 00000001800157c8     SameFolder.obj
 0001:000147c8       $unwind$?AddUIntEditField@PluginDialogBuilder@@UEAAPEAUFarDialogItem@@PEAIH@Z 00000001800157c8     SameFolder.obj
 0001:000147c8       $unwind$?AddDialogItem@?$DialogBuilderBase@UFarDialogItem@@@@IEAAPEAUFarDialogItem@@W4FARDIALOGITEMTYPES@@PEB_W@Z 00000001800157c8     SameFolder.obj
 0001:000147e0       $unwind$?UpdateBorderSize@?$DialogBuilderBase@UFarDialogItem@@@@IEAAXXZ 00000001800157e0     SameFolder.obj
 0001:000147f0       $chain$1$?UpdateBorderSize@?$DialogBuilderBase@UFarDialogItem@@@@IEAAXXZ 00000001800157f0     SameFolder.obj
 0001:00014808       $chain$2$?UpdateBorderSize@?$DialogBuilderBase@UFarDialogItem@@@@IEAAXXZ 0000000180015808     SameFolder.obj
 0001:0001481c       $chain$3$?UpdateBorderSize@?$DialogBuilderBase@UFarDialogItem@@@@IEAAXXZ 000000018001581c     SameFolder.obj
 0001:0001482c       $chain$4$?UpdateBorderSize@?$DialogBuilderBase@UFarDialogItem@@@@IEAAXXZ 000000018001582c     SameFolder.obj
 0001:0001483c       $unwind$??1?$DialogBuilderBase@UFarDialogItem@@@@MEAA@XZ 000000018001583c     SameFolder.obj
 0001:00014848       $chain$0$??1?$DialogBuilderBase@UFarDialogItem@@@@MEAA@XZ 0000000180015848     SameFolder.obj
 0001:0001485c       $chain$1$??1?$DialogBuilderBase@UFarDialogItem@@@@MEAA@XZ 000000018001585c     SameFolder.obj
 0001:0001486c       $unwind$?AddButtons@?$DialogBuilderBase@UFarDialogItem@@@@QEAAXHPEBHHH@Z 000000018001586c     SameFolder.obj
 0001:00014878       $chain$4$?AddButtons@?$DialogBuilderBase@UFarDialogItem@@@@QEAAXHPEBHHH@Z 0000000180015878     SameFolder.obj
 0001:0001489c       $chain$5$?AddButtons@?$DialogBuilderBase@UFarDialogItem@@@@QEAAXHPEBHHH@Z 000000018001589c     SameFolder.obj
 0001:000148ac       $unwind$?DoShowDialog@PluginDialogBuilder@@MEAA_JXZ 00000001800158ac     SameFolder.obj
 0001:000148b8       $unwind$__acrt_stdio_flush_nolock 00000001800158b8     libucrt:fflush.obj
 0001:000148b8       $unwind$??$common_lseek_nolock@_J@@YA_JH_JH@Z 00000001800158b8     libucrt:lseek.obj
 0001:000148b8       $unwind$_DllMainCRTStartup 00000001800158b8     LIBCMT:dll_dllmain.obj
 0001:000148b8       $unwind$__acrt_getptd_noexit 00000001800158b8     libucrt:per_thread_data.obj
 0001:000148b8       $unwind$_exception_enabled 00000001800158b8     libucrt:libm_error.obj
 0001:000148b8       $unwind$__acrt_execute_initializers 00000001800158b8     libucrt:shared_initialization.obj
 0001:000148b8       $unwind$__vcrt_getptd_noexit 00000001800158b8     libvcruntime:per_thread_data.obj
 0001:000148b8       $unwind$__acrt_InitializeCriticalSectionEx 00000001800158b8     libucrt:winapi_thunks.obj
 0001:000148b8       $unwind$__acrt_getptd      00000001800158b8     libucrt:per_thread_data.obj
 0001:000148b8       $unwind$??0_LocaleUpdate@@QEAA@QEAU__crt_locale_pointers@@@Z 00000001800158b8     libucrt:output.obj
 0001:000148b8       $unwind$?free_crt_array_internal@@YAXQEAPEBX_K@Z 00000001800158b8     libucrt:inittime.obj
 0001:000148b8       $unwind$__vcrt_InitializeCriticalSectionEx 00000001800158b8     libvcruntime:winapi_downlevel.obj
 0001:000148b8       $unwind$?CreateCheckBoxBinding@PluginDialogBuilder@@MEAAPEAU?$DialogItemBinding@UFarDialogItem@@@@PEAHH@Z 00000001800158b8     SameFolder.obj
 0001:000148c8       $unwind$?dllmain_crt_process_attach@@YAHQEAUHINSTANCE__@@QEAX@Z 00000001800158c8     LIBCMT:dll_dllmain.obj
 0001:00014904       $unwind$__acrt_initialize_lowio$fin$0 0000000180015904     libucrt:ioinit.obj
 0001:00014904       $unwind$fclose$fin$0       0000000180015904     libucrt:fclose.obj
 0001:00014904       $unwind$_IsNonwritableInCurrentImage$filt$0 0000000180015904     LIBCMT:pesect.obj
 0001:00014904       $unwind$raise$fin$0        0000000180015904     libucrt:signal.obj
 0001:00014904       $unwind$?filt$0@?0???R<lambda_6e4b09c48022b2350581041d5f6b0c4c>@@QEBA@XZ@4HA 0000000180015904     libucrt:exit.obj
 0001:00014904       $unwind$_fcloseall$fin$0   0000000180015904     libucrt:closeall.obj
 0001:00014904       $unwind$?fin$0@?0???$?RV<lambda_2d41944a1d46af3157314b8a01080d33>@@AEAV<lambda_8f455de75cd7d7f24b4096f044d8b9e6>@@V<lambda_aa500f224e6afead328df44964fe2772>@@@?$__crt_seh_guarded_call@X@@QEAAX$$QEAV<lambda_2d41944a1d46af3157314b8a01080d33>@@AEAV<lambda_8f455de75cd7d7f24b4096f044d8b9e6>@@$$QEAV<lambda_aa500f224e6afead328df44964fe2772>@@@Z@4HA 0000000180015904     libucrt:per_thread_data.obj
 0001:00014904       $unwind$?fin$0@?0???$?RV<lambda_410d79af7f07d98d83a3f525b3859a53>@@AEAV<lambda_3e16ef9562a7dcce91392c22ab16ea36>@@V<lambda_38119f0e861e05405d8a144b9b982f0a>@@@?$__crt_seh_guarded_call@X@@QEAAX$$QEAV<lambda_410d79af7f07d98d83a3f525b3859a53>@@AEAV<lambda_3e16ef9562a7dcce91392c22ab16ea36>@@$$QEAV<lambda_38119f0e861e05405d8a144b9b982f0a>@@@Z@4HA 0000000180015904     libucrt:wsetlocale.obj
 0001:00014904       $unwind$?fin$0@?0??update_thread_multibyte_data_internal@@YAPEAU__crt_multibyte_data@@QEAU__acrt_ptd@@QEAPEAU1@@Z@4HA 0000000180015904     libucrt:mbctype.obj
 0001:00014904       $unwind$?fin$0@?0???$?RV<lambda_0ae27a3a962d80f24befdcbee591983d>@@AEAV<lambda_8d0ee55de4b1038c4002e0adecdf1839>@@V<lambda_dc504788e8f1664fe9b84e20bfb512f2>@@@?$__crt_seh_guarded_call@X@@QEAAX$$QEAV<lambda_0ae27a3a962d80f24befdcbee591983d>@@AEAV<lambda_8d0ee55de4b1038c4002e0adecdf1839>@@$$QEAV<lambda_dc504788e8f1664fe9b84e20bfb512f2>@@@Z@4HA 0000000180015904     libucrt:per_thread_data.obj
 0001:00014904       $unwind$__acrt_lowio_ensure_fh_exists$fin$0 0000000180015904     libucrt:osfinfo.obj
 0001:00014904       $unwind$?fin$0@?0??dllmain_crt_process_attach@@YAHQEAUHINSTANCE__@@QEAX@Z@4HA 0000000180015904     LIBCMT:dll_dllmain.obj
 0001:00014904       $unwind$?fin$0@?0???$?RV<lambda_751a882b2c74d4b022dec766aa51a29a>@@AEAV<lambda_628dfdc04ba53c8bfc02c9951375f3f5>@@V<lambda_f6c7be5f7998530c34de24c7437d6b54>@@@?$__crt_seh_guarded_call@H@@QEAAH$$QEAV<lambda_751a882b2c74d4b022dec766aa51a29a>@@AEAV<lambda_628dfdc04ba53c8bfc02c9951375f3f5>@@$$QEAV<lambda_f6c7be5f7998530c34de24c7437d6b54>@@@Z@4HA 0000000180015904     libucrt:close.obj
 0001:00014904       $unwind$__acrt_update_thread_locale_data$fin$0 0000000180015904     libucrt:locale_refcounting.obj
 0001:00014904       $unwind$?fin$0@?0???$?RV<lambda_886d6c58226a84441f68b9f2b8217b83>@@AEAV<lambda_ab61a845afdef5b7c387490eaf3616ee>@@V<lambda_f7f22ab5edc0698d5f6905b0d3f44752>@@@?$__crt_seh_guarded_call@X@@QEAAX$$QEAV<lambda_886d6c58226a84441f68b9f2b8217b83>@@AEAV<lambda_ab61a845afdef5b7c387490eaf3616ee>@@$$QEAV<lambda_f7f22ab5edc0698d5f6905b0d3f44752>@@@Z@4HA 0000000180015904     libucrt:fflush.obj
 0001:00014904       $unwind$?fin$0@?0???$?RV<lambda_842d9ff0dc9ef11c61343bbaebe7f885>@@AEAV<lambda_c5860995281e5c4ce005b3de8f5874ee>@@V<lambda_d90129c13df834fdcbf8d2b88dafcf2d>@@@?$__crt_seh_guarded_call@X@@QEAAX$$QEAV<lambda_842d9ff0dc9ef11c61343bbaebe7f885>@@AEAV<lambda_c5860995281e5c4ce005b3de8f5874ee>@@$$QEAV<lambda_d90129c13df834fdcbf8d2b88dafcf2d>@@@Z@4HA 0000000180015904     libucrt:fflush.obj
 0001:00014904       $unwind$?fin$0@?0???$?RV<lambda_aa87e3671a710a21b5dc78c0bdf72e11>@@AEAV<lambda_92619d2358a28f41a33ba319515a20b9>@@V<lambda_6992ecaafeb10aed2b74cb1fae11a551>@@@?$__crt_seh_guarded_call@X@@QEAAX$$QEAV<lambda_aa87e3671a710a21b5dc78c0bdf72e11>@@AEAV<lambda_92619d2358a28f41a33ba319515a20b9>@@$$QEAV<lambda_6992ecaafeb10aed2b74cb1fae11a551>@@@Z@4HA 0000000180015904     libucrt:per_thread_data.obj
 0001:00014904       $unwind$__DestructExceptionObject$filt$0 0000000180015904     libvcruntime:ehhelpers.obj
 0001:00014904       $unwind$?fin$0@?0???$?RV<lambda_efdfa57d1f175319df784efa44bb7b81>@@AEAV<lambda_5f0a4c1567f8adc6734073e5d1e1b35c>@@V<lambda_2e8a7d3640ea6ccb4c2413664c2db6fd>@@@?$__crt_seh_guarded_call@X@@QEAAX$$QEAV<lambda_efdfa57d1f175319df784efa44bb7b81>@@AEAV<lambda_5f0a4c1567f8adc6734073e5d1e1b35c>@@$$QEAV<lambda_2e8a7d3640ea6ccb4c2413664c2db6fd>@@@Z@4HA 0000000180015904     libucrt:mbctype.obj
 0001:00014904       $unwind$_query_new_handler$fin$0 0000000180015904     libucrt:new_handler.obj
 0001:00014904       $unwind$?fin$0@?0???$?RV<lambda_450d765d439847d4c735a33c368b5fc0>@@AEAV<lambda_44731a7d0e6d81c3e6aa82d741081786>@@V<lambda_601a2a7da3b7a96e9554ac7215c4b07c>@@@?$__crt_seh_guarded_call@P6AXH@Z@@QEAAP6AXH@Z$$QEAV<lambda_450d765d439847d4c735a33c368b5fc0>@@AEAV<lambda_44731a7d0e6d81c3e6aa82d741081786>@@$$QEAV<lambda_601a2a7da3b7a96e9554ac7215c4b07c>@@@Z@4HA 0000000180015904     libucrt:signal.obj
 0001:00014904       $unwind$?fin$0@?0??dllmain_crt_process_detach@@YAH_N@Z@4HA 0000000180015904     LIBCMT:dll_dllmain.obj
 0001:00014904       $unwind$_write$fin$0       0000000180015904     libucrt:write.obj
 0001:00014904       $unwind$?fin$0@?0???$?RV<lambda_f2e299630e499de9f9a165e60fcd3db5>@@AEAV<lambda_2ae9d31cdba2644fcbeaf08da7c24588>@@V<lambda_40d01ff24d0e7b3814fdbdcee8eab3c7>@@@?$__crt_seh_guarded_call@X@@QEAAX$$QEAV<lambda_f2e299630e499de9f9a165e60fcd3db5>@@AEAV<lambda_2ae9d31cdba2644fcbeaf08da7c24588>@@$$QEAV<lambda_40d01ff24d0e7b3814fdbdcee8eab3c7>@@@Z@4HA 0000000180015904     libucrt:per_thread_data.obj
 0001:00014904       $unwind$?fin$0@?0???$?RV<lambda_d80eeec6fff315bfe5c115232f3240e3>@@AEAV<lambda_6e4b09c48022b2350581041d5f6b0c4c>@@V<lambda_2358e3775559c9db80273638284d5e45>@@@?$__crt_seh_guarded_call@X@@QEAAX$$QEAV<lambda_d80eeec6fff315bfe5c115232f3240e3>@@AEAV<lambda_6e4b09c48022b2350581041d5f6b0c4c>@@$$QEAV<lambda_2358e3775559c9db80273638284d5e45>@@@Z@4HA 0000000180015904     libucrt:exit.obj
 0001:00014904       $unwind$?fin$0@?0???$?RV<lambda_7777bce6b2f8c936911f934f8298dc43>@@AEAV<lambda_f03950bc5685219e0bcd2087efbe011e>@@V<lambda_3883c3dff614d5e0c5f61bb1ac94921c>@@@?$__crt_seh_guarded_call@H@@QEAAH$$QEAV<lambda_7777bce6b2f8c936911f934f8298dc43>@@AEAV<lambda_f03950bc5685219e0bcd2087efbe011e>@@$$QEAV<lambda_3883c3dff614d5e0c5f61bb1ac94921c>@@@Z@4HA 0000000180015904     libucrt:onexit.obj
 0001:00014904       $unwind$?fin$0@?0???$?RV<lambda_a37b2b86f63e897a80ea819b0eb08c01>@@AEAV<lambda_38ce7e780aa69e748d6df282ebc68efe>@@V<lambda_99fb1378e971ab6e7edea83e3a7a83a2>@@@?$__crt_seh_guarded_call@H@@QEAAH$$QEAV<lambda_a37b2b86f63e897a80ea819b0eb08c01>@@AEAV<lambda_38ce7e780aa69e748d6df282ebc68efe>@@$$QEAV<lambda_99fb1378e971ab6e7edea83e3a7a83a2>@@@Z@4HA 0000000180015904     libucrt:commit.obj
 0001:00014904       $unwind$_ctrlfp$filt$0     0000000180015904     libucrt:fpctrl.obj
 0001:0001490c       $unwind$?dllmain_crt_process_detach@@YAH_N@Z 000000018001590c     LIBCMT:dll_dllmain.obj
 0001:00014944       $unwind$?dllmain_dispatch@@YAHQEAUHINSTANCE__@@KQEAX@Z 0000000180015944     LIBCMT:dll_dllmain.obj
 0001:0001496c       $unwind$?filt$0@?0??dllmain_dispatch@@YAHQEAUHINSTANCE__@@KQEAX@Z@4HA 000000018001596c     LIBCMT:dll_dllmain.obj
 0001:00014974       $unwind$?__scrt_throw_std_bad_array_new_length@@YAXXZ 0000000180015974     LIBCMT:throw_bad_alloc.obj
 0001:00014974       $unwind$_raise_exc         0000000180015974     libucrt:fpexcept.obj
 0001:00014974       $unwind$?__scrt_throw_std_bad_alloc@@YAXXZ 0000000180015974     LIBCMT:throw_bad_alloc.obj
 0001:0001497c       $unwind$__security_init_cookie 000000018001597c     LIBCMT:gs_support.obj
 0001:00014988       $unwind$__scrt_is_nonwritable_in_current_image 0000000180015988     LIBCMT:utility.obj
 0001:000149a8       $unwind$__scrt_is_nonwritable_in_current_image$filt$0 00000001800159a8     LIBCMT:utility.obj
 0001:000149b0       $unwind$_isleadbyte_l      00000001800159b0     libucrt:_wctype.obj
 0001:000149b0       $unwind$__scrt_initialize_onexit_tables 00000001800159b0     LIBCMT:utility.obj
 0001:000149b0       $unwind$__dcrt_lowio_ensure_console_output_initialized 00000001800159b0     libucrt:initcon.obj
 0001:000149b0       $unwind$?getSystemCP@@YAHH@Z 00000001800159b0     libucrt:mbctype.obj
 0001:000149b8       $unwind$_seh_filter_exe    00000001800159b8     libucrt:exception_filter.obj
 0001:000149b8       $unwind$__acrt_free_locale 00000001800159b8     libucrt:locale_refcounting.obj
 0001:000149b8       $unwind$__acrt_lowio_create_handle_array 00000001800159b8     libucrt:osfinfo.obj
 0001:000149b8       $unwind$?setSBCS@@YAXPEAU__crt_multibyte_data@@@Z 00000001800159b8     libucrt:mbctype.obj
 0001:000149b8       $unwind$__scrt_dllmain_exception_filter 00000001800159b8     LIBCMT:utility.obj
 0001:000149b8       $unwind$_recalloc_base     00000001800159b8     libucrt:recalloc.obj
 0001:000149b8       $unwind$_initterm          00000001800159b8     libucrt:initterm.obj
 0001:000149cc       $unwind$__scrt_fastfail    00000001800159cc     LIBCMT:utility_desktop.obj
 0001:000149dc       $unwind$__isa_available_init 00000001800159dc     LIBCMT:cpu_disp.obj
 0001:000149f0       $xdatasym                  00000001800159f0     LIBCMT:guard_dispatch.obj
 0001:000149f8       $xdatasym                  00000001800159f8     libvcruntime:memset.obj
 0001:00014a08       $unwind$__C_specific_handler 0000000180015a08     libvcruntime:riscchandler.obj
 0001:00014a24       $unwind$_free_osfhnd       0000000180015a24     libucrt:osfinfo.obj
 0001:00014a24       $unwind$__std_exception_copy 0000000180015a24     libvcruntime:std_exception.obj
 0001:00014a38       $unwind$_CxxThrowException 0000000180015a38     libvcruntime:throw.obj
 0001:00014a48       $xdatasym                  0000000180015a48     libvcruntime:notify.obj
 0001:00014a54       $unwind$__DestructExceptionObject 0000000180015a54     libvcruntime:ehhelpers.obj
 0001:00014a74       $unwind$__acrt_initialize_winapi_thunks 0000000180015a74     libucrt:winapi_thunks.obj
 0001:00014a74       $unwind$__vcrt_initialize_winapi_thunks 0000000180015a74     libvcruntime:winapi_downlevel.obj
 0001:00014a7c       $unwind$__vcrt_uninitialize_winapi_thunks 0000000180015a7c     libvcruntime:winapi_downlevel.obj
 0001:00014a84       $unwind$?try_get_function@@YAPEAXW4function_id@?A0x14c33c87@@QEBDQEBW4module_id@2@2@Z 0000000180015a84     libvcruntime:winapi_downlevel.obj
 0001:00014a84       $unwind$?try_get_function@@YAPEAXW4function_id@?A0x391cf84c@@QEBDQEBW4module_id@2@2@Z 0000000180015a84     libucrt:winapi_thunks.obj
 0001:00014aa0       $xdatasym                  0000000180015aa0     libvcruntime:memcpy.obj
 0001:00014ab0       $xdatasym                  0000000180015ab0     libvcruntime:handlers.obj
 0001:00014ac0       $unwind$_query_new_handler 0000000180015ac0     libucrt:new_handler.obj
 0001:00014ae0       $unwind$?common_exit@@YAXHW4_crt_exit_cleanup_mode@@W4_crt_exit_return_mode@@@Z 0000000180015ae0     libucrt:exit.obj
 0001:00014aec       $unwind$??R<lambda_6e4b09c48022b2350581041d5f6b0c4c>@@QEBA@XZ 0000000180015aec     libucrt:exit.obj
 0001:00014b0c       $unwind$??$?RV<lambda_d80eeec6fff315bfe5c115232f3240e3>@@AEAV<lambda_6e4b09c48022b2350581041d5f6b0c4c>@@V<lambda_2358e3775559c9db80273638284d5e45>@@@?$__crt_seh_guarded_call@X@@QEAAX$$QEAV<lambda_d80eeec6fff315bfe5c115232f3240e3>@@AEAV<lambda_6e4b09c48022b2350581041d5f6b0c4c>@@$$QEAV<lambda_2358e3775559c9db80273638284d5e45>@@@Z 0000000180015b0c     libucrt:exit.obj
 0001:00014b30       $unwind$_configure_narrow_argv 0000000180015b30     libucrt:argv_parsing.obj
 0001:00014b44       $unwind$??$parse_command_line@D@@YAXPEADPEAPEAD0PEA_K2@Z 0000000180015b44     libucrt:argv_parsing.obj
 0001:00014b60       $unwind$??$free_environment@D@@YAXQEAPEAD@Z 0000000180015b60     libucrt:environment_initialization.obj
 0001:00014b60       $unwind$??$free_environment@_W@@YAXQEAPEA_W@Z 0000000180015b60     libucrt:environment_initialization.obj
 0001:00014b6c       $unwind$??$create_environment@D@@YAQEAPEADQEAD@Z 0000000180015b6c     libucrt:environment_initialization.obj
 0001:00014b84       $unwind$_execute_onexit_table 0000000180015b84     libucrt:onexit.obj
 0001:00014b8c       $unwind$??R<lambda_f03950bc5685219e0bcd2087efbe011e>@@QEBAHXZ 0000000180015b8c     libucrt:onexit.obj
 0001:00014ba4       $unwind$??$?RV<lambda_7777bce6b2f8c936911f934f8298dc43>@@AEAV<lambda_f03950bc5685219e0bcd2087efbe011e>@@V<lambda_3883c3dff614d5e0c5f61bb1ac94921c>@@@?$__crt_seh_guarded_call@H@@QEAAH$$QEAV<lambda_7777bce6b2f8c936911f934f8298dc43>@@AEAV<lambda_f03950bc5685219e0bcd2087efbe011e>@@$$QEAV<lambda_3883c3dff614d5e0c5f61bb1ac94921c>@@@Z 0000000180015ba4     libucrt:onexit.obj
 0001:00014bc8       $unwind$terminate          0000000180015bc8     libucrt:terminate.obj
 0001:00014be8       $xdatasym                  0000000180015be8     libucrt:strncmp.obj
 0001:00014bec       $unwind$__acrt_locale_free_numeric 0000000180015bec     libucrt:initnum.obj
 0001:00014bec       $unwind$?destroy_fls@@YAXPEAX@Z 0000000180015bec     libucrt:per_thread_data.obj
 0001:00014bec       $unwind$__acrt_locale_free_lc_time_if_unreferenced 0000000180015bec     libucrt:locale_refcounting.obj
 0001:00014bec       $unwind$_free_base         0000000180015bec     libucrt:free_base.obj
 0001:00014bf4       $unwind$?construct_ptd_array@@YAXQEAU__acrt_ptd@@@Z 0000000180015bf4     libucrt:per_thread_data.obj
 0001:00014bfc       $unwind$?destroy_ptd_array@@YAXQEAU__acrt_ptd@@@Z 0000000180015bfc     libucrt:per_thread_data.obj
 0001:00014c04       $unwind$??$?RV<lambda_0ae27a3a962d80f24befdcbee591983d>@@AEAV<lambda_8d0ee55de4b1038c4002e0adecdf1839>@@V<lambda_dc504788e8f1664fe9b84e20bfb512f2>@@@?$__crt_seh_guarded_call@X@@QEAAX$$QEAV<lambda_0ae27a3a962d80f24befdcbee591983d>@@AEAV<lambda_8d0ee55de4b1038c4002e0adecdf1839>@@$$QEAV<lambda_dc504788e8f1664fe9b84e20bfb512f2>@@@Z 0000000180015c04     libucrt:per_thread_data.obj
 0001:00014c28       $unwind$??$?RV<lambda_aa87e3671a710a21b5dc78c0bdf72e11>@@AEAV<lambda_92619d2358a28f41a33ba319515a20b9>@@V<lambda_6992ecaafeb10aed2b74cb1fae11a551>@@@?$__crt_seh_guarded_call@X@@QEAAX$$QEAV<lambda_aa87e3671a710a21b5dc78c0bdf72e11>@@AEAV<lambda_92619d2358a28f41a33ba319515a20b9>@@$$QEAV<lambda_6992ecaafeb10aed2b74cb1fae11a551>@@@Z 0000000180015c28     libucrt:per_thread_data.obj
 0001:00014c4c       $unwind$??$?RV<lambda_f2e299630e499de9f9a165e60fcd3db5>@@AEAV<lambda_2ae9d31cdba2644fcbeaf08da7c24588>@@V<lambda_40d01ff24d0e7b3814fdbdcee8eab3c7>@@@?$__crt_seh_guarded_call@X@@QEAAX$$QEAV<lambda_f2e299630e499de9f9a165e60fcd3db5>@@AEAV<lambda_2ae9d31cdba2644fcbeaf08da7c24588>@@$$QEAV<lambda_40d01ff24d0e7b3814fdbdcee8eab3c7>@@@Z 0000000180015c4c     libucrt:per_thread_data.obj
 0001:00014c70       $unwind$??$?RV<lambda_2d41944a1d46af3157314b8a01080d33>@@AEAV<lambda_8f455de75cd7d7f24b4096f044d8b9e6>@@V<lambda_aa500f224e6afead328df44964fe2772>@@@?$__crt_seh_guarded_call@X@@QEAAX$$QEAV<lambda_2d41944a1d46af3157314b8a01080d33>@@AEAV<lambda_8f455de75cd7d7f24b4096f044d8b9e6>@@$$QEAV<lambda_aa500f224e6afead328df44964fe2772>@@@Z 0000000180015c70     libucrt:per_thread_data.obj
 0001:00014c94       $unwind$_invalid_parameter_noinfo 0000000180015c94     libucrt:invalid_parameter.obj
 0001:00014c94       $unwind$_log10_special     0000000180015c94     libucrt:log_special.obj
 0001:00014c9c       $unwind$__acrt_call_reportfault 0000000180015c9c     libucrt:invalid_parameter.obj
 0001:00014cbc       $unwind$_invalid_parameter 0000000180015cbc     libucrt:invalid_parameter.obj
 0001:00014cd0       $unwind$??$__acrt_mbs_to_wcs_cp@U__crt_win32_buffer_internal_dynamic_resizing@@@@YAHQEBDAEAV?$__crt_win32_buffer@_WU__crt_win32_buffer_internal_dynamic_resizing@@@@I@Z 0000000180015cd0     libucrt:argv_wildcards.obj
 0001:00014ce8       $unwind$??$__acrt_wcs_to_mbs_cp@U__crt_win32_buffer_internal_dynamic_resizing@@@@YAHQEB_WAEAV?$__crt_win32_buffer@DU__crt_win32_buffer_internal_dynamic_resizing@@@@I@Z 0000000180015ce8     libucrt:argv_wildcards.obj
 0001:00014ce8       $unwind$__dcrt_get_narrow_environment_from_os 0000000180015ce8     libucrt:get_environment_from_os.obj
 0001:00014d00       $unwind$??$common_expand_argv_wildcards@D@@YAHQEAPEADQEAPEAPEAD@Z 0000000180015d00     libucrt:argv_wildcards.obj
 0001:00014d18       $unwind$??$copy_and_add_argument_to_buffer@D@@YAHQEBD0_KAEAV?$argument_list@D@?A0x5f5c8891@@@Z 0000000180015d18     libucrt:argv_wildcards.obj
 0001:00014d34       $unwind$??$expand_argument_wildcards@D@@YAHQEAD0AEAV?$argument_list@D@?A0x5f5c8891@@@Z 0000000180015d34     libucrt:argv_wildcards.obj
 0001:00014d58       $unwind$__acrt_GetModuleFileNameA 0000000180015d58     libucrt:getmodulefilenamea.obj
 0001:00014d74       $unwind$??$__acrt_wcs_to_mbs_cp@U__crt_win32_buffer_no_resizing@@@@YAHQEB_WAEAV?$__crt_win32_buffer@DU__crt_win32_buffer_no_resizing@@@@I@Z 0000000180015d74     libucrt:getmodulefilenamea.obj
 0001:00014d74       $unwind$__dcrt_write_console 0000000180015d74     libucrt:initcon.obj
 0001:00014d88       $unwind$_setmbcp_nolock    0000000180015d88     libucrt:mbctype.obj
 0001:00014da8       $unwind$?update_thread_multibyte_data_internal@@YAPEAU__crt_multibyte_data@@QEAU__acrt_ptd@@QEAPEAU1@@Z 0000000180015da8     libucrt:mbctype.obj
 0001:00014dd0       $unwind$?setmbcp_internal@@YAHH_NQEAU__acrt_ptd@@QEAPEAU__crt_multibyte_data@@@Z 0000000180015dd0     libucrt:mbctype.obj
 0001:00014de0       $unwind$?setSBUpLow@@YAXPEAU__crt_multibyte_data@@@Z 0000000180015de0     libucrt:mbctype.obj
 0001:00014dfc       $unwind$??$?RV<lambda_efdfa57d1f175319df784efa44bb7b81>@@AEAV<lambda_5f0a4c1567f8adc6734073e5d1e1b35c>@@V<lambda_2e8a7d3640ea6ccb4c2413664c2db6fd>@@@?$__crt_seh_guarded_call@X@@QEAAX$$QEAV<lambda_efdfa57d1f175319df784efa44bb7b81>@@AEAV<lambda_5f0a4c1567f8adc6734073e5d1e1b35c>@@$$QEAV<lambda_2e8a7d3640ea6ccb4c2413664c2db6fd>@@@Z 0000000180015dfc     libucrt:mbctype.obj
 0001:00014e20       $unwind$?x_ismbbtype_l@@YAHPEAU__crt_locale_pointers@@IHH@Z 0000000180015e20     libucrt:ismbbyte.obj
 0001:00014e30       $unwind$__GSHandlerCheckCommon 0000000180015e30     LIBCMT:gshandler.obj
 0001:00014e30       $unwind$__acrt_WideCharToMultiByte 0000000180015e30     libucrt:widechartomultibyte.obj
 0001:00014e38       $unwind$_mbtowc_l          0000000180015e38     libucrt:mbtowc.obj
 0001:00014e38       $unwind$__acrt_LCMapStringEx 0000000180015e38     libucrt:winapi_thunks.obj
 0001:00014e4c       $unwind$__acrt_initialize_lowio 0000000180015e4c     libucrt:ioinit.obj
 0001:00014e6c       $unwind$?initialize_inherited_file_handles_nolock@@YAXXZ 0000000180015e6c     libucrt:ioinit.obj
 0001:00014e88       $unwind$__acrt_initialize_stdio 0000000180015e88     libucrt:_file.obj
 0001:00014e88       $unwind$?initialize_stdio_handles_nolock@@YAXXZ 0000000180015e88     libucrt:ioinit.obj
 0001:00014ea0       $unwind$__acrt_uninitialize_locale 0000000180015ea0     libucrt:wsetlocale.obj
 0001:00014ea0       $unwind$__acrt_get_sigabrt_handler 0000000180015ea0     libucrt:signal.obj
 0001:00014ea8       $unwind$raise              0000000180015ea8     libucrt:signal.obj
 0001:00014ee4       $unwind$??$?RV<lambda_450d765d439847d4c735a33c368b5fc0>@@AEAV<lambda_44731a7d0e6d81c3e6aa82d741081786>@@V<lambda_601a2a7da3b7a96e9554ac7215c4b07c>@@@?$__crt_seh_guarded_call@P6AXH@Z@@QEAAP6AXH@Z$$QEAV<lambda_450d765d439847d4c735a33c368b5fc0>@@AEAV<lambda_44731a7d0e6d81c3e6aa82d741081786>@@$$QEAV<lambda_601a2a7da3b7a96e9554ac7215c4b07c>@@@Z 0000000180015ee4     libucrt:signal.obj
 0001:00014f08       $unwind$?common_flush_all@@YAH_N@Z 0000000180015f08     libucrt:fflush.obj
 0001:00014f10       $unwind$??$?RV<lambda_842d9ff0dc9ef11c61343bbaebe7f885>@@AEAV<lambda_c5860995281e5c4ce005b3de8f5874ee>@@V<lambda_d90129c13df834fdcbf8d2b88dafcf2d>@@@?$__crt_seh_guarded_call@X@@QEAAX$$QEAV<lambda_842d9ff0dc9ef11c61343bbaebe7f885>@@AEAV<lambda_c5860995281e5c4ce005b3de8f5874ee>@@$$QEAV<lambda_d90129c13df834fdcbf8d2b88dafcf2d>@@@Z 0000000180015f10     libucrt:fflush.obj
 0001:00014f34       $unwind$??$?RV<lambda_886d6c58226a84441f68b9f2b8217b83>@@AEAV<lambda_ab61a845afdef5b7c387490eaf3616ee>@@V<lambda_f7f22ab5edc0698d5f6905b0d3f44752>@@@?$__crt_seh_guarded_call@X@@QEAAX$$QEAV<lambda_886d6c58226a84441f68b9f2b8217b83>@@AEAV<lambda_ab61a845afdef5b7c387490eaf3616ee>@@$$QEAV<lambda_f7f22ab5edc0698d5f6905b0d3f44752>@@@Z 0000000180015f34     libucrt:fflush.obj
 0001:00014f5c       $unwind$??$?RV<lambda_410d79af7f07d98d83a3f525b3859a53>@@AEAV<lambda_3e16ef9562a7dcce91392c22ab16ea36>@@V<lambda_38119f0e861e05405d8a144b9b982f0a>@@@?$__crt_seh_guarded_call@X@@QEAAX$$QEAV<lambda_410d79af7f07d98d83a3f525b3859a53>@@AEAV<lambda_3e16ef9562a7dcce91392c22ab16ea36>@@$$QEAV<lambda_38119f0e861e05405d8a144b9b982f0a>@@@Z 0000000180015f5c     libucrt:wsetlocale.obj
 0001:00014f84       $unwind$__acrt_update_thread_locale_data 0000000180015f84     libucrt:locale_refcounting.obj
 0001:00014fa8       $unwind$qsort              0000000180015fa8     libucrt:qsort.obj
 0001:00014fc0       $chain$4$qsort             0000000180015fc0     libucrt:qsort.obj
 0001:00014fe4       $chain$5$qsort             0000000180015fe4     libucrt:qsort.obj
 0001:00014ff4       $unwind$strpbrk            0000000180015ff4     libucrt:strpbrk.obj
 0001:00015004       $unwind$fallbackMethod     0000000180016004     libucrt:strpbrk.obj
 0001:00015014       $unwind$_mbsdec_l          0000000180016014     libucrt:mbsdec.obj
 0001:00015020       $unwind$__acrt_GetStringTypeA 0000000180016020     libucrt:getstringtypea.obj
 0001:00015048       $unwind$__acrt_LCMapStringA 0000000180016048     libucrt:lcmapstringa.obj
 0001:00015058       $unwind$?__acrt_LCMapStringA_stat@@YAHPEAU__crt_locale_pointers@@PEB_WKPEBDHPEADHHH@Z 0000000180016058     libucrt:lcmapstringa.obj
 0001:00015080       $unwind$?GetTableIndexFromLocaleName@@YAHPEB_W@Z 0000000180016080     libucrt:lcidtoname_downlevel.obj
 0001:00015098       $unwind$__acrt_lowio_destroy_handle_array 0000000180016098     libucrt:osfinfo.obj
 0001:000150a8       $unwind$__acrt_lowio_ensure_fh_exists 00000001800160a8     libucrt:osfinfo.obj
 0001:000150d4       $unwind$_close             00000001800160d4     libucrt:close.obj
 0001:000150d4       $unwind$_commit            00000001800160d4     libucrt:commit.obj
 0001:000150dc       $unwind$??$?RV<lambda_a37b2b86f63e897a80ea819b0eb08c01>@@AEAV<lambda_38ce7e780aa69e748d6df282ebc68efe>@@V<lambda_99fb1378e971ab6e7edea83e3a7a83a2>@@@?$__crt_seh_guarded_call@H@@QEAAH$$QEAV<lambda_a37b2b86f63e897a80ea819b0eb08c01>@@AEAV<lambda_38ce7e780aa69e748d6df282ebc68efe>@@$$QEAV<lambda_99fb1378e971ab6e7edea83e3a7a83a2>@@@Z 00000001800160dc     libucrt:commit.obj
 0001:00015100       $unwind$_write             0000000180016100     libucrt:write.obj
 0001:00015130       $unwind$_write_nolock      0000000180016130     libucrt:write.obj
 0001:00015148       $unwind$?write_double_translated_ansi_nolock@@YA?AUwrite_result@?A0x17268360@@HQEBDI@Z 0000000180016148     libucrt:write.obj
 0001:0001516c       $unwind$?write_text_utf16le_nolock@@YA?AUwrite_result@?A0x17268360@@HQEBDI@Z 000000018001616c     libucrt:write.obj
 0001:0001516c       $unwind$?write_text_ansi_nolock@@YA?AUwrite_result@?A0x17268360@@HQEBDI@Z 000000018001616c     libucrt:write.obj
 0001:0001518c       $unwind$?write_text_utf8_nolock@@YA?AUwrite_result@?A0x17268360@@HQEBDI@Z 000000018001618c     libucrt:write.obj
 0001:000151b0       $unwind$_fcloseall         00000001800161b0     libucrt:closeall.obj
 0001:000151d4       $unwind$?__mbrtowc_utf8@__crt_mbstring@@YA_KPEA_WPEBD_KPEAU_Mbstatet@@@Z 00000001800161d4     libucrt:mbrtowc.obj
 0001:000151dc       $unwind$?__mbsrtowcs_utf8@__crt_mbstring@@YA_KPEA_WPEAPEBD_KPEAU_Mbstatet@@@Z 00000001800161dc     libucrt:mbrtowc.obj
 0001:000151f4       $unwind$__acrt_locale_free_monetary 00000001800161f4     libucrt:initmon.obj
 0001:000151fc       $unwind$__acrt_locale_free_time 00000001800161fc     libucrt:inittime.obj
 0001:0001520c       $unwind$_putwch_nolock     000000018001620c     libucrt:putwch.obj
 0001:00015214       $unwind$fclose             0000000180016214     libucrt:fclose.obj
 0001:00015238       $unwind$?__mbrtoc32_utf8@__crt_mbstring@@YA_KPEA_UPEBD_KPEAU_Mbstatet@@@Z 0000000180016238     libucrt:mbrtoc32.obj
 0001:00015258       $xdatasym                  0000000180016258     libucrt:log10.obj
 0001:00015264       $unwind$??$?RV<lambda_751a882b2c74d4b022dec766aa51a29a>@@AEAV<lambda_628dfdc04ba53c8bfc02c9951375f3f5>@@V<lambda_f6c7be5f7998530c34de24c7437d6b54>@@@?$__crt_seh_guarded_call@H@@QEAAH$$QEAV<lambda_751a882b2c74d4b022dec766aa51a29a>@@AEAV<lambda_628dfdc04ba53c8bfc02c9951375f3f5>@@$$QEAV<lambda_f6c7be5f7998530c34de24c7437d6b54>@@@Z 0000000180016264     libucrt:close.obj
 0001:00015288       $unwind$_call_matherr      0000000180016288     libucrt:libm_error.obj
 0001:00015290       $unwind$_handle_error      0000000180016290     libucrt:libm_error.obj
 0001:000152b0       $unwind$__acrt_initialize_fma3 00000001800162b0     libucrt:fma3_available.obj
 0001:000152b8       $unwind$_log_special_common 00000001800162b8     libucrt:log_special.obj
 0001:000152c8       $xdatasym                  00000001800162c8     libucrt:fpsr.obj
 0001:000152d0       $unwind$_raise_exc_ex      00000001800162d0     libucrt:fpexcept.obj
 0001:000152e4       $unwind$_ctrlfp            00000001800162e4     libucrt:fpctrl.obj
 0001:0001530c       $unwind$_IsNonwritableInCurrentImage 000000018001630c     LIBCMT:pesect.obj
 0001:00015330       $xdatasym                  0000000180016330     LIBCMT:amdsecgs.obj
 0001:00015334       $unwind$__report_securityfailure 0000000180016334     LIBCMT:gs_report.obj
 0001:0001533c       $unwind$__report_gsfailure 000000018001633c     LIBCMT:gs_report.obj
 0001:00015344       $unwind$capture_current_context 0000000180016344     LIBCMT:gs_report.obj
 0001:00015350       $unwind$capture_previous_context 0000000180016350     LIBCMT:gs_report.obj
 0001:00015360       $xdatasym                  0000000180016360     libvcruntime:memcmp.obj
 0001:00015460       .edata                     0000000180016460     SameFolder.exp
 0001:00015488       rgpv                       0000000180016488     SameFolder.exp
 0001:0001549c       rgszName                   000000018001649c     SameFolder.exp
 0001:000154b0       rgwOrd                     00000001800164b0     SameFolder.exp
 0001:000154ba       szName                     00000001800164ba     SameFolder.exp
 0001:000154c9       $N00001                    00000001800164c9     SameFolder.exp
 0001:000154d4       $N00002                    00000001800164d4     SameFolder.exp
 0001:000154e3       $N00003                    00000001800164e3     SameFolder.exp
 0001:000154f2       $N00004                    00000001800164f2     SameFolder.exp
 0001:000154f8       $N00005                    00000001800164f8     SameFolder.exp
 0002:00000040       ?__vcrt_flsindex@@3KA      0000000180017040     libvcruntime:per_thread_data.obj
 0002:00000054       ?__acrt_flsindex@@3KA      0000000180017054     libucrt:per_thread_data.obj
 0002:00000058       ?errno_no_memory@@3HA      0000000180017058     libucrt:errno.obj
 0002:0000005c       ?doserrno_no_memory@@3KA   000000018001705c     libucrt:errno.obj
 0002:00000060       _mbctypes                  0000000180017060     libucrt:mbctype.obj
 0002:00000170       _mbcasemaps                0000000180017170     libucrt:mbctype.obj
 0002:00000270       ?__rgctypeflag@@3PADA      0000000180017270     libucrt:mbctype.obj
 0002:00000280       ?__rgcode_page_info@@3PAUcode_page_info@@A 0000000180017280     libucrt:mbctype.obj
 0002:000009c0       ?__dcrt_lowio_console_output_handle@@3PEAXEA 00000001800179c0     libucrt:initcon.obj
 0002:000009d0       ?dazSupported@?1??_ctrlfp@@9@9 00000001800179d0     libucrt:fpctrl.obj
 0002:00000d38       ?PluginMenuStrings@?1??GetPluginInfoW@@9@4PAPEB_WA 0000000180017d38     SameFolder.obj
 0002:00000d40       ?PluginConfigStrings@?1??GetPluginInfoW@@9@4PAPEB_WA 0000000180017d40     SameFolder.obj
 0002:00000d48       ?DiskMenuStrings@?1??GetPluginInfoW@@9@4PAPEB_WA 0000000180017d48     SameFolder.obj
 0002:00000d50       ?__proc_attached@@3HA      0000000180017d50     LIBCMT:dll_dllmain.obj
 0002:00000d90       ?is_initialized_as_dll@@3_NA 0000000180017d90     LIBCMT:utility.obj
 0002:00000d91       ?module_local_atexit_table_initialized@@3_NA 0000000180017d91     LIBCMT:utility.obj
 0002:00000d98       ?module_local_atexit_table@@3U_onexit_table_t@@A 0000000180017d98     LIBCMT:utility.obj
 0002:00000db0       ?module_local_at_quick_exit_table@@3U_onexit_table_t@@A 0000000180017db0     LIBCMT:utility.obj
 0002:00000e18       ?heap@@3V_HeapManager@@A   0000000180017e18     libvcruntime:undname.obj
 0002:00000e40       ?__vcrt_startup_thread_ptd@@3U__vcrt_ptd@@A 0000000180017e40     libvcruntime:per_thread_data.obj
 0002:00000ed0       __vcrt_lock_table          0000000180017ed0     libvcruntime:locks.obj
 0002:00000ef8       __vcrt_locks_initialized   0000000180017ef8     libvcruntime:locks.obj
 0002:00000f00       ?module_handles@@3PAPEAUHINSTANCE__@@A 0000000180017f00     libvcruntime:winapi_downlevel.obj
 0002:00000f18       ?encoded_function_pointers@@3PAPEAXA 0000000180017f18     libvcruntime:winapi_downlevel.obj
 0002:00000f48       ?__acrt_new_handler@@3V?$dual_state_global@P6AH_K@Z@__crt_state_management@@A 0000000180017f48     libucrt:new_handler.obj
 0002:00000f50       ?c_termination_complete@@3JA 0000000180017f50     libucrt:exit.obj
 0002:00000f58       ?thread_local_exit_callback_func@@3P6AXPEAXK0@ZEA 0000000180017f58     libucrt:exit.obj
 0002:00000f70       ?program_name@?1???$common_configure_argv@D@@YAHW4_crt_argv_mode@@@Z@4PADA 0000000180017f70     libucrt:argv_parsing.obj
 0002:000010d0       ?__acrt_lock_table@@3PAU_RTL_CRITICAL_SECTION@@A 00000001800180d0     libucrt:locks.obj
 0002:00001300       ?__acrt_locks_initialized@@3IA 0000000180018300     libucrt:locks.obj
 0002:00001308       ?__acrt_invalid_parameter_handler@@3V?$dual_state_global@P6AXPEB_W00I_K@Z@__crt_state_management@@A 0000000180018308     libucrt:invalid_parameter.obj
 0002:00001328       ?fSystemSet@@3HA           0000000180018328     libucrt:mbctype.obj
 0002:0000132c       ?initialized@?1??__acrt_initialize_multibyte@@9@4_NA 000000018001832c     libucrt:mbctype.obj
 0002:00001360       ?module_handles@@3PAPEAUHINSTANCE__@@A 0000000180018360     libucrt:winapi_thunks.obj
 0002:00001400       ?encoded_function_pointers@@3PAPEAXA 0000000180018400     libucrt:winapi_thunks.obj
 0002:00001928       ?ctrlc_action@@3V?$dual_state_global@P6AXH@Z@__crt_state_management@@A 0000000180018928     libucrt:signal.obj
 0002:00001930       ?ctrlbreak_action@@3V?$dual_state_global@P6AXH@Z@__crt_state_management@@A 0000000180018930     libucrt:signal.obj
 0002:00001938       ?abort_action@@3V?$dual_state_global@P6AXH@Z@__crt_state_management@@A 0000000180018938     libucrt:signal.obj
 0002:00001940       ?term_action@@3V?$dual_state_global@P6AXH@Z@__crt_state_management@@A 0000000180018940     libucrt:signal.obj
 0002:00001948       ?user_matherr@@3V?$dual_state_global@P6AHPEAU_exception@@@Z@__crt_state_management@@A 0000000180018948     libucrt:matherr.obj
 0002:00001978       ?internal_state@?1??_mbtowc_l@@9@4U_Mbstatet@@A 0000000180018978     libucrt:mbtowc.obj
 0002:00001984       ?__acrt_global_new_mode@@3V?$dual_state_global@J@__crt_state_management@@A 0000000180018984     libucrt:new_mode.obj
 0002:00001990       ?__acrt_app_type@@3W4_crt_app_type@@A 0000000180018990     libucrt:report_runtime_error.obj
 0002:00001998       ?internal_pst@?1??__mbrtoc32_utf8@__crt_mbstring@@YA_KPEA_UPEBD_KPEAU_Mbstatet@@@Z@4U3@A 0000000180018998     libucrt:mbrtoc32.obj
 0002:000019b0       GS_ExceptionRecord         00000001800189b0     LIBCMT:gs_report.obj
 0002:00001a50       GS_ContextRecord           0000000180018a50     LIBCMT:gs_report.obj
 0003:0000000c       $pdata$??1?$DialogBuilderBase@UFarDialogItem@@@@MEAA@XZ 000000018001900c     SameFolder.obj
 0003:00000018       $pdata$0$??1?$DialogBuilderBase@UFarDialogItem@@@@MEAA@XZ 0000000180019018     SameFolder.obj
 0003:00000024       $pdata$1$??1?$DialogBuilderBase@UFarDialogItem@@@@MEAA@XZ 0000000180019024     SameFolder.obj
 0003:00000030       $pdata$??_G?$DialogBuilderBase@UFarDialogItem@@@@MEAAPEAXI@Z 0000000180019030     SameFolder.obj
 0003:0000003c       $pdata$??_G?$DialogItemBinding@UFarDialogItem@@@@UEAAPEAXI@Z 000000018001903c     SameFolder.obj
 0003:00000048       $pdata$??_GPluginCheckBoxBinding@@UEAAPEAXI@Z 0000000180019048     SameFolder.obj
 0003:00000054       $pdata$??_GPluginDialogBuilder@@UEAAPEAXI@Z 0000000180019054     SameFolder.obj
 0003:00000060       $pdata$??_GPluginUIntEditFieldBinding@@UEAAPEAXI@Z 0000000180019060     SameFolder.obj
 0003:00000060       $pdata$??_GPluginIntEditFieldBinding@@UEAAPEAXI@Z 0000000180019060     SameFolder.obj
 0003:0000006c       $pdata$??_GPluginRadioButtonBinding@@UEAAPEAXI@Z 000000018001906c     SameFolder.obj
 0003:00000078       $pdata$?AddButtons@?$DialogBuilderBase@UFarDialogItem@@@@QEAAXHPEBHHH@Z 0000000180019078     SameFolder.obj
 0003:00000084       $pdata$4$?AddButtons@?$DialogBuilderBase@UFarDialogItem@@@@QEAAXHPEBHHH@Z 0000000180019084     SameFolder.obj
 0003:00000090       $pdata$5$?AddButtons@?$DialogBuilderBase@UFarDialogItem@@@@QEAAXHPEBHHH@Z 0000000180019090     SameFolder.obj
 0003:0000009c       $pdata$?AddDialogItem@?$DialogBuilderBase@UFarDialogItem@@@@IEAAPEAUFarDialogItem@@W4FARDIALOGITEMTYPES@@PEB_W@Z 000000018001909c     SameFolder.obj
 0003:000000a8       $pdata$?AddIntEditField@PluginDialogBuilder@@UEAAPEAUFarDialogItem@@PEAHH@Z 00000001800190a8     SameFolder.obj
 0003:000000b4       $pdata$?AddUIntEditField@PluginDialogBuilder@@UEAAPEAUFarDialogItem@@PEAIH@Z 00000001800190b4     SameFolder.obj
 0003:000000c0       $pdata$?CreateCheckBoxBinding@PluginDialogBuilder@@MEAAPEAU?$DialogItemBinding@UFarDialogItem@@@@PEAHH@Z 00000001800190c0     SameFolder.obj
 0003:000000cc       $pdata$?CreateRadioButtonBinding@PluginDialogBuilder@@MEAAPEAU?$DialogItemBinding@UFarDialogItem@@@@PEAH@Z 00000001800190cc     SameFolder.obj
 0003:000000d8       $pdata$?DoShowDialog@PluginDialogBuilder@@MEAA_JXZ 00000001800190d8     SameFolder.obj
 0003:000000e4       $pdata$?InitDialogItem@PluginDialogBuilder@@MEAAXPEAUFarDialogItem@@PEB_W@Z 00000001800190e4     SameFolder.obj
 0003:000000f0       $pdata$?SaveValue@PluginCheckBoxBinding@@UEAAXPEAUFarDialogItem@@H@Z 00000001800190f0     SameFolder.obj
 0003:000000fc       $pdata$?SaveValue@PluginIntEditFieldBinding@@UEAAXPEAUFarDialogItem@@H@Z 00000001800190fc     SameFolder.obj
 0003:00000108       $pdata$?SaveValue@PluginRadioButtonBinding@@UEAAXPEAUFarDialogItem@@H@Z 0000000180019108     SameFolder.obj
 0003:00000114       $pdata$?SaveValue@PluginUIntEditFieldBinding@@UEAAXPEAUFarDialogItem@@H@Z 0000000180019114     SameFolder.obj
 0003:00000120       $pdata$?UpdateBorderSize@?$DialogBuilderBase@UFarDialogItem@@@@IEAAXXZ 0000000180019120     SameFolder.obj
 0003:0000012c       $pdata$1$?UpdateBorderSize@?$DialogBuilderBase@UFarDialogItem@@@@IEAAXXZ 000000018001912c     SameFolder.obj
 0003:00000138       $pdata$2$?UpdateBorderSize@?$DialogBuilderBase@UFarDialogItem@@@@IEAAXXZ 0000000180019138     SameFolder.obj
 0003:00000144       $pdata$3$?UpdateBorderSize@?$DialogBuilderBase@UFarDialogItem@@@@IEAAXXZ 0000000180019144     SameFolder.obj
 0003:00000150       $pdata$4$?UpdateBorderSize@?$DialogBuilderBase@UFarDialogItem@@@@IEAAXXZ 0000000180019150     SameFolder.obj
 0003:0000015c       $pdata$ConfigureW          000000018001915c     SameFolder.obj
 0003:00000168       $pdata$2$ConfigureW        0000000180019168     SameFolder.obj
 0003:00000174       $pdata$3$ConfigureW        0000000180019174     SameFolder.obj
 0003:00000180       $pdata$4$ConfigureW        0000000180019180     SameFolder.obj
 0003:0000018c       $pdata$5$ConfigureW        000000018001918c     SameFolder.obj
 0003:00000198       $pdata$GetGlobalInfoW      0000000180019198     SameFolder.obj
 0003:000001a4       $pdata$GetPluginInfoW      00000001800191a4     SameFolder.obj
 0003:000001b0       $pdata$OpenW               00000001800191b0     SameFolder.obj
 0003:000001bc       $pdata$0$OpenW             00000001800191bc     SameFolder.obj
 0003:000001c8       $pdata$2$OpenW             00000001800191c8     SameFolder.obj
 0003:000001d4       $pdata$3$OpenW             00000001800191d4     SameFolder.obj
 0003:000001e0       $pdata$5$OpenW             00000001800191e0     SameFolder.obj
 0003:000001ec       $pdata$6$OpenW             00000001800191ec     SameFolder.obj
 0003:000001f8       $pdata$SetStartupInfoW     00000001800191f8     SameFolder.obj
 0003:00000204       $pdata$??2@YAPEAX_K@Z      0000000180019204     LIBCMT:new_scalar.obj
 0003:00000210       $pdata$?dllmain_crt_dispatch@@YAHQEAUHINSTANCE__@@KQEAX@Z 0000000180019210     LIBCMT:dll_dllmain.obj
 0003:0000021c       $pdata$?dllmain_crt_process_attach@@YAHQEAUHINSTANCE__@@QEAX@Z 000000018001921c     LIBCMT:dll_dllmain.obj
 0003:00000228       $pdata$?dllmain_crt_process_detach@@YAH_N@Z 0000000180019228     LIBCMT:dll_dllmain.obj
 0003:00000234       $pdata$?dllmain_dispatch@@YAHQEAUHINSTANCE__@@KQEAX@Z 0000000180019234     LIBCMT:dll_dllmain.obj
 0003:00000240       $pdata$_DllMainCRTStartup  0000000180019240     LIBCMT:dll_dllmain.obj
 0003:0000024c       $pdata$??0bad_alloc@std@@QEAA@AEBV01@@Z 000000018001924c     LIBCMT:throw_bad_alloc.obj
 0003:00000258       $pdata$??0bad_array_new_length@std@@QEAA@AEBV01@@Z 0000000180019258     LIBCMT:throw_bad_alloc.obj
 0003:00000264       $pdata$??0exception@std@@QEAA@AEBV01@@Z 0000000180019264     LIBCMT:throw_bad_alloc.obj
 0003:00000270       $pdata$??_Gbad_array_new_length@std@@UEAAPEAXI@Z 0000000180019270     LIBCMT:throw_bad_alloc.obj
 0003:00000270       $pdata$??_Gbad_alloc@std@@UEAAPEAXI@Z 0000000180019270     LIBCMT:throw_bad_alloc.obj
 0003:00000270       $pdata$??_Gexception@std@@UEAAPEAXI@Z 0000000180019270     LIBCMT:throw_bad_alloc.obj
 0003:0000027c       $pdata$?__scrt_throw_std_bad_alloc@@YAXXZ 000000018001927c     LIBCMT:throw_bad_alloc.obj
 0003:00000288       $pdata$?__scrt_throw_std_bad_array_new_length@@YAXXZ 0000000180019288     LIBCMT:throw_bad_alloc.obj
 0003:00000294       $pdata$__security_init_cookie 0000000180019294     LIBCMT:gs_support.obj
 0003:000002a0       $pdata$__scrt_initialize_default_local_stdio_options 00000001800192a0     LIBCMT:default_local_stdio_options.obj
 0003:000002ac       $pdata$__scrt_acquire_startup_lock 00000001800192ac     LIBCMT:utility.obj
 0003:000002b8       $pdata$__scrt_dllmain_after_initialize_c 00000001800192b8     LIBCMT:utility.obj
 0003:000002c4       $pdata$__scrt_dllmain_before_initialize_c 00000001800192c4     LIBCMT:utility.obj
 0003:000002d0       $pdata$__scrt_dllmain_crt_thread_attach 00000001800192d0     LIBCMT:utility.obj
 0003:000002dc       $pdata$__scrt_dllmain_crt_thread_detach 00000001800192dc     LIBCMT:utility.obj
 0003:000002e8       $pdata$__scrt_dllmain_exception_filter 00000001800192e8     LIBCMT:utility.obj
 0003:000002f4       $pdata$__scrt_dllmain_uninitialize_c 00000001800192f4     LIBCMT:utility.obj
 0003:00000300       $pdata$__scrt_dllmain_uninitialize_critical 0000000180019300     LIBCMT:utility.obj
 0003:0000030c       $pdata$__scrt_initialize_crt 000000018001930c     LIBCMT:utility.obj
 0003:00000318       $pdata$__scrt_initialize_onexit_tables 0000000180019318     LIBCMT:utility.obj
 0003:00000324       $pdata$__scrt_is_nonwritable_in_current_image 0000000180019324     LIBCMT:utility.obj
 0003:00000330       $pdata$__scrt_release_startup_lock 0000000180019330     LIBCMT:utility.obj
 0003:0000033c       $pdata$__scrt_uninitialize_crt 000000018001933c     LIBCMT:utility.obj
 0003:00000348       $pdata$__scrt_fastfail     0000000180019348     LIBCMT:utility_desktop.obj
 0003:00000354       $pdata$_RTC_Initialize     0000000180019354     LIBCMT:initsect.obj
 0003:00000360       $pdata$_RTC_Terminate      0000000180019360     LIBCMT:initsect.obj
 0003:0000036c       $pdata$??_Gtype_info@@UEAAPEAXI@Z 000000018001936c     LIBCMT:std_type_info_static.obj
 0003:00000378       $pdata$__isa_available_init 0000000180019378     LIBCMT:cpu_disp.obj
 0003:0000039c       $pdata$__C_specific_handler 000000018001939c     libvcruntime:riscchandler.obj
 0003:000003a8       $pdata$__std_exception_copy 00000001800193a8     libvcruntime:std_exception.obj
 0003:000003b4       $pdata$__std_exception_destroy 00000001800193b4     libvcruntime:std_exception.obj
 0003:000003c0       $pdata$_CxxThrowException  00000001800193c0     libvcruntime:throw.obj
 0003:000003cc       $pdata$__std_type_info_destroy_list 00000001800193cc     libvcruntime:std_type_info.obj
 0003:000003d8       $pdata$__vcrt_initialize   00000001800193d8     libvcruntime:initialization.obj
 0003:000003e4       $pdata$__vcrt_thread_attach 00000001800193e4     libvcruntime:initialization.obj
 0003:000003f0       $pdata$__vcrt_thread_detach 00000001800193f0     libvcruntime:initialization.obj
 0003:000003fc       $pdata$__vcrt_uninitialize 00000001800193fc     libvcruntime:initialization.obj
 0003:00000408       $pdata$__vcrt_uninitialize_critical 0000000180019408     libvcruntime:initialization.obj
 0003:00000438       $pdata$__DestructExceptionObject 0000000180019438     libvcruntime:ehhelpers.obj
 0003:00000444       $pdata$__vcrt_freefls      0000000180019444     libvcruntime:per_thread_data.obj
 0003:00000450       $pdata$__vcrt_freeptd      0000000180019450     libvcruntime:per_thread_data.obj
 0003:0000045c       $pdata$__vcrt_getptd_noexit 000000018001945c     libvcruntime:per_thread_data.obj
 0003:00000468       $pdata$__vcrt_initialize_ptd 0000000180019468     libvcruntime:per_thread_data.obj
 0003:00000474       $pdata$__vcrt_uninitialize_ptd 0000000180019474     libvcruntime:per_thread_data.obj
 0003:00000480       $pdata$__vcrt_initialize_locks 0000000180019480     libvcruntime:locks.obj
 0003:0000048c       $pdata$__vcrt_uninitialize_locks 000000018001948c     libvcruntime:locks.obj
 0003:00000498       $pdata$?try_get_function@@YAPEAXW4function_id@?A0x14c33c87@@QEBDQEBW4module_id@2@2@Z 0000000180019498     libvcruntime:winapi_downlevel.obj
 0003:000004a4       $pdata$__vcrt_FlsAlloc     00000001800194a4     libvcruntime:winapi_downlevel.obj
 0003:000004b0       $pdata$__vcrt_FlsFree      00000001800194b0     libvcruntime:winapi_downlevel.obj
 0003:000004bc       $pdata$__vcrt_FlsGetValue  00000001800194bc     libvcruntime:winapi_downlevel.obj
 0003:000004c8       $pdata$__vcrt_FlsSetValue  00000001800194c8     libvcruntime:winapi_downlevel.obj
 0003:000004d4       $pdata$__vcrt_InitializeCriticalSectionEx 00000001800194d4     libvcruntime:winapi_downlevel.obj
 0003:000004e0       $pdata$__vcrt_initialize_winapi_thunks 00000001800194e0     libvcruntime:winapi_downlevel.obj
 0003:000004ec       $pdata$__vcrt_uninitialize_winapi_thunks 00000001800194ec     libvcruntime:winapi_downlevel.obj
 0003:00000528       $pdata$_callnewh           0000000180019528     libucrt:new_handler.obj
 0003:00000534       $pdata$_query_new_handler  0000000180019534     libucrt:new_handler.obj
 0003:00000540       $pdata$_initterm           0000000180019540     libucrt:initterm.obj
 0003:0000054c       $pdata$_initterm_e         000000018001954c     libucrt:initterm.obj
 0003:00000558       $pdata$_seh_filter_exe     0000000180019558     libucrt:exception_filter.obj
 0003:00000564       $pdata$??$?RV<lambda_d80eeec6fff315bfe5c115232f3240e3>@@AEAV<lambda_6e4b09c48022b2350581041d5f6b0c4c>@@V<lambda_2358e3775559c9db80273638284d5e45>@@@?$__crt_seh_guarded_call@X@@QEAAX$$QEAV<lambda_d80eeec6fff315bfe5c115232f3240e3>@@AEAV<lambda_6e4b09c48022b2350581041d5f6b0c4c>@@$$QEAV<lambda_2358e3775559c9db80273638284d5e45>@@@Z 0000000180019564     libucrt:exit.obj
 0003:00000570       $pdata$??R<lambda_6e4b09c48022b2350581041d5f6b0c4c>@@QEBA@XZ 0000000180019570     libucrt:exit.obj
 0003:0000057c       $pdata$?common_exit@@YAXHW4_crt_exit_cleanup_mode@@W4_crt_exit_return_mode@@@Z 000000018001957c     libucrt:exit.obj
 0003:00000588       $pdata$?exit_or_terminate_process@@YAXI@Z 0000000180019588     libucrt:exit.obj
 0003:00000594       $pdata$?try_cor_exit_process@@YAXI@Z 0000000180019594     libucrt:exit.obj
 0003:000005a0       $pdata$??$parse_command_line@D@@YAXPEADPEAPEAD0PEA_K2@Z 00000001800195a0     libucrt:argv_parsing.obj
 0003:000005ac       $pdata$__acrt_allocate_buffer_for_argv 00000001800195ac     libucrt:argv_parsing.obj
 0003:000005b8       $pdata$_configure_narrow_argv 00000001800195b8     libucrt:argv_parsing.obj
 0003:000005c4       $pdata$??$common_initialize_environment_nolock@D@@YAHXZ 00000001800195c4     libucrt:environment_initialization.obj
 0003:000005d0       $pdata$??$create_environment@D@@YAQEAPEADQEAD@Z 00000001800195d0     libucrt:environment_initialization.obj
 0003:000005dc       $pdata$??$free_environment@_W@@YAXQEAPEA_W@Z 00000001800195dc     libucrt:environment_initialization.obj
 0003:000005dc       $pdata$??$free_environment@D@@YAXQEAPEAD@Z 00000001800195dc     libucrt:environment_initialization.obj
 0003:000005e8       $pdata$??$uninitialize_environment_internal@D@@YAXAEAPEAPEAD@Z 00000001800195e8     libucrt:environment_initialization.obj
 0003:000005f4       $pdata$??$uninitialize_environment_internal@_W@@YAXAEAPEAPEA_W@Z 00000001800195f4     libucrt:environment_initialization.obj
 0003:00000600       $pdata$__dcrt_uninitialize_environments_nolock 0000000180019600     libucrt:environment_initialization.obj
 0003:0000060c       $pdata$??$?RV<lambda_7777bce6b2f8c936911f934f8298dc43>@@AEAV<lambda_f03950bc5685219e0bcd2087efbe011e>@@V<lambda_3883c3dff614d5e0c5f61bb1ac94921c>@@@?$__crt_seh_guarded_call@H@@QEAAH$$QEAV<lambda_7777bce6b2f8c936911f934f8298dc43>@@AEAV<lambda_f03950bc5685219e0bcd2087efbe011e>@@$$QEAV<lambda_3883c3dff614d5e0c5f61bb1ac94921c>@@@Z 000000018001960c     libucrt:onexit.obj
 0003:00000618       $pdata$??R<lambda_f03950bc5685219e0bcd2087efbe011e>@@QEBAHXZ 0000000180019618     libucrt:onexit.obj
 0003:00000624       $pdata$_execute_onexit_table 0000000180019624     libucrt:onexit.obj
 0003:00000630       $pdata$initialize_c        0000000180019630     libucrt:initialization.obj
 0003:0000063c       $pdata$uninitialize_environment 000000018001963c     libucrt:initialization.obj
 0003:00000648       $pdata$initialize_pointers 0000000180019648     libucrt:initialization.obj
 0003:00000654       $pdata$uninitialize_allocated_memory 0000000180019654     libucrt:initialization.obj
 0003:00000660       $pdata$uninitialize_allocated_io_buffers 0000000180019660     libucrt:initialization.obj
 0003:0000066c       $pdata$__acrt_thread_attach 000000018001966c     libucrt:initialization.obj
 0003:00000678       $pdata$__acrt_thread_detach 0000000180019678     libucrt:initialization.obj
 0003:00000684       $pdata$__acrt_uninitialize 0000000180019684     libucrt:initialization.obj
 0003:00000690       $pdata$__acrt_uninitialize_critical 0000000180019690     libucrt:initialization.obj
 0003:0000069c       $pdata$terminate           000000018001969c     libucrt:terminate.obj
 0003:000006a8       $pdata$strcpy_s            00000001800196a8     libucrt:strcpy_s.obj
 0003:000006b4       $pdata$??0_LocaleUpdate@@QEAA@QEAU__crt_locale_pointers@@@Z 00000001800196b4     libucrt:output.obj
 0003:000006cc       $pdata$abort               00000001800196cc     libucrt:abort.obj
 0003:000006d8       $pdata$_free_base          00000001800196d8     libucrt:free_base.obj
 0003:000006e4       $pdata$_malloc_base        00000001800196e4     libucrt:malloc_base.obj
 0003:000006f0       $pdata$__acrt_initialize_locks 00000001800196f0     libucrt:locks.obj
 0003:000006fc       $pdata$__acrt_uninitialize_locks 00000001800196fc     libucrt:locks.obj
 0003:00000708       $pdata$??$?RV<lambda_0ae27a3a962d80f24befdcbee591983d>@@AEAV<lambda_8d0ee55de4b1038c4002e0adecdf1839>@@V<lambda_dc504788e8f1664fe9b84e20bfb512f2>@@@?$__crt_seh_guarded_call@X@@QEAAX$$QEAV<lambda_0ae27a3a962d80f24befdcbee591983d>@@AEAV<lambda_8d0ee55de4b1038c4002e0adecdf1839>@@$$QEAV<lambda_dc504788e8f1664fe9b84e20bfb512f2>@@@Z 0000000180019708     libucrt:per_thread_data.obj
 0003:00000714       $pdata$??$?RV<lambda_2d41944a1d46af3157314b8a01080d33>@@AEAV<lambda_8f455de75cd7d7f24b4096f044d8b9e6>@@V<lambda_aa500f224e6afead328df44964fe2772>@@@?$__crt_seh_guarded_call@X@@QEAAX$$QEAV<lambda_2d41944a1d46af3157314b8a01080d33>@@AEAV<lambda_8f455de75cd7d7f24b4096f044d8b9e6>@@$$QEAV<lambda_aa500f224e6afead328df44964fe2772>@@@Z 0000000180019714     libucrt:per_thread_data.obj
 0003:00000720       $pdata$??$?RV<lambda_aa87e3671a710a21b5dc78c0bdf72e11>@@AEAV<lambda_92619d2358a28f41a33ba319515a20b9>@@V<lambda_6992ecaafeb10aed2b74cb1fae11a551>@@@?$__crt_seh_guarded_call@X@@QEAAX$$QEAV<lambda_aa87e3671a710a21b5dc78c0bdf72e11>@@AEAV<lambda_92619d2358a28f41a33ba319515a20b9>@@$$QEAV<lambda_6992ecaafeb10aed2b74cb1fae11a551>@@@Z 0000000180019720     libucrt:per_thread_data.obj
 0003:0000072c       $pdata$??$?RV<lambda_f2e299630e499de9f9a165e60fcd3db5>@@AEAV<lambda_2ae9d31cdba2644fcbeaf08da7c24588>@@V<lambda_40d01ff24d0e7b3814fdbdcee8eab3c7>@@@?$__crt_seh_guarded_call@X@@QEAAX$$QEAV<lambda_f2e299630e499de9f9a165e60fcd3db5>@@AEAV<lambda_2ae9d31cdba2644fcbeaf08da7c24588>@@$$QEAV<lambda_40d01ff24d0e7b3814fdbdcee8eab3c7>@@@Z 000000018001972c     libucrt:per_thread_data.obj
 0003:00000738       $pdata$?construct_ptd_array@@YAXQEAU__acrt_ptd@@@Z 0000000180019738     libucrt:per_thread_data.obj
 0003:00000744       $pdata$?destroy_fls@@YAXPEAX@Z 0000000180019744     libucrt:per_thread_data.obj
 0003:00000750       $pdata$?destroy_ptd_array@@YAXQEAU__acrt_ptd@@@Z 0000000180019750     libucrt:per_thread_data.obj
 0003:0000075c       $pdata$?replace_current_thread_locale_nolock@@YAXQEAU__acrt_ptd@@QEAU__crt_locale_data@@@Z 000000018001975c     libucrt:per_thread_data.obj
 0003:00000768       $pdata$__acrt_freeptd      0000000180019768     libucrt:per_thread_data.obj
 0003:00000774       $pdata$__acrt_getptd       0000000180019774     libucrt:per_thread_data.obj
 0003:00000780       $pdata$__acrt_getptd_head  0000000180019780     libucrt:per_thread_data.obj
 0003:0000078c       $pdata$__acrt_getptd_noexit 000000018001978c     libucrt:per_thread_data.obj
 0003:00000798       $pdata$__acrt_initialize_ptd 0000000180019798     libucrt:per_thread_data.obj
 0003:000007a4       $pdata$__acrt_uninitialize_ptd 00000001800197a4     libucrt:per_thread_data.obj
 0003:000007b0       $pdata$__acrt_get_process_end_policy 00000001800197b0     libucrt:win_policies.obj
 0003:000007bc       $pdata$__acrt_call_reportfault 00000001800197bc     libucrt:invalid_parameter.obj
 0003:000007c8       $pdata$_invalid_parameter  00000001800197c8     libucrt:invalid_parameter.obj
 0003:000007d4       $pdata$_invalid_parameter_noinfo 00000001800197d4     libucrt:invalid_parameter.obj
 0003:000007e0       $pdata$_invoke_watson      00000001800197e0     libucrt:invalid_parameter.obj
 0003:000007ec       $pdata$__acrt_errno_map_os_error 00000001800197ec     libucrt:errno.obj
 0003:000007f8       $pdata$__doserrno          00000001800197f8     libucrt:errno.obj
 0003:00000804       $pdata$_errno              0000000180019804     libucrt:errno.obj
 0003:00000810       $pdata$_calloc_base        0000000180019810     libucrt:calloc_base.obj
 0003:0000081c       $pdata$??$__acrt_mbs_to_wcs_cp@U__crt_win32_buffer_internal_dynamic_resizing@@@@YAHQEBDAEAV?$__crt_win32_buffer@_WU__crt_win32_buffer_internal_dynamic_resizing@@@@I@Z 000000018001981c     libucrt:argv_wildcards.obj
 0003:00000828       $pdata$??$__acrt_wcs_to_mbs_cp@U__crt_win32_buffer_internal_dynamic_resizing@@@@YAHQEB_WAEAV?$__crt_win32_buffer@DU__crt_win32_buffer_internal_dynamic_resizing@@@@I@Z 0000000180019828     libucrt:argv_wildcards.obj
 0003:00000834       $pdata$??$common_expand_argv_wildcards@D@@YAHQEAPEADQEAPEAPEAD@Z 0000000180019834     libucrt:argv_wildcards.obj
 0003:00000840       $pdata$??$copy_and_add_argument_to_buffer@D@@YAHQEBD0_KAEAV?$argument_list@D@?A0x5f5c8891@@@Z 0000000180019840     libucrt:argv_wildcards.obj
 0003:0000084c       $pdata$??$expand_argument_wildcards@D@@YAHQEAD0AEAV?$argument_list@D@?A0x5f5c8891@@@Z 000000018001984c     libucrt:argv_wildcards.obj
 0003:00000858       $pdata$??$__acrt_wcs_to_mbs_cp@U__crt_win32_buffer_no_resizing@@@@YAHQEB_WAEAV?$__crt_win32_buffer@DU__crt_win32_buffer_no_resizing@@@@I@Z 0000000180019858     libucrt:getmodulefilenamea.obj
 0003:00000864       $pdata$__acrt_GetModuleFileNameA 0000000180019864     libucrt:getmodulefilenamea.obj
 0003:00000870       $pdata$??$?RV<lambda_efdfa57d1f175319df784efa44bb7b81>@@AEAV<lambda_5f0a4c1567f8adc6734073e5d1e1b35c>@@V<lambda_2e8a7d3640ea6ccb4c2413664c2db6fd>@@@?$__crt_seh_guarded_call@X@@QEAAX$$QEAV<lambda_efdfa57d1f175319df784efa44bb7b81>@@AEAV<lambda_5f0a4c1567f8adc6734073e5d1e1b35c>@@$$QEAV<lambda_2e8a7d3640ea6ccb4c2413664c2db6fd>@@@Z 0000000180019870     libucrt:mbctype.obj
 0003:0000087c       $pdata$?getSystemCP@@YAHH@Z 000000018001987c     libucrt:mbctype.obj
 0003:00000888       $pdata$?setSBCS@@YAXPEAU__crt_multibyte_data@@@Z 0000000180019888     libucrt:mbctype.obj
 0003:00000894       $pdata$?setSBUpLow@@YAXPEAU__crt_multibyte_data@@@Z 0000000180019894     libucrt:mbctype.obj
 0003:000008a0       $pdata$?setmbcp_internal@@YAHH_NQEAU__acrt_ptd@@QEAPEAU__crt_multibyte_data@@@Z 00000001800198a0     libucrt:mbctype.obj
 0003:000008ac       $pdata$?update_thread_multibyte_data_internal@@YAPEAU__crt_multibyte_data@@QEAU__acrt_ptd@@QEAPEAU1@@Z 00000001800198ac     libucrt:mbctype.obj
 0003:000008b8       $pdata$__acrt_initialize_multibyte 00000001800198b8     libucrt:mbctype.obj
 0003:000008c4       $pdata$__acrt_update_thread_multibyte_data 00000001800198c4     libucrt:mbctype.obj
 0003:000008d0       $pdata$_setmbcp_nolock     00000001800198d0     libucrt:mbctype.obj
 0003:000008dc       $pdata$?x_ismbbtype_l@@YAHPEAU__crt_locale_pointers@@IHH@Z 00000001800198dc     libucrt:ismbbyte.obj
 0003:000008e8       $pdata$__acrt_initialize_command_line 00000001800198e8     libucrt:argv_data.obj
 0003:000008f4       $pdata$__acrt_WideCharToMultiByte 00000001800198f4     libucrt:widechartomultibyte.obj
 0003:00000900       $pdata$__dcrt_get_narrow_environment_from_os 0000000180019900     libucrt:get_environment_from_os.obj
 0003:0000090c       $pdata$_recalloc_base      000000018001990c     libucrt:recalloc.obj
 0003:00000918       $pdata$?try_get_function@@YAPEAXW4function_id@?A0x391cf84c@@QEBDQEBW4module_id@2@2@Z 0000000180019918     libucrt:winapi_thunks.obj
 0003:00000924       $pdata$__acrt_AppPolicyGetProcessTerminationMethodInternal 0000000180019924     libucrt:winapi_thunks.obj
 0003:00000930       $pdata$__acrt_AreFileApisANSI 0000000180019930     libucrt:winapi_thunks.obj
 0003:0000093c       $pdata$__acrt_FlsAlloc     000000018001993c     libucrt:winapi_thunks.obj
 0003:00000948       $pdata$__acrt_FlsFree      0000000180019948     libucrt:winapi_thunks.obj
 0003:00000954       $pdata$__acrt_FlsGetValue  0000000180019954     libucrt:winapi_thunks.obj
 0003:00000960       $pdata$__acrt_FlsSetValue  0000000180019960     libucrt:winapi_thunks.obj
 0003:0000096c       $pdata$__acrt_InitializeCriticalSectionEx 000000018001996c     libucrt:winapi_thunks.obj
 0003:00000978       $pdata$__acrt_LCMapStringEx 0000000180019978     libucrt:winapi_thunks.obj
 0003:00000984       $pdata$__acrt_LocaleNameToLCID 0000000180019984     libucrt:winapi_thunks.obj
 0003:00000990       $pdata$__acrt_initialize_winapi_thunks 0000000180019990     libucrt:winapi_thunks.obj
 0003:0000099c       $pdata$__acrt_uninitialize_winapi_thunks 000000018001999c     libucrt:winapi_thunks.obj
 0003:000009a8       $pdata$__acrt_initialize_heap 00000001800199a8     libucrt:heap_handle.obj
 0003:000009b4       $pdata$?initialize_inherited_file_handles_nolock@@YAXXZ 00000001800199b4     libucrt:ioinit.obj
 0003:000009c0       $pdata$?initialize_stdio_handles_nolock@@YAXXZ 00000001800199c0     libucrt:ioinit.obj
 0003:000009cc       $pdata$__acrt_initialize_lowio 00000001800199cc     libucrt:ioinit.obj
 0003:000009d8       $pdata$__acrt_uninitialize_lowio 00000001800199d8     libucrt:ioinit.obj
 0003:000009e4       $pdata$__acrt_execute_initializers 00000001800199e4     libucrt:shared_initialization.obj
 0003:000009f0       $pdata$__acrt_execute_uninitializers 00000001800199f0     libucrt:shared_initialization.obj
 0003:000009fc       $pdata$??$?RV<lambda_450d765d439847d4c735a33c368b5fc0>@@AEAV<lambda_44731a7d0e6d81c3e6aa82d741081786>@@V<lambda_601a2a7da3b7a96e9554ac7215c4b07c>@@@?$__crt_seh_guarded_call@P6AXH@Z@@QEAAP6AXH@Z$$QEAV<lambda_450d765d439847d4c735a33c368b5fc0>@@AEAV<lambda_44731a7d0e6d81c3e6aa82d741081786>@@$$QEAV<lambda_601a2a7da3b7a96e9554ac7215c4b07c>@@@Z 00000001800199fc     libucrt:signal.obj
 0003:00000a08       $pdata$__acrt_get_sigabrt_handler 0000000180019a08     libucrt:signal.obj
 0003:00000a14       $pdata$raise               0000000180019a14     libucrt:signal.obj
 0003:00000a20       $pdata$??$?RV<lambda_842d9ff0dc9ef11c61343bbaebe7f885>@@AEAV<lambda_c5860995281e5c4ce005b3de8f5874ee>@@V<lambda_d90129c13df834fdcbf8d2b88dafcf2d>@@@?$__crt_seh_guarded_call@X@@QEAAX$$QEAV<lambda_842d9ff0dc9ef11c61343bbaebe7f885>@@AEAV<lambda_c5860995281e5c4ce005b3de8f5874ee>@@$$QEAV<lambda_d90129c13df834fdcbf8d2b88dafcf2d>@@@Z 0000000180019a20     libucrt:fflush.obj
 0003:00000a2c       $pdata$??$?RV<lambda_886d6c58226a84441f68b9f2b8217b83>@@AEAV<lambda_ab61a845afdef5b7c387490eaf3616ee>@@V<lambda_f7f22ab5edc0698d5f6905b0d3f44752>@@@?$__crt_seh_guarded_call@X@@QEAAX$$QEAV<lambda_886d6c58226a84441f68b9f2b8217b83>@@AEAV<lambda_ab61a845afdef5b7c387490eaf3616ee>@@$$QEAV<lambda_f7f22ab5edc0698d5f6905b0d3f44752>@@@Z 0000000180019a2c     libucrt:fflush.obj
 0003:00000a38       $pdata$?common_flush_all@@YAH_N@Z 0000000180019a38     libucrt:fflush.obj
 0003:00000a44       $pdata$__acrt_stdio_flush_nolock 0000000180019a44     libucrt:fflush.obj
 0003:00000a50       $pdata$_fflush_nolock      0000000180019a50     libucrt:fflush.obj
 0003:00000a5c       $pdata$__acrt_initialize_stdio 0000000180019a5c     libucrt:_file.obj
 0003:00000a68       $pdata$__acrt_uninitialize_stdio 0000000180019a68     libucrt:_file.obj
 0003:00000a74       $pdata$_mbtowc_l           0000000180019a74     libucrt:mbtowc.obj
 0003:00000a80       $pdata$__acrt_update_locale_info 0000000180019a80     libucrt:locale_update.obj
 0003:00000a8c       $pdata$__acrt_update_multibyte_info 0000000180019a8c     libucrt:locale_update.obj
 0003:00000a98       $pdata$_fileno             0000000180019a98     libucrt:fileno.obj
 0003:00000aa4       $pdata$??$?RV<lambda_410d79af7f07d98d83a3f525b3859a53>@@AEAV<lambda_3e16ef9562a7dcce91392c22ab16ea36>@@V<lambda_38119f0e861e05405d8a144b9b982f0a>@@@?$__crt_seh_guarded_call@X@@QEAAX$$QEAV<lambda_410d79af7f07d98d83a3f525b3859a53>@@AEAV<lambda_3e16ef9562a7dcce91392c22ab16ea36>@@$$QEAV<lambda_38119f0e861e05405d8a144b9b982f0a>@@@Z 0000000180019aa4     libucrt:wsetlocale.obj
 0003:00000ab0       $pdata$__acrt_uninitialize_locale 0000000180019ab0     libucrt:wsetlocale.obj
 0003:00000abc       $pdata$__pctype_func       0000000180019abc     libucrt:ctype.obj
 0003:00000ac8       $pdata$__acrt_free_locale  0000000180019ac8     libucrt:locale_refcounting.obj
 0003:00000ad4       $pdata$__acrt_locale_free_lc_time_if_unreferenced 0000000180019ad4     libucrt:locale_refcounting.obj
 0003:00000ae0       $pdata$__acrt_release_locale_ref 0000000180019ae0     libucrt:locale_refcounting.obj
 0003:00000aec       $pdata$__acrt_update_thread_locale_data 0000000180019aec     libucrt:locale_refcounting.obj
 0003:00000af8       $pdata$_updatetlocinfoEx_nolock 0000000180019af8     libucrt:locale_refcounting.obj
 0003:00000b04       $pdata$qsort               0000000180019b04     libucrt:qsort.obj
 0003:00000b10       $pdata$4$qsort             0000000180019b10     libucrt:qsort.obj
 0003:00000b1c       $pdata$5$qsort             0000000180019b1c     libucrt:qsort.obj
 0003:00000b28       $pdata$strncpy_s           0000000180019b28     libucrt:strncpy_s.obj
 0003:00000b34       $pdata$fallbackMethod      0000000180019b34     libucrt:strpbrk.obj
 0003:00000b40       $pdata$strpbrk             0000000180019b40     libucrt:strpbrk.obj
 0003:00000b4c       $pdata$_mbsdec_l           0000000180019b4c     libucrt:mbsdec.obj
 0003:00000b58       $pdata$__acrt_GetStringTypeA 0000000180019b58     libucrt:getstringtypea.obj
 0003:00000b64       $pdata$?__acrt_LCMapStringA_stat@@YAHPEAU__crt_locale_pointers@@PEB_WKPEBDHPEADHHH@Z 0000000180019b64     libucrt:lcmapstringa.obj
 0003:00000b70       $pdata$__acrt_LCMapStringA 0000000180019b70     libucrt:lcmapstringa.obj
 0003:00000b7c       $pdata$?initialize_multibyte@@YAHXZ 0000000180019b7c     libucrt:multibyte_initializer.obj
 0003:00000b88       $pdata$_msize_base         0000000180019b88     libucrt:msize.obj
 0003:00000b94       $pdata$_realloc_base       0000000180019b94     libucrt:realloc_base.obj
 0003:00000ba0       $pdata$?GetTableIndexFromLocaleName@@YAHPEB_W@Z 0000000180019ba0     libucrt:lcidtoname_downlevel.obj
 0003:00000bac       $pdata$__acrt_DownlevelLocaleNameToLCID 0000000180019bac     libucrt:lcidtoname_downlevel.obj
 0003:00000bb8       $pdata$__acrt_lowio_create_handle_array 0000000180019bb8     libucrt:osfinfo.obj
 0003:00000bc4       $pdata$__acrt_lowio_destroy_handle_array 0000000180019bc4     libucrt:osfinfo.obj
 0003:00000bd0       $pdata$__acrt_lowio_ensure_fh_exists 0000000180019bd0     libucrt:osfinfo.obj
 0003:00000bdc       $pdata$_free_osfhnd        0000000180019bdc     libucrt:osfinfo.obj
 0003:00000be8       $pdata$_get_osfhandle      0000000180019be8     libucrt:osfinfo.obj
 0003:00000bf4       $pdata$??$?RV<lambda_a37b2b86f63e897a80ea819b0eb08c01>@@AEAV<lambda_38ce7e780aa69e748d6df282ebc68efe>@@V<lambda_99fb1378e971ab6e7edea83e3a7a83a2>@@@?$__crt_seh_guarded_call@H@@QEAAH$$QEAV<lambda_a37b2b86f63e897a80ea819b0eb08c01>@@AEAV<lambda_38ce7e780aa69e748d6df282ebc68efe>@@$$QEAV<lambda_99fb1378e971ab6e7edea83e3a7a83a2>@@@Z 0000000180019bf4     libucrt:commit.obj
 0003:00000c00       $pdata$_commit             0000000180019c00     libucrt:commit.obj
 0003:00000c0c       $pdata$?write_double_translated_ansi_nolock@@YA?AUwrite_result@?A0x17268360@@HQEBDI@Z 0000000180019c0c     libucrt:write.obj
 0003:00000c18       $pdata$?write_text_ansi_nolock@@YA?AUwrite_result@?A0x17268360@@HQEBDI@Z 0000000180019c18     libucrt:write.obj
 0003:00000c24       $pdata$?write_text_utf16le_nolock@@YA?AUwrite_result@?A0x17268360@@HQEBDI@Z 0000000180019c24     libucrt:write.obj
 0003:00000c30       $pdata$?write_text_utf8_nolock@@YA?AUwrite_result@?A0x17268360@@HQEBDI@Z 0000000180019c30     libucrt:write.obj
 0003:00000c3c       $pdata$_write              0000000180019c3c     libucrt:write.obj
 0003:00000c48       $pdata$_write_nolock       0000000180019c48     libucrt:write.obj
 0003:00000c54       $pdata$_fcloseall          0000000180019c54     libucrt:closeall.obj
 0003:00000c60       $pdata$__acrt_stdio_free_buffer_nolock 0000000180019c60     libucrt:_freebuf.obj
 0003:00000c6c       $pdata$_isatty             0000000180019c6c     libucrt:isatty.obj
 0003:00000c78       $pdata$_isleadbyte_l       0000000180019c78     libucrt:_wctype.obj
 0003:00000c84       $pdata$?__mbrtowc_utf8@__crt_mbstring@@YA_KPEA_WPEBD_KPEAU_Mbstatet@@@Z 0000000180019c84     libucrt:mbrtowc.obj
 0003:00000c90       $pdata$?__mbsrtowcs_utf8@__crt_mbstring@@YA_KPEA_WPEAPEBD_KPEAU_Mbstatet@@@Z 0000000180019c90     libucrt:mbrtowc.obj
 0003:00000c9c       $pdata$__acrt_locale_free_monetary 0000000180019c9c     libucrt:initmon.obj
 0003:00000ca8       $pdata$__acrt_locale_free_numeric 0000000180019ca8     libucrt:initnum.obj
 0003:00000cb4       $pdata$?free_crt_array_internal@@YAXQEAPEBX_K@Z 0000000180019cb4     libucrt:inittime.obj
 0003:00000cc0       $pdata$__acrt_locale_free_time 0000000180019cc0     libucrt:inittime.obj
 0003:00000ccc       $pdata$??$common_lseek_nolock@_J@@YA_JH_JH@Z 0000000180019ccc     libucrt:lseek.obj
 0003:00000cd8       $pdata$_putwch_nolock      0000000180019cd8     libucrt:putwch.obj
 0003:00000ce4       $pdata$_fclose_nolock      0000000180019ce4     libucrt:fclose.obj
 0003:00000cf0       $pdata$fclose              0000000180019cf0     libucrt:fclose.obj
 0003:00000cfc       $pdata$?__mbrtoc32_utf8@__crt_mbstring@@YA_KPEA_UPEBD_KPEAU_Mbstatet@@@Z 0000000180019cfc     libucrt:mbrtoc32.obj
 0003:00000d14       $pdata$__dcrt_lowio_ensure_console_output_initialized 0000000180019d14     libucrt:initcon.obj
 0003:00000d20       $pdata$__dcrt_terminate_console_output 0000000180019d20     libucrt:initcon.obj
 0003:00000d2c       $pdata$__dcrt_write_console 0000000180019d2c     libucrt:initcon.obj
 0003:00000d38       $pdata$??$?RV<lambda_751a882b2c74d4b022dec766aa51a29a>@@AEAV<lambda_628dfdc04ba53c8bfc02c9951375f3f5>@@V<lambda_f6c7be5f7998530c34de24c7437d6b54>@@@?$__crt_seh_guarded_call@H@@QEAAH$$QEAV<lambda_751a882b2c74d4b022dec766aa51a29a>@@AEAV<lambda_628dfdc04ba53c8bfc02c9951375f3f5>@@$$QEAV<lambda_f6c7be5f7998530c34de24c7437d6b54>@@@Z 0000000180019d38     libucrt:close.obj
 0003:00000d44       $pdata$_close              0000000180019d44     libucrt:close.obj
 0003:00000d50       $pdata$_close_nolock       0000000180019d50     libucrt:close.obj
 0003:00000d5c       $pdata$_call_matherr       0000000180019d5c     libucrt:libm_error.obj
 0003:00000d68       $pdata$_exception_enabled  0000000180019d68     libucrt:libm_error.obj
 0003:00000d74       $pdata$_handle_error       0000000180019d74     libucrt:libm_error.obj
 0003:00000d80       $pdata$__acrt_initialize_fma3 0000000180019d80     libucrt:fma3_available.obj
 0003:00000d8c       $pdata$_log10_special      0000000180019d8c     libucrt:log_special.obj
 0003:00000d98       $pdata$_log_special_common 0000000180019d98     libucrt:log_special.obj
 0003:00000db0       $pdata$_raise_exc          0000000180019db0     libucrt:fpexcept.obj
 0003:00000dbc       $pdata$_raise_exc_ex       0000000180019dbc     libucrt:fpexcept.obj
 0003:00000dc8       $pdata$_set_errno_from_matherr 0000000180019dc8     libucrt:fpexcept.obj
 0003:00000dd4       $pdata$_clrfp              0000000180019dd4     libucrt:fpctrl.obj
 0003:00000de0       $pdata$_ctrlfp             0000000180019de0     libucrt:fpctrl.obj
 0003:00000dec       $pdata$_set_statfp         0000000180019dec     libucrt:fpctrl.obj
 0003:00000df8       $pdata$_statfp             0000000180019df8     libucrt:fpctrl.obj
 0003:00000e04       $pdata$_IsNonwritableInCurrentImage 0000000180019e04     LIBCMT:pesect.obj
 0003:00000e10       $pdata$__GSHandlerCheck    0000000180019e10     LIBCMT:gshandler.obj
 0003:00000e1c       $pdata$__GSHandlerCheckCommon 0000000180019e1c     LIBCMT:gshandler.obj
 0003:00000e34       $pdata$__raise_securityfailure 0000000180019e34     LIBCMT:gs_report.obj
 0003:00000e40       $pdata$__report_gsfailure  0000000180019e40     LIBCMT:gs_report.obj
 0003:00000e4c       $pdata$__report_rangecheckfailure 0000000180019e4c     LIBCMT:gs_report.obj
 0003:00000e58       $pdata$__report_securityfailure 0000000180019e58     LIBCMT:gs_report.obj
 0003:00000e64       $pdata$capture_current_context 0000000180019e64     LIBCMT:gs_report.obj
 0003:00000e70       $pdata$capture_previous_context 0000000180019e70     LIBCMT:gs_report.obj
 0003:00000e94       $pdata$?fin$0@?0??dllmain_crt_process_attach@@YAHQEAUHINSTANCE__@@QEAX@Z@4HA 0000000180019e94     LIBCMT:dll_dllmain.obj
 0003:00000ea0       $pdata$?fin$0@?0??dllmain_crt_process_detach@@YAH_N@Z@4HA 0000000180019ea0     LIBCMT:dll_dllmain.obj
 0003:00000eac       $pdata$?filt$0@?0??dllmain_dispatch@@YAHQEAUHINSTANCE__@@KQEAX@Z@4HA 0000000180019eac     LIBCMT:dll_dllmain.obj
 0003:00000eb8       $pdata$__scrt_is_nonwritable_in_current_image$filt$0 0000000180019eb8     LIBCMT:utility.obj
 0003:00000ec4       $pdata$__DestructExceptionObject$filt$0 0000000180019ec4     libvcruntime:ehhelpers.obj
 0003:00000ed0       $pdata$_query_new_handler$fin$0 0000000180019ed0     libucrt:new_handler.obj
 0003:00000edc       $pdata$?fin$0@?0???$?RV<lambda_7777bce6b2f8c936911f934f8298dc43>@@AEAV<lambda_f03950bc5685219e0bcd2087efbe011e>@@V<lambda_3883c3dff614d5e0c5f61bb1ac94921c>@@@?$__crt_seh_guarded_call@H@@QEAAH$$QEAV<lambda_7777bce6b2f8c936911f934f8298dc43>@@AEAV<lambda_f03950bc5685219e0bcd2087efbe011e>@@$$QEAV<lambda_3883c3dff614d5e0c5f61bb1ac94921c>@@@Z@4HA 0000000180019edc     libucrt:onexit.obj
 0003:00000edc       $pdata$?fin$0@?0???$?RV<lambda_2d41944a1d46af3157314b8a01080d33>@@AEAV<lambda_8f455de75cd7d7f24b4096f044d8b9e6>@@V<lambda_aa500f224e6afead328df44964fe2772>@@@?$__crt_seh_guarded_call@X@@QEAAX$$QEAV<lambda_2d41944a1d46af3157314b8a01080d33>@@AEAV<lambda_8f455de75cd7d7f24b4096f044d8b9e6>@@$$QEAV<lambda_aa500f224e6afead328df44964fe2772>@@@Z@4HA 0000000180019edc     libucrt:per_thread_data.obj
 0003:00000edc       $pdata$?fin$0@?0???$?RV<lambda_0ae27a3a962d80f24befdcbee591983d>@@AEAV<lambda_8d0ee55de4b1038c4002e0adecdf1839>@@V<lambda_dc504788e8f1664fe9b84e20bfb512f2>@@@?$__crt_seh_guarded_call@X@@QEAAX$$QEAV<lambda_0ae27a3a962d80f24befdcbee591983d>@@AEAV<lambda_8d0ee55de4b1038c4002e0adecdf1839>@@$$QEAV<lambda_dc504788e8f1664fe9b84e20bfb512f2>@@@Z@4HA 0000000180019edc     libucrt:per_thread_data.obj
 0003:00000edc       $pdata$?fin$0@?0???$?RV<lambda_d80eeec6fff315bfe5c115232f3240e3>@@AEAV<lambda_6e4b09c48022b2350581041d5f6b0c4c>@@V<lambda_2358e3775559c9db80273638284d5e45>@@@?$__crt_seh_guarded_call@X@@QEAAX$$QEAV<lambda_d80eeec6fff315bfe5c115232f3240e3>@@AEAV<lambda_6e4b09c48022b2350581041d5f6b0c4c>@@$$QEAV<lambda_2358e3775559c9db80273638284d5e45>@@@Z@4HA 0000000180019edc     libucrt:exit.obj
 0003:00000edc       $pdata$?fin$0@?0???$?RV<lambda_450d765d439847d4c735a33c368b5fc0>@@AEAV<lambda_44731a7d0e6d81c3e6aa82d741081786>@@V<lambda_601a2a7da3b7a96e9554ac7215c4b07c>@@@?$__crt_seh_guarded_call@P6AXH@Z@@QEAAP6AXH@Z$$QEAV<lambda_450d765d439847d4c735a33c368b5fc0>@@AEAV<lambda_44731a7d0e6d81c3e6aa82d741081786>@@$$QEAV<lambda_601a2a7da3b7a96e9554ac7215c4b07c>@@@Z@4HA 0000000180019edc     libucrt:signal.obj
 0003:00000edc       $pdata$?fin$0@?0???$?RV<lambda_aa87e3671a710a21b5dc78c0bdf72e11>@@AEAV<lambda_92619d2358a28f41a33ba319515a20b9>@@V<lambda_6992ecaafeb10aed2b74cb1fae11a551>@@@?$__crt_seh_guarded_call@X@@QEAAX$$QEAV<lambda_aa87e3671a710a21b5dc78c0bdf72e11>@@AEAV<lambda_92619d2358a28f41a33ba319515a20b9>@@$$QEAV<lambda_6992ecaafeb10aed2b74cb1fae11a551>@@@Z@4HA 0000000180019edc     libucrt:per_thread_data.obj
 0003:00000edc       $pdata$?fin$0@?0???$?RV<lambda_efdfa57d1f175319df784efa44bb7b81>@@AEAV<lambda_5f0a4c1567f8adc6734073e5d1e1b35c>@@V<lambda_2e8a7d3640ea6ccb4c2413664c2db6fd>@@@?$__crt_seh_guarded_call@X@@QEAAX$$QEAV<lambda_efdfa57d1f175319df784efa44bb7b81>@@AEAV<lambda_5f0a4c1567f8adc6734073e5d1e1b35c>@@$$QEAV<lambda_2e8a7d3640ea6ccb4c2413664c2db6fd>@@@Z@4HA 0000000180019edc     libucrt:mbctype.obj
 0003:00000edc       $pdata$?fin$0@?0???$?RV<lambda_f2e299630e499de9f9a165e60fcd3db5>@@AEAV<lambda_2ae9d31cdba2644fcbeaf08da7c24588>@@V<lambda_40d01ff24d0e7b3814fdbdcee8eab3c7>@@@?$__crt_seh_guarded_call@X@@QEAAX$$QEAV<lambda_f2e299630e499de9f9a165e60fcd3db5>@@AEAV<lambda_2ae9d31cdba2644fcbeaf08da7c24588>@@$$QEAV<lambda_40d01ff24d0e7b3814fdbdcee8eab3c7>@@@Z@4HA 0000000180019edc     libucrt:per_thread_data.obj
 0003:00000ee8       $pdata$?filt$0@?0???R<lambda_6e4b09c48022b2350581041d5f6b0c4c>@@QEBA@XZ@4HA 0000000180019ee8     libucrt:exit.obj
 0003:00000ef4       $pdata$?fin$0@?0??update_thread_multibyte_data_internal@@YAPEAU__crt_multibyte_data@@QEAU__acrt_ptd@@QEAPEAU1@@Z@4HA 0000000180019ef4     libucrt:mbctype.obj
 0003:00000f00       $pdata$__acrt_initialize_lowio$fin$0 0000000180019f00     libucrt:ioinit.obj
 0003:00000f00       $pdata$__acrt_lowio_ensure_fh_exists$fin$0 0000000180019f00     libucrt:osfinfo.obj
 0003:00000f0c       $pdata$raise$fin$0         0000000180019f0c     libucrt:signal.obj
 0003:00000f18       $pdata$?fin$0@?0???$?RV<lambda_842d9ff0dc9ef11c61343bbaebe7f885>@@AEAV<lambda_c5860995281e5c4ce005b3de8f5874ee>@@V<lambda_d90129c13df834fdcbf8d2b88dafcf2d>@@@?$__crt_seh_guarded_call@X@@QEAAX$$QEAV<lambda_842d9ff0dc9ef11c61343bbaebe7f885>@@AEAV<lambda_c5860995281e5c4ce005b3de8f5874ee>@@$$QEAV<lambda_d90129c13df834fdcbf8d2b88dafcf2d>@@@Z@4HA 0000000180019f18     libucrt:fflush.obj
 0003:00000f24       $pdata$?fin$0@?0???$?RV<lambda_886d6c58226a84441f68b9f2b8217b83>@@AEAV<lambda_ab61a845afdef5b7c387490eaf3616ee>@@V<lambda_f7f22ab5edc0698d5f6905b0d3f44752>@@@?$__crt_seh_guarded_call@X@@QEAAX$$QEAV<lambda_886d6c58226a84441f68b9f2b8217b83>@@AEAV<lambda_ab61a845afdef5b7c387490eaf3616ee>@@$$QEAV<lambda_f7f22ab5edc0698d5f6905b0d3f44752>@@@Z@4HA 0000000180019f24     libucrt:fflush.obj
 0003:00000f30       $pdata$?fin$0@?0???$?RV<lambda_410d79af7f07d98d83a3f525b3859a53>@@AEAV<lambda_3e16ef9562a7dcce91392c22ab16ea36>@@V<lambda_38119f0e861e05405d8a144b9b982f0a>@@@?$__crt_seh_guarded_call@X@@QEAAX$$QEAV<lambda_410d79af7f07d98d83a3f525b3859a53>@@AEAV<lambda_3e16ef9562a7dcce91392c22ab16ea36>@@$$QEAV<lambda_38119f0e861e05405d8a144b9b982f0a>@@@Z@4HA 0000000180019f30     libucrt:wsetlocale.obj
 0003:00000f3c       $pdata$__acrt_update_thread_locale_data$fin$0 0000000180019f3c     libucrt:locale_refcounting.obj
 0003:00000f48       $pdata$?fin$0@?0???$?RV<lambda_751a882b2c74d4b022dec766aa51a29a>@@AEAV<lambda_628dfdc04ba53c8bfc02c9951375f3f5>@@V<lambda_f6c7be5f7998530c34de24c7437d6b54>@@@?$__crt_seh_guarded_call@H@@QEAAH$$QEAV<lambda_751a882b2c74d4b022dec766aa51a29a>@@AEAV<lambda_628dfdc04ba53c8bfc02c9951375f3f5>@@$$QEAV<lambda_f6c7be5f7998530c34de24c7437d6b54>@@@Z@4HA 0000000180019f48     libucrt:close.obj
 0003:00000f48       $pdata$?fin$0@?0???$?RV<lambda_a37b2b86f63e897a80ea819b0eb08c01>@@AEAV<lambda_38ce7e780aa69e748d6df282ebc68efe>@@V<lambda_99fb1378e971ab6e7edea83e3a7a83a2>@@@?$__crt_seh_guarded_call@H@@QEAAH$$QEAV<lambda_a37b2b86f63e897a80ea819b0eb08c01>@@AEAV<lambda_38ce7e780aa69e748d6df282ebc68efe>@@$$QEAV<lambda_99fb1378e971ab6e7edea83e3a7a83a2>@@@Z@4HA 0000000180019f48     libucrt:commit.obj
 0003:00000f54       $pdata$_write$fin$0        0000000180019f54     libucrt:write.obj
 0003:00000f60       $pdata$_fcloseall$fin$0    0000000180019f60     libucrt:closeall.obj
 0003:00000f6c       $pdata$fclose$fin$0        0000000180019f6c     libucrt:fclose.obj
 0003:00000f78       $pdata$_ctrlfp$filt$0      0000000180019f78     libucrt:fpctrl.obj
 0003:00000f84       $pdata$_IsNonwritableInCurrentImage$filt$0 0000000180019f84     LIBCMT:pesect.obj
 0004:000004b0       .idata$6                   000000018001a4b0     kernel32:KERNEL32.dll
 0005:00000060       $R000000                   000000018001b060     SameFolder.res
